Component: Arm Compiler for Embedded 6.21 Tool: armlink [5ec1fa00]

==============================================================================

Section Cross References

    startup_stm32f030xc.o(STACK) refers (Special) to heapauxi.o(.text) for __use_two_region_memory
    startup_stm32f030xc.o(HEAP) refers (Special) to heapauxi.o(.text) for __use_two_region_memory
    startup_stm32f030xc.o(RESET) refers (Special) to heapauxi.o(.text) for __use_two_region_memory
    startup_stm32f030xc.o(RESET) refers to startup_stm32f030xc.o(STACK) for __initial_sp
    startup_stm32f030xc.o(RESET) refers to startup_stm32f030xc.o(.text) for Reset_Handler
    startup_stm32f030xc.o(RESET) refers to stm32f0xx_it.o(.text.NMI_Handler) for NMI_Handler
    startup_stm32f030xc.o(RESET) refers to stm32f0xx_it.o(.text.HardFault_Handler) for HardFault_Handler
    startup_stm32f030xc.o(RESET) refers to stm32f0xx_it.o(.text.SVC_Handler) for SVC_Handler
    startup_stm32f030xc.o(RESET) refers to stm32f0xx_it.o(.text.PendSV_Handler) for PendSV_Handler
    startup_stm32f030xc.o(RESET) refers to stm32f0xx_it.o(.text.SysTick_Handler) for SysTick_Handler
    startup_stm32f030xc.o(.text) refers (Special) to heapauxi.o(.text) for __use_two_region_memory
    startup_stm32f030xc.o(.text) refers to system_stm32f0xx.o(.text.SystemInit) for SystemInit
    startup_stm32f030xc.o(.text) refers to __main.o(!!!main) for __main
    startup_stm32f030xc.o(.text) refers to startup_stm32f030xc.o(HEAP) for Heap_Mem
    startup_stm32f030xc.o(.text) refers to startup_stm32f030xc.o(STACK) for Stack_Mem
    main.o(.text) refers (Special) to _printf_percent.o(.ARM.Collect$$_printf_percent$$00000000) for _printf_percent
    main.o(.text) refers (Special) to _printf_pad.o(.text) for _printf_pre_padding
    main.o(.text) refers (Special) to _printf_c.o(.ARM.Collect$$_printf_percent$$00000013) for _printf_c
    main.o(.text) refers (Special) to _printf_s.o(.ARM.Collect$$_printf_percent$$00000014) for _printf_s
    main.o(.text) refers (Special) to _printf_x.o(.ARM.Collect$$_printf_percent$$0000000C) for _printf_x
    main.o(.text) refers (Special) to _printf_f.o(.ARM.Collect$$_printf_percent$$00000003) for _printf_f
    main.o(.text) refers (Special) to _printf_hex_int.o(.text) for _printf_longlong_hex
    main.o(.text) refers (Special) to printf1.o(x$fpl$printf1) for _printf_fp_dec
    main.o(.text) refers (Special) to _printf_str.o(.text) for _printf_str
    main.o(.text.main) refers (Special) to _printf_percent.o(.ARM.Collect$$_printf_percent$$00000000) for _printf_percent
    main.o(.text.main) refers (Special) to _printf_pad.o(.text) for _printf_pre_padding
    main.o(.text.main) refers (Special) to _printf_c.o(.ARM.Collect$$_printf_percent$$00000013) for _printf_c
    main.o(.text.main) refers (Special) to _printf_s.o(.ARM.Collect$$_printf_percent$$00000014) for _printf_s
    main.o(.text.main) refers (Special) to _printf_x.o(.ARM.Collect$$_printf_percent$$0000000C) for _printf_x
    main.o(.text.main) refers (Special) to _printf_f.o(.ARM.Collect$$_printf_percent$$00000003) for _printf_f
    main.o(.text.main) refers (Special) to _printf_hex_int.o(.text) for _printf_longlong_hex
    main.o(.text.main) refers (Special) to printf1.o(x$fpl$printf1) for _printf_fp_dec
    main.o(.text.main) refers (Special) to _printf_str.o(.text) for _printf_str
    main.o(.text.main) refers to stm32f0xx_hal.o(.text.HAL_Init) for HAL_Init
    main.o(.text.main) refers to main.o(.text.SystemClock_Config) for SystemClock_Config
    main.o(.text.main) refers to stm32f0xx_hal_i2c.o(.text.HAL_I2C_Init) for HAL_I2C_Init
    main.o(.text.main) refers to stm32f0xx_hal_i2c_ex.o(.text.HAL_I2CEx_ConfigAnalogFilter) for HAL_I2CEx_ConfigAnalogFilter
    main.o(.text.main) refers to stm32f0xx_hal_i2c_ex.o(.text.HAL_I2CEx_ConfigDigitalFilter) for HAL_I2CEx_ConfigDigitalFilter
    main.o(.text.main) refers to stm32f0xx_hal_rtc.o(.text.HAL_RTC_Init) for HAL_RTC_Init
    main.o(.text.main) refers to stm32f0xx_hal_rtc.o(.text.HAL_RTC_SetTime) for HAL_RTC_SetTime
    main.o(.text.main) refers to stm32f0xx_hal_rtc.o(.text.HAL_RTC_SetDate) for HAL_RTC_SetDate
    main.o(.text.main) refers to ssd1306.o(.text.init_OLED) for init_OLED
    main.o(.text.main) refers to ssd1306.o(.text.clear_display) for clear_display
    main.o(.text.main) refers to bmp280+aht20.o(.text.BMP280_init) for BMP280_init
    main.o(.text.main) refers to stm32f0xx_hal.o(.text.HAL_Delay) for HAL_Delay
    main.o(.text.main) refers to ssd1306.o(.text.OLCD_write_string) for OLCD_write_string
    main.o(.text.main) refers to stm32f0xx_hal_rtc.o(.text.HAL_RTC_GetTime) for HAL_RTC_GetTime
    main.o(.text.main) refers to stm32f0xx_hal_rtc.o(.text.HAL_RTC_GetDate) for HAL_RTC_GetDate
    main.o(.text.main) refers to noretval__2sprintf.o(.text) for __2sprintf
    main.o(.text.main) refers to bmp280+aht20.o(.text.AHT20_Read) for AHT20_Read
    main.o(.text.main) refers to bmp280+aht20.o(.text.BMP280_calc_values) for BMP280_calc_values
    main.o(.text.main) refers to f2d.o(.text) for __aeabi_f2d
    main.o(.text.main) refers to main.o(.bss.hi2c1) for hi2c1
    main.o(.text.main) refers to main.o(.bss..L_MergedGlobals.16) for [Anonymous Symbol]
    main.o(.text.main) refers to main.o(.data..L_MergedGlobals) for [Anonymous Symbol]
    main.o(.text.main) refers to bmp280+aht20.o(.bss..L_MergedGlobals) for BMP280_Temperature
    main.o(.ARM.exidx.text.main) refers (Special) to _printf_percent.o(.ARM.Collect$$_printf_percent$$00000000) for _printf_percent
    main.o(.ARM.exidx.text.main) refers (Special) to _printf_pad.o(.text) for _printf_pre_padding
    main.o(.ARM.exidx.text.main) refers (Special) to _printf_c.o(.ARM.Collect$$_printf_percent$$00000013) for _printf_c
    main.o(.ARM.exidx.text.main) refers (Special) to _printf_s.o(.ARM.Collect$$_printf_percent$$00000014) for _printf_s
    main.o(.ARM.exidx.text.main) refers (Special) to _printf_x.o(.ARM.Collect$$_printf_percent$$0000000C) for _printf_x
    main.o(.ARM.exidx.text.main) refers (Special) to _printf_f.o(.ARM.Collect$$_printf_percent$$00000003) for _printf_f
    main.o(.ARM.exidx.text.main) refers (Special) to _printf_hex_int.o(.text) for _printf_longlong_hex
    main.o(.ARM.exidx.text.main) refers (Special) to printf1.o(x$fpl$printf1) for _printf_fp_dec
    main.o(.ARM.exidx.text.main) refers (Special) to _printf_str.o(.text) for _printf_str
    main.o(.ARM.exidx.text.main) refers to main.o(.text.main) for [Anonymous Symbol]
    main.o(.text.SystemClock_Config) refers (Special) to _printf_percent.o(.ARM.Collect$$_printf_percent$$00000000) for _printf_percent
    main.o(.text.SystemClock_Config) refers (Special) to _printf_pad.o(.text) for _printf_pre_padding
    main.o(.text.SystemClock_Config) refers (Special) to _printf_c.o(.ARM.Collect$$_printf_percent$$00000013) for _printf_c
    main.o(.text.SystemClock_Config) refers (Special) to _printf_s.o(.ARM.Collect$$_printf_percent$$00000014) for _printf_s
    main.o(.text.SystemClock_Config) refers (Special) to _printf_x.o(.ARM.Collect$$_printf_percent$$0000000C) for _printf_x
    main.o(.text.SystemClock_Config) refers (Special) to _printf_f.o(.ARM.Collect$$_printf_percent$$00000003) for _printf_f
    main.o(.text.SystemClock_Config) refers (Special) to _printf_hex_int.o(.text) for _printf_longlong_hex
    main.o(.text.SystemClock_Config) refers (Special) to printf1.o(x$fpl$printf1) for _printf_fp_dec
    main.o(.text.SystemClock_Config) refers (Special) to _printf_str.o(.text) for _printf_str
    main.o(.text.SystemClock_Config) refers to stm32f0xx_hal_pwr.o(.text.HAL_PWR_EnableBkUpAccess) for HAL_PWR_EnableBkUpAccess
    main.o(.text.SystemClock_Config) refers to stm32f0xx_hal_rcc.o(.text.HAL_RCC_OscConfig) for HAL_RCC_OscConfig
    main.o(.text.SystemClock_Config) refers to stm32f0xx_hal_rcc.o(.text.HAL_RCC_ClockConfig) for HAL_RCC_ClockConfig
    main.o(.text.SystemClock_Config) refers to stm32f0xx_hal_rcc_ex.o(.text.HAL_RCCEx_PeriphCLKConfig) for HAL_RCCEx_PeriphCLKConfig
    main.o(.ARM.exidx.text.SystemClock_Config) refers (Special) to _printf_percent.o(.ARM.Collect$$_printf_percent$$00000000) for _printf_percent
    main.o(.ARM.exidx.text.SystemClock_Config) refers (Special) to _printf_pad.o(.text) for _printf_pre_padding
    main.o(.ARM.exidx.text.SystemClock_Config) refers (Special) to _printf_c.o(.ARM.Collect$$_printf_percent$$00000013) for _printf_c
    main.o(.ARM.exidx.text.SystemClock_Config) refers (Special) to _printf_s.o(.ARM.Collect$$_printf_percent$$00000014) for _printf_s
    main.o(.ARM.exidx.text.SystemClock_Config) refers (Special) to _printf_x.o(.ARM.Collect$$_printf_percent$$0000000C) for _printf_x
    main.o(.ARM.exidx.text.SystemClock_Config) refers (Special) to _printf_f.o(.ARM.Collect$$_printf_percent$$00000003) for _printf_f
    main.o(.ARM.exidx.text.SystemClock_Config) refers (Special) to _printf_hex_int.o(.text) for _printf_longlong_hex
    main.o(.ARM.exidx.text.SystemClock_Config) refers (Special) to printf1.o(x$fpl$printf1) for _printf_fp_dec
    main.o(.ARM.exidx.text.SystemClock_Config) refers (Special) to _printf_str.o(.text) for _printf_str
    main.o(.ARM.exidx.text.SystemClock_Config) refers to main.o(.text.SystemClock_Config) for [Anonymous Symbol]
    main.o(.text.Error_Handler) refers (Special) to _printf_percent.o(.ARM.Collect$$_printf_percent$$00000000) for _printf_percent
    main.o(.text.Error_Handler) refers (Special) to _printf_pad.o(.text) for _printf_pre_padding
    main.o(.text.Error_Handler) refers (Special) to _printf_c.o(.ARM.Collect$$_printf_percent$$00000013) for _printf_c
    main.o(.text.Error_Handler) refers (Special) to _printf_s.o(.ARM.Collect$$_printf_percent$$00000014) for _printf_s
    main.o(.text.Error_Handler) refers (Special) to _printf_x.o(.ARM.Collect$$_printf_percent$$0000000C) for _printf_x
    main.o(.text.Error_Handler) refers (Special) to _printf_f.o(.ARM.Collect$$_printf_percent$$00000003) for _printf_f
    main.o(.text.Error_Handler) refers (Special) to _printf_hex_int.o(.text) for _printf_longlong_hex
    main.o(.text.Error_Handler) refers (Special) to printf1.o(x$fpl$printf1) for _printf_fp_dec
    main.o(.text.Error_Handler) refers (Special) to _printf_str.o(.text) for _printf_str
    main.o(.ARM.exidx.text.Error_Handler) refers (Special) to _printf_percent.o(.ARM.Collect$$_printf_percent$$00000000) for _printf_percent
    main.o(.ARM.exidx.text.Error_Handler) refers (Special) to _printf_pad.o(.text) for _printf_pre_padding
    main.o(.ARM.exidx.text.Error_Handler) refers (Special) to _printf_c.o(.ARM.Collect$$_printf_percent$$00000013) for _printf_c
    main.o(.ARM.exidx.text.Error_Handler) refers (Special) to _printf_s.o(.ARM.Collect$$_printf_percent$$00000014) for _printf_s
    main.o(.ARM.exidx.text.Error_Handler) refers (Special) to _printf_x.o(.ARM.Collect$$_printf_percent$$0000000C) for _printf_x
    main.o(.ARM.exidx.text.Error_Handler) refers (Special) to _printf_f.o(.ARM.Collect$$_printf_percent$$00000003) for _printf_f
    main.o(.ARM.exidx.text.Error_Handler) refers (Special) to _printf_hex_int.o(.text) for _printf_longlong_hex
    main.o(.ARM.exidx.text.Error_Handler) refers (Special) to printf1.o(x$fpl$printf1) for _printf_fp_dec
    main.o(.ARM.exidx.text.Error_Handler) refers (Special) to _printf_str.o(.text) for _printf_str
    main.o(.ARM.exidx.text.Error_Handler) refers to main.o(.text.Error_Handler) for [Anonymous Symbol]
    main.o(.rodata.str1.1) refers (Special) to _printf_percent.o(.ARM.Collect$$_printf_percent$$00000000) for _printf_percent
    main.o(.rodata.str1.1) refers (Special) to _printf_pad.o(.text) for _printf_pre_padding
    main.o(.rodata.str1.1) refers (Special) to _printf_c.o(.ARM.Collect$$_printf_percent$$00000013) for _printf_c
    main.o(.rodata.str1.1) refers (Special) to _printf_s.o(.ARM.Collect$$_printf_percent$$00000014) for _printf_s
    main.o(.rodata.str1.1) refers (Special) to _printf_x.o(.ARM.Collect$$_printf_percent$$0000000C) for _printf_x
    main.o(.rodata.str1.1) refers (Special) to _printf_f.o(.ARM.Collect$$_printf_percent$$00000003) for _printf_f
    main.o(.rodata.str1.1) refers (Special) to _printf_hex_int.o(.text) for _printf_longlong_hex
    main.o(.rodata.str1.1) refers (Special) to printf1.o(x$fpl$printf1) for _printf_fp_dec
    main.o(.rodata.str1.1) refers (Special) to _printf_str.o(.text) for _printf_str
    main.o(.bss.hi2c1) refers (Special) to _printf_percent.o(.ARM.Collect$$_printf_percent$$00000000) for _printf_percent
    main.o(.bss.hi2c1) refers (Special) to _printf_pad.o(.text) for _printf_pre_padding
    main.o(.bss.hi2c1) refers (Special) to _printf_c.o(.ARM.Collect$$_printf_percent$$00000013) for _printf_c
    main.o(.bss.hi2c1) refers (Special) to _printf_s.o(.ARM.Collect$$_printf_percent$$00000014) for _printf_s
    main.o(.bss.hi2c1) refers (Special) to _printf_x.o(.ARM.Collect$$_printf_percent$$0000000C) for _printf_x
    main.o(.bss.hi2c1) refers (Special) to _printf_f.o(.ARM.Collect$$_printf_percent$$00000003) for _printf_f
    main.o(.bss.hi2c1) refers (Special) to _printf_hex_int.o(.text) for _printf_longlong_hex
    main.o(.bss.hi2c1) refers (Special) to printf1.o(x$fpl$printf1) for _printf_fp_dec
    main.o(.bss.hi2c1) refers (Special) to _printf_str.o(.text) for _printf_str
    main.o(.ARM.use_no_argv) refers (Special) to _printf_percent.o(.ARM.Collect$$_printf_percent$$00000000) for _printf_percent
    main.o(.ARM.use_no_argv) refers (Special) to _printf_pad.o(.text) for _printf_pre_padding
    main.o(.ARM.use_no_argv) refers (Special) to _printf_c.o(.ARM.Collect$$_printf_percent$$00000013) for _printf_c
    main.o(.ARM.use_no_argv) refers (Special) to _printf_s.o(.ARM.Collect$$_printf_percent$$00000014) for _printf_s
    main.o(.ARM.use_no_argv) refers (Special) to _printf_x.o(.ARM.Collect$$_printf_percent$$0000000C) for _printf_x
    main.o(.ARM.use_no_argv) refers (Special) to _printf_f.o(.ARM.Collect$$_printf_percent$$00000003) for _printf_f
    main.o(.ARM.use_no_argv) refers (Special) to _printf_hex_int.o(.text) for _printf_longlong_hex
    main.o(.ARM.use_no_argv) refers (Special) to printf1.o(x$fpl$printf1) for _printf_fp_dec
    main.o(.ARM.use_no_argv) refers (Special) to _printf_str.o(.text) for _printf_str
    main.o(.data..L_MergedGlobals) refers (Special) to _printf_percent.o(.ARM.Collect$$_printf_percent$$00000000) for _printf_percent
    main.o(.data..L_MergedGlobals) refers (Special) to _printf_pad.o(.text) for _printf_pre_padding
    main.o(.data..L_MergedGlobals) refers (Special) to _printf_c.o(.ARM.Collect$$_printf_percent$$00000013) for _printf_c
    main.o(.data..L_MergedGlobals) refers (Special) to _printf_s.o(.ARM.Collect$$_printf_percent$$00000014) for _printf_s
    main.o(.data..L_MergedGlobals) refers (Special) to _printf_x.o(.ARM.Collect$$_printf_percent$$0000000C) for _printf_x
    main.o(.data..L_MergedGlobals) refers (Special) to _printf_f.o(.ARM.Collect$$_printf_percent$$00000003) for _printf_f
    main.o(.data..L_MergedGlobals) refers (Special) to _printf_hex_int.o(.text) for _printf_longlong_hex
    main.o(.data..L_MergedGlobals) refers (Special) to printf1.o(x$fpl$printf1) for _printf_fp_dec
    main.o(.data..L_MergedGlobals) refers (Special) to _printf_str.o(.text) for _printf_str
    main.o(.data..L_MergedGlobals) refers to main.o(.rodata.str1.1) for [Anonymous Symbol]
    main.o(.bss..L_MergedGlobals.16) refers (Special) to _printf_percent.o(.ARM.Collect$$_printf_percent$$00000000) for _printf_percent
    main.o(.bss..L_MergedGlobals.16) refers (Special) to _printf_pad.o(.text) for _printf_pre_padding
    main.o(.bss..L_MergedGlobals.16) refers (Special) to _printf_c.o(.ARM.Collect$$_printf_percent$$00000013) for _printf_c
    main.o(.bss..L_MergedGlobals.16) refers (Special) to _printf_s.o(.ARM.Collect$$_printf_percent$$00000014) for _printf_s
    main.o(.bss..L_MergedGlobals.16) refers (Special) to _printf_x.o(.ARM.Collect$$_printf_percent$$0000000C) for _printf_x
    main.o(.bss..L_MergedGlobals.16) refers (Special) to _printf_f.o(.ARM.Collect$$_printf_percent$$00000003) for _printf_f
    main.o(.bss..L_MergedGlobals.16) refers (Special) to _printf_hex_int.o(.text) for _printf_longlong_hex
    main.o(.bss..L_MergedGlobals.16) refers (Special) to printf1.o(x$fpl$printf1) for _printf_fp_dec
    main.o(.bss..L_MergedGlobals.16) refers (Special) to _printf_str.o(.text) for _printf_str
    stm32f0xx_it.o(.ARM.exidx.text.NMI_Handler) refers to stm32f0xx_it.o(.text.NMI_Handler) for [Anonymous Symbol]
    stm32f0xx_it.o(.ARM.exidx.text.HardFault_Handler) refers to stm32f0xx_it.o(.text.HardFault_Handler) for [Anonymous Symbol]
    stm32f0xx_it.o(.ARM.exidx.text.SVC_Handler) refers to stm32f0xx_it.o(.text.SVC_Handler) for [Anonymous Symbol]
    stm32f0xx_it.o(.ARM.exidx.text.PendSV_Handler) refers to stm32f0xx_it.o(.text.PendSV_Handler) for [Anonymous Symbol]
    stm32f0xx_it.o(.text.SysTick_Handler) refers to stm32f0xx_hal.o(.text.HAL_IncTick) for HAL_IncTick
    stm32f0xx_it.o(.ARM.exidx.text.SysTick_Handler) refers to stm32f0xx_it.o(.text.SysTick_Handler) for [Anonymous Symbol]
    stm32f0xx_hal_msp.o(.ARM.exidx.text.HAL_MspInit) refers to stm32f0xx_hal_msp.o(.text.HAL_MspInit) for [Anonymous Symbol]
    stm32f0xx_hal_msp.o(.text.HAL_I2C_MspInit) refers to stm32f0xx_hal_gpio.o(.text.HAL_GPIO_Init) for HAL_GPIO_Init
    stm32f0xx_hal_msp.o(.ARM.exidx.text.HAL_I2C_MspInit) refers to stm32f0xx_hal_msp.o(.text.HAL_I2C_MspInit) for [Anonymous Symbol]
    stm32f0xx_hal_msp.o(.text.HAL_I2C_MspDeInit) refers to stm32f0xx_hal_gpio.o(.text.HAL_GPIO_DeInit) for HAL_GPIO_DeInit
    stm32f0xx_hal_msp.o(.ARM.exidx.text.HAL_I2C_MspDeInit) refers to stm32f0xx_hal_msp.o(.text.HAL_I2C_MspDeInit) for [Anonymous Symbol]
    stm32f0xx_hal_msp.o(.ARM.exidx.text.HAL_RTC_MspInit) refers to stm32f0xx_hal_msp.o(.text.HAL_RTC_MspInit) for [Anonymous Symbol]
    stm32f0xx_hal_msp.o(.ARM.exidx.text.HAL_RTC_MspDeInit) refers to stm32f0xx_hal_msp.o(.text.HAL_RTC_MspDeInit) for [Anonymous Symbol]
    bmp280+aht20.o(.text.BMP280_init) refers to stm32f0xx_hal_i2c.o(.text.HAL_I2C_Mem_Read) for HAL_I2C_Mem_Read
    bmp280+aht20.o(.text.BMP280_init) refers to bmp280+aht20.o(.bss..L_MergedGlobals) for [Anonymous Symbol]
    bmp280+aht20.o(.text.BMP280_init) refers to main.o(.bss.hi2c1) for hi2c1
    bmp280+aht20.o(.ARM.exidx.text.BMP280_init) refers to bmp280+aht20.o(.text.BMP280_init) for [Anonymous Symbol]
    bmp280+aht20.o(.text.BMP280_get_calib_values) refers to stm32f0xx_hal_i2c.o(.text.HAL_I2C_Mem_Read) for HAL_I2C_Mem_Read
    bmp280+aht20.o(.text.BMP280_get_calib_values) refers to main.o(.bss.hi2c1) for hi2c1
    bmp280+aht20.o(.text.BMP280_get_calib_values) refers to bmp280+aht20.o(.bss..L_MergedGlobals) for [Anonymous Symbol]
    bmp280+aht20.o(.ARM.exidx.text.BMP280_get_calib_values) refers to bmp280+aht20.o(.text.BMP280_get_calib_values) for [Anonymous Symbol]
    bmp280+aht20.o(.text.BMP280_calc_values) refers to stm32f0xx_hal_i2c.o(.text.HAL_I2C_Mem_Read) for HAL_I2C_Mem_Read
    bmp280+aht20.o(.text.BMP280_calc_values) refers to dflti.o(.text) for __aeabi_i2d
    bmp280+aht20.o(.text.BMP280_calc_values) refers to dmul.o(.text) for __aeabi_dmul
    bmp280+aht20.o(.text.BMP280_calc_values) refers to daddsub.o(.text) for __aeabi_dadd
    bmp280+aht20.o(.text.BMP280_calc_values) refers to ddiv.o(.text) for __aeabi_ddiv
    bmp280+aht20.o(.text.BMP280_calc_values) refers to d2f.o(.text) for __aeabi_d2f
    bmp280+aht20.o(.text.BMP280_calc_values) refers to dfixi.o(.text) for __aeabi_d2iz
    bmp280+aht20.o(.text.BMP280_calc_values) refers to f2d.o(.text) for __aeabi_f2d
    bmp280+aht20.o(.text.BMP280_calc_values) refers to pow.o(i.pow) for pow
    bmp280+aht20.o(.text.BMP280_calc_values) refers to main.o(.bss.hi2c1) for hi2c1
    bmp280+aht20.o(.text.BMP280_calc_values) refers to bmp280+aht20.o(.bss..L_MergedGlobals) for [Anonymous Symbol]
    bmp280+aht20.o(.ARM.exidx.text.BMP280_calc_values) refers to bmp280+aht20.o(.text.BMP280_calc_values) for [Anonymous Symbol]
    bmp280+aht20.o(.text.AHT20_init) refers to stm32f0xx_hal_i2c.o(.text.HAL_I2C_Master_Transmit) for HAL_I2C_Master_Transmit
    bmp280+aht20.o(.text.AHT20_init) refers to main.o(.bss.hi2c1) for hi2c1
    bmp280+aht20.o(.ARM.exidx.text.AHT20_init) refers to bmp280+aht20.o(.text.AHT20_init) for [Anonymous Symbol]
    bmp280+aht20.o(.text.AHT20_Read) refers to stm32f0xx_hal_i2c.o(.text.HAL_I2C_Master_Transmit) for HAL_I2C_Master_Transmit
    bmp280+aht20.o(.text.AHT20_Read) refers to stm32f0xx_hal.o(.text.HAL_Delay) for HAL_Delay
    bmp280+aht20.o(.text.AHT20_Read) refers to stm32f0xx_hal_i2c.o(.text.HAL_I2C_Master_Receive) for HAL_I2C_Master_Receive
    bmp280+aht20.o(.text.AHT20_Read) refers to fflti.o(.text) for __aeabi_ui2f
    bmp280+aht20.o(.text.AHT20_Read) refers to fmul.o(x$fpl$fmul) for __aeabi_fmul
    bmp280+aht20.o(.text.AHT20_Read) refers to faddsub.o(x$fpl$fadd) for __aeabi_fadd
    bmp280+aht20.o(.text.AHT20_Read) refers to main.o(.bss.hi2c1) for hi2c1
    bmp280+aht20.o(.text.AHT20_Read) refers to bmp280+aht20.o(.bss..L_MergedGlobals) for [Anonymous Symbol]
    bmp280+aht20.o(.ARM.exidx.text.AHT20_Read) refers to bmp280+aht20.o(.text.AHT20_Read) for [Anonymous Symbol]
    ssd1306.o(.text.init_OLED) refers to stm32f0xx_hal_i2c.o(.text.HAL_I2C_Master_Transmit) for HAL_I2C_Master_Transmit
    ssd1306.o(.text.init_OLED) refers to ssd1306.o(.bss.data_stream) for data_stream
    ssd1306.o(.text.init_OLED) refers to ssd1306.o(.data.OLED_init) for OLED_init
    ssd1306.o(.text.init_OLED) refers to main.o(.bss.hi2c1) for hi2c1
    ssd1306.o(.ARM.exidx.text.init_OLED) refers to ssd1306.o(.text.init_OLED) for [Anonymous Symbol]
    ssd1306.o(.text.sendcommand) refers to stm32f0xx_hal_i2c.o(.text.HAL_I2C_Master_Transmit) for HAL_I2C_Master_Transmit
    ssd1306.o(.text.sendcommand) refers to ssd1306.o(.bss.data_stream) for data_stream
    ssd1306.o(.text.sendcommand) refers to main.o(.bss.hi2c1) for hi2c1
    ssd1306.o(.ARM.exidx.text.sendcommand) refers to ssd1306.o(.text.sendcommand) for [Anonymous Symbol]
    ssd1306.o(.text.SendChar) refers to stm32f0xx_hal_i2c.o(.text.HAL_I2C_Master_Transmit) for HAL_I2C_Master_Transmit
    ssd1306.o(.text.SendChar) refers to ssd1306.o(.bss.data_stream) for data_stream
    ssd1306.o(.text.SendChar) refers to main.o(.bss.hi2c1) for hi2c1
    ssd1306.o(.ARM.exidx.text.SendChar) refers to ssd1306.o(.text.SendChar) for [Anonymous Symbol]
    ssd1306.o(.text.displayOn) refers to stm32f0xx_hal_i2c.o(.text.HAL_I2C_Master_Transmit) for HAL_I2C_Master_Transmit
    ssd1306.o(.text.displayOn) refers to ssd1306.o(.bss.data_stream) for data_stream
    ssd1306.o(.text.displayOn) refers to main.o(.bss.hi2c1) for hi2c1
    ssd1306.o(.ARM.exidx.text.displayOn) refers to ssd1306.o(.text.displayOn) for [Anonymous Symbol]
    ssd1306.o(.text.displayOff) refers to stm32f0xx_hal_i2c.o(.text.HAL_I2C_Master_Transmit) for HAL_I2C_Master_Transmit
    ssd1306.o(.text.displayOff) refers to ssd1306.o(.bss.data_stream) for data_stream
    ssd1306.o(.text.displayOff) refers to main.o(.bss.hi2c1) for hi2c1
    ssd1306.o(.ARM.exidx.text.displayOff) refers to ssd1306.o(.text.displayOff) for [Anonymous Symbol]
    ssd1306.o(.text.setXY) refers to stm32f0xx_hal_i2c.o(.text.HAL_I2C_Master_Transmit) for HAL_I2C_Master_Transmit
    ssd1306.o(.text.setXY) refers to ssd1306.o(.bss.data_stream) for data_stream
    ssd1306.o(.text.setXY) refers to main.o(.bss.hi2c1) for hi2c1
    ssd1306.o(.ARM.exidx.text.setXY) refers to ssd1306.o(.text.setXY) for [Anonymous Symbol]
    ssd1306.o(.text.clear_display) refers to stm32f0xx_hal_i2c.o(.text.HAL_I2C_Master_Transmit) for HAL_I2C_Master_Transmit
    ssd1306.o(.text.clear_display) refers to ssd1306.o(.bss.data_stream) for data_stream
    ssd1306.o(.text.clear_display) refers to main.o(.bss.hi2c1) for hi2c1
    ssd1306.o(.ARM.exidx.text.clear_display) refers to ssd1306.o(.text.clear_display) for [Anonymous Symbol]
    ssd1306.o(.text.OLCD_write_string) refers to stm32f0xx_hal_i2c.o(.text.HAL_I2C_Master_Transmit) for HAL_I2C_Master_Transmit
    ssd1306.o(.text.OLCD_write_string) refers to ssd1306.o(.bss.data_stream) for data_stream
    ssd1306.o(.text.OLCD_write_string) refers to main.o(.bss.hi2c1) for hi2c1
    ssd1306.o(.text.OLCD_write_string) refers to ssd1306.o(.data.myFont) for myFont
    ssd1306.o(.ARM.exidx.text.OLCD_write_string) refers to ssd1306.o(.text.OLCD_write_string) for [Anonymous Symbol]
    stm32f0xx_hal_i2c.o(.text.HAL_I2C_Init) refers to stm32f0xx_hal_msp.o(.text.HAL_I2C_MspInit) for HAL_I2C_MspInit
    stm32f0xx_hal_i2c.o(.ARM.exidx.text.HAL_I2C_Init) refers to stm32f0xx_hal_i2c.o(.text.HAL_I2C_Init) for [Anonymous Symbol]
    stm32f0xx_hal_i2c.o(.ARM.exidx.text.HAL_I2C_MspInit) refers to stm32f0xx_hal_i2c.o(.text.HAL_I2C_MspInit) for [Anonymous Symbol]
    stm32f0xx_hal_i2c.o(.text.HAL_I2C_DeInit) refers to stm32f0xx_hal_msp.o(.text.HAL_I2C_MspDeInit) for HAL_I2C_MspDeInit
    stm32f0xx_hal_i2c.o(.ARM.exidx.text.HAL_I2C_DeInit) refers to stm32f0xx_hal_i2c.o(.text.HAL_I2C_DeInit) for [Anonymous Symbol]
    stm32f0xx_hal_i2c.o(.ARM.exidx.text.HAL_I2C_MspDeInit) refers to stm32f0xx_hal_i2c.o(.text.HAL_I2C_MspDeInit) for [Anonymous Symbol]
    stm32f0xx_hal_i2c.o(.text.HAL_I2C_Master_Transmit) refers to stm32f0xx_hal.o(.text.HAL_GetTick) for HAL_GetTick
    stm32f0xx_hal_i2c.o(.text.HAL_I2C_Master_Transmit) refers to stm32f0xx_hal_i2c.o(.text.I2C_IsErrorOccurred) for I2C_IsErrorOccurred
    stm32f0xx_hal_i2c.o(.text.HAL_I2C_Master_Transmit) refers to stm32f0xx_hal_i2c.o(.text.I2C_WaitOnTXISFlagUntilTimeout) for I2C_WaitOnTXISFlagUntilTimeout
    stm32f0xx_hal_i2c.o(.text.HAL_I2C_Master_Transmit) refers to stm32f0xx_hal_i2c.o(.text.I2C_WaitOnFlagUntilTimeout) for I2C_WaitOnFlagUntilTimeout
    stm32f0xx_hal_i2c.o(.text.HAL_I2C_Master_Transmit) refers to stm32f0xx_hal_i2c.o(.text.I2C_WaitOnSTOPFlagUntilTimeout) for I2C_WaitOnSTOPFlagUntilTimeout
    stm32f0xx_hal_i2c.o(.ARM.exidx.text.HAL_I2C_Master_Transmit) refers to stm32f0xx_hal_i2c.o(.text.HAL_I2C_Master_Transmit) for [Anonymous Symbol]
    stm32f0xx_hal_i2c.o(.text.I2C_WaitOnFlagUntilTimeout) refers to stm32f0xx_hal_i2c.o(.text.I2C_IsErrorOccurred) for I2C_IsErrorOccurred
    stm32f0xx_hal_i2c.o(.text.I2C_WaitOnFlagUntilTimeout) refers to stm32f0xx_hal.o(.text.HAL_GetTick) for HAL_GetTick
    stm32f0xx_hal_i2c.o(.ARM.exidx.text.I2C_WaitOnFlagUntilTimeout) refers to stm32f0xx_hal_i2c.o(.text.I2C_WaitOnFlagUntilTimeout) for [Anonymous Symbol]
    stm32f0xx_hal_i2c.o(.text.I2C_WaitOnTXISFlagUntilTimeout) refers to stm32f0xx_hal_i2c.o(.text.I2C_IsErrorOccurred) for I2C_IsErrorOccurred
    stm32f0xx_hal_i2c.o(.text.I2C_WaitOnTXISFlagUntilTimeout) refers to stm32f0xx_hal.o(.text.HAL_GetTick) for HAL_GetTick
    stm32f0xx_hal_i2c.o(.ARM.exidx.text.I2C_WaitOnTXISFlagUntilTimeout) refers to stm32f0xx_hal_i2c.o(.text.I2C_WaitOnTXISFlagUntilTimeout) for [Anonymous Symbol]
    stm32f0xx_hal_i2c.o(.text.I2C_WaitOnSTOPFlagUntilTimeout) refers to stm32f0xx_hal_i2c.o(.text.I2C_IsErrorOccurred) for I2C_IsErrorOccurred
    stm32f0xx_hal_i2c.o(.text.I2C_WaitOnSTOPFlagUntilTimeout) refers to stm32f0xx_hal.o(.text.HAL_GetTick) for HAL_GetTick
    stm32f0xx_hal_i2c.o(.ARM.exidx.text.I2C_WaitOnSTOPFlagUntilTimeout) refers to stm32f0xx_hal_i2c.o(.text.I2C_WaitOnSTOPFlagUntilTimeout) for [Anonymous Symbol]
    stm32f0xx_hal_i2c.o(.text.HAL_I2C_Master_Receive) refers to stm32f0xx_hal.o(.text.HAL_GetTick) for HAL_GetTick
    stm32f0xx_hal_i2c.o(.text.HAL_I2C_Master_Receive) refers to stm32f0xx_hal_i2c.o(.text.I2C_IsErrorOccurred) for I2C_IsErrorOccurred
    stm32f0xx_hal_i2c.o(.text.HAL_I2C_Master_Receive) refers to stm32f0xx_hal_i2c.o(.text.I2C_WaitOnRXNEFlagUntilTimeout) for I2C_WaitOnRXNEFlagUntilTimeout
    stm32f0xx_hal_i2c.o(.text.HAL_I2C_Master_Receive) refers to stm32f0xx_hal_i2c.o(.text.I2C_WaitOnFlagUntilTimeout) for I2C_WaitOnFlagUntilTimeout
    stm32f0xx_hal_i2c.o(.text.HAL_I2C_Master_Receive) refers to stm32f0xx_hal_i2c.o(.text.I2C_WaitOnSTOPFlagUntilTimeout) for I2C_WaitOnSTOPFlagUntilTimeout
    stm32f0xx_hal_i2c.o(.ARM.exidx.text.HAL_I2C_Master_Receive) refers to stm32f0xx_hal_i2c.o(.text.HAL_I2C_Master_Receive) for [Anonymous Symbol]
    stm32f0xx_hal_i2c.o(.text.I2C_WaitOnRXNEFlagUntilTimeout) refers to stm32f0xx_hal_i2c.o(.text.I2C_IsErrorOccurred) for I2C_IsErrorOccurred
    stm32f0xx_hal_i2c.o(.text.I2C_WaitOnRXNEFlagUntilTimeout) refers to stm32f0xx_hal.o(.text.HAL_GetTick) for HAL_GetTick
    stm32f0xx_hal_i2c.o(.ARM.exidx.text.I2C_WaitOnRXNEFlagUntilTimeout) refers to stm32f0xx_hal_i2c.o(.text.I2C_WaitOnRXNEFlagUntilTimeout) for [Anonymous Symbol]
    stm32f0xx_hal_i2c.o(.text.HAL_I2C_Slave_Transmit) refers to stm32f0xx_hal.o(.text.HAL_GetTick) for HAL_GetTick
    stm32f0xx_hal_i2c.o(.text.HAL_I2C_Slave_Transmit) refers to stm32f0xx_hal_i2c.o(.text.I2C_WaitOnFlagUntilTimeout) for I2C_WaitOnFlagUntilTimeout
    stm32f0xx_hal_i2c.o(.text.HAL_I2C_Slave_Transmit) refers to stm32f0xx_hal_i2c.o(.text.I2C_WaitOnTXISFlagUntilTimeout) for I2C_WaitOnTXISFlagUntilTimeout
    stm32f0xx_hal_i2c.o(.text.HAL_I2C_Slave_Transmit) refers to stm32f0xx_hal_i2c.o(.text.I2C_WaitOnSTOPFlagUntilTimeout) for I2C_WaitOnSTOPFlagUntilTimeout
    stm32f0xx_hal_i2c.o(.ARM.exidx.text.HAL_I2C_Slave_Transmit) refers to stm32f0xx_hal_i2c.o(.text.HAL_I2C_Slave_Transmit) for [Anonymous Symbol]
    stm32f0xx_hal_i2c.o(.text.HAL_I2C_Slave_Receive) refers to stm32f0xx_hal.o(.text.HAL_GetTick) for HAL_GetTick
    stm32f0xx_hal_i2c.o(.text.HAL_I2C_Slave_Receive) refers to stm32f0xx_hal_i2c.o(.text.I2C_WaitOnFlagUntilTimeout) for I2C_WaitOnFlagUntilTimeout
    stm32f0xx_hal_i2c.o(.text.HAL_I2C_Slave_Receive) refers to stm32f0xx_hal_i2c.o(.text.I2C_WaitOnRXNEFlagUntilTimeout) for I2C_WaitOnRXNEFlagUntilTimeout
    stm32f0xx_hal_i2c.o(.text.HAL_I2C_Slave_Receive) refers to stm32f0xx_hal_i2c.o(.text.I2C_WaitOnSTOPFlagUntilTimeout) for I2C_WaitOnSTOPFlagUntilTimeout
    stm32f0xx_hal_i2c.o(.ARM.exidx.text.HAL_I2C_Slave_Receive) refers to stm32f0xx_hal_i2c.o(.text.HAL_I2C_Slave_Receive) for [Anonymous Symbol]
    stm32f0xx_hal_i2c.o(.text.HAL_I2C_Master_Transmit_IT) refers to stm32f0xx_hal_i2c.o(.text.I2C_Master_ISR_IT) for I2C_Master_ISR_IT
    stm32f0xx_hal_i2c.o(.ARM.exidx.text.HAL_I2C_Master_Transmit_IT) refers to stm32f0xx_hal_i2c.o(.text.HAL_I2C_Master_Transmit_IT) for [Anonymous Symbol]
    stm32f0xx_hal_i2c.o(.text.I2C_Master_ISR_IT) refers to stm32f0xx_hal_i2c.o(.text.I2C_ITMasterCplt) for I2C_ITMasterCplt
    stm32f0xx_hal_i2c.o(.text.I2C_Master_ISR_IT) refers to stm32f0xx_hal_i2c.o(.text.I2C_ITMasterSeqCplt) for I2C_ITMasterSeqCplt
    stm32f0xx_hal_i2c.o(.text.I2C_Master_ISR_IT) refers to stm32f0xx_hal_i2c.o(.text.I2C_ITError) for I2C_ITError
    stm32f0xx_hal_i2c.o(.ARM.exidx.text.I2C_Master_ISR_IT) refers to stm32f0xx_hal_i2c.o(.text.I2C_Master_ISR_IT) for [Anonymous Symbol]
    stm32f0xx_hal_i2c.o(.text.HAL_I2C_Master_Receive_IT) refers to stm32f0xx_hal_i2c.o(.text.I2C_Master_ISR_IT) for I2C_Master_ISR_IT
    stm32f0xx_hal_i2c.o(.ARM.exidx.text.HAL_I2C_Master_Receive_IT) refers to stm32f0xx_hal_i2c.o(.text.HAL_I2C_Master_Receive_IT) for [Anonymous Symbol]
    stm32f0xx_hal_i2c.o(.text.HAL_I2C_Slave_Transmit_IT) refers to stm32f0xx_hal_i2c.o(.text.I2C_Slave_ISR_IT) for I2C_Slave_ISR_IT
    stm32f0xx_hal_i2c.o(.ARM.exidx.text.HAL_I2C_Slave_Transmit_IT) refers to stm32f0xx_hal_i2c.o(.text.HAL_I2C_Slave_Transmit_IT) for [Anonymous Symbol]
    stm32f0xx_hal_i2c.o(.text.I2C_Slave_ISR_IT) refers to stm32f0xx_hal_i2c.o(.text.I2C_ITSlaveCplt) for I2C_ITSlaveCplt
    stm32f0xx_hal_i2c.o(.text.I2C_Slave_ISR_IT) refers to stm32f0xx_hal_i2c.o(.text.I2C_ITError) for I2C_ITError
    stm32f0xx_hal_i2c.o(.text.I2C_Slave_ISR_IT) refers to stm32f0xx_hal_i2c.o(.text.HAL_I2C_ListenCpltCallback) for HAL_I2C_ListenCpltCallback
    stm32f0xx_hal_i2c.o(.text.I2C_Slave_ISR_IT) refers to stm32f0xx_hal_i2c.o(.text.I2C_ITAddrCplt) for I2C_ITAddrCplt
    stm32f0xx_hal_i2c.o(.text.I2C_Slave_ISR_IT) refers to stm32f0xx_hal_i2c.o(.text.HAL_I2C_SlaveRxCpltCallback) for HAL_I2C_SlaveRxCpltCallback
    stm32f0xx_hal_i2c.o(.text.I2C_Slave_ISR_IT) refers to stm32f0xx_hal_i2c.o(.text.HAL_I2C_SlaveTxCpltCallback) for HAL_I2C_SlaveTxCpltCallback
    stm32f0xx_hal_i2c.o(.text.I2C_Slave_ISR_IT) refers to stm32f0xx_hal_i2c.o(.text.I2C_ITSlaveSeqCplt) for I2C_ITSlaveSeqCplt
    stm32f0xx_hal_i2c.o(.ARM.exidx.text.I2C_Slave_ISR_IT) refers to stm32f0xx_hal_i2c.o(.text.I2C_Slave_ISR_IT) for [Anonymous Symbol]
    stm32f0xx_hal_i2c.o(.text.HAL_I2C_Slave_Receive_IT) refers to stm32f0xx_hal_i2c.o(.text.I2C_Slave_ISR_IT) for I2C_Slave_ISR_IT
    stm32f0xx_hal_i2c.o(.ARM.exidx.text.HAL_I2C_Slave_Receive_IT) refers to stm32f0xx_hal_i2c.o(.text.HAL_I2C_Slave_Receive_IT) for [Anonymous Symbol]
    stm32f0xx_hal_i2c.o(.text.HAL_I2C_Master_Transmit_DMA) refers to stm32f0xx_hal_dma.o(.text.HAL_DMA_Start_IT) for HAL_DMA_Start_IT
    stm32f0xx_hal_i2c.o(.text.HAL_I2C_Master_Transmit_DMA) refers to stm32f0xx_hal_i2c.o(.text.I2C_Master_ISR_DMA) for I2C_Master_ISR_DMA
    stm32f0xx_hal_i2c.o(.text.HAL_I2C_Master_Transmit_DMA) refers to stm32f0xx_hal_i2c.o(.text.I2C_DMAError) for I2C_DMAError
    stm32f0xx_hal_i2c.o(.text.HAL_I2C_Master_Transmit_DMA) refers to stm32f0xx_hal_i2c.o(.text.I2C_DMAMasterTransmitCplt) for I2C_DMAMasterTransmitCplt
    stm32f0xx_hal_i2c.o(.text.HAL_I2C_Master_Transmit_DMA) refers to stm32f0xx_hal_i2c.o(.text.I2C_Master_ISR_IT) for I2C_Master_ISR_IT
    stm32f0xx_hal_i2c.o(.ARM.exidx.text.HAL_I2C_Master_Transmit_DMA) refers to stm32f0xx_hal_i2c.o(.text.HAL_I2C_Master_Transmit_DMA) for [Anonymous Symbol]
    stm32f0xx_hal_i2c.o(.text.I2C_Master_ISR_DMA) refers to stm32f0xx_hal_i2c.o(.text.I2C_ITMasterCplt) for I2C_ITMasterCplt
    stm32f0xx_hal_i2c.o(.text.I2C_Master_ISR_DMA) refers to stm32f0xx_hal_i2c.o(.text.I2C_ITError) for I2C_ITError
    stm32f0xx_hal_i2c.o(.text.I2C_Master_ISR_DMA) refers to stm32f0xx_hal_i2c.o(.text.HAL_I2C_MasterRxCpltCallback) for HAL_I2C_MasterRxCpltCallback
    stm32f0xx_hal_i2c.o(.text.I2C_Master_ISR_DMA) refers to stm32f0xx_hal_i2c.o(.text.I2C_ITMasterSeqCplt) for I2C_ITMasterSeqCplt
    stm32f0xx_hal_i2c.o(.text.I2C_Master_ISR_DMA) refers to stm32f0xx_hal_i2c.o(.text.HAL_I2C_MasterTxCpltCallback) for HAL_I2C_MasterTxCpltCallback
    stm32f0xx_hal_i2c.o(.text.I2C_Master_ISR_DMA) refers to stm32f0xx_hal_i2c.o(.text.I2C_Slave_ISR_DMA) for I2C_Slave_ISR_DMA
    stm32f0xx_hal_i2c.o(.text.I2C_Master_ISR_DMA) refers to stm32f0xx_hal_i2c.o(.text.I2C_Mem_ISR_DMA) for I2C_Mem_ISR_DMA
    stm32f0xx_hal_i2c.o(.ARM.exidx.text.I2C_Master_ISR_DMA) refers to stm32f0xx_hal_i2c.o(.text.I2C_Master_ISR_DMA) for [Anonymous Symbol]
    stm32f0xx_hal_i2c.o(.text.I2C_DMAMasterTransmitCplt) refers to stm32f0xx_hal_dma.o(.text.HAL_DMA_Start_IT) for HAL_DMA_Start_IT
    stm32f0xx_hal_i2c.o(.text.I2C_DMAMasterTransmitCplt) refers to stm32f0xx_hal_i2c.o(.text.I2C_ITError) for I2C_ITError
    stm32f0xx_hal_i2c.o(.text.I2C_DMAMasterTransmitCplt) refers to stm32f0xx_hal_i2c.o(.text.I2C_Slave_ISR_DMA) for I2C_Slave_ISR_DMA
    stm32f0xx_hal_i2c.o(.text.I2C_DMAMasterTransmitCplt) refers to stm32f0xx_hal_i2c.o(.text.I2C_Master_ISR_DMA) for I2C_Master_ISR_DMA
    stm32f0xx_hal_i2c.o(.text.I2C_DMAMasterTransmitCplt) refers to stm32f0xx_hal_i2c.o(.text.I2C_Mem_ISR_DMA) for I2C_Mem_ISR_DMA
    stm32f0xx_hal_i2c.o(.ARM.exidx.text.I2C_DMAMasterTransmitCplt) refers to stm32f0xx_hal_i2c.o(.text.I2C_DMAMasterTransmitCplt) for [Anonymous Symbol]
    stm32f0xx_hal_i2c.o(.text.I2C_DMAError) refers to stm32f0xx_hal_i2c.o(.text.I2C_ITError) for I2C_ITError
    stm32f0xx_hal_i2c.o(.ARM.exidx.text.I2C_DMAError) refers to stm32f0xx_hal_i2c.o(.text.I2C_DMAError) for [Anonymous Symbol]
    stm32f0xx_hal_i2c.o(.text.HAL_I2C_Master_Receive_DMA) refers to stm32f0xx_hal_dma.o(.text.HAL_DMA_Start_IT) for HAL_DMA_Start_IT
    stm32f0xx_hal_i2c.o(.text.HAL_I2C_Master_Receive_DMA) refers to stm32f0xx_hal_i2c.o(.text.I2C_Master_ISR_DMA) for I2C_Master_ISR_DMA
    stm32f0xx_hal_i2c.o(.text.HAL_I2C_Master_Receive_DMA) refers to stm32f0xx_hal_i2c.o(.text.I2C_Master_ISR_IT) for I2C_Master_ISR_IT
    stm32f0xx_hal_i2c.o(.text.HAL_I2C_Master_Receive_DMA) refers to stm32f0xx_hal_i2c.o(.text.I2C_DMAError) for I2C_DMAError
    stm32f0xx_hal_i2c.o(.text.HAL_I2C_Master_Receive_DMA) refers to stm32f0xx_hal_i2c.o(.text.I2C_DMAMasterReceiveCplt) for I2C_DMAMasterReceiveCplt
    stm32f0xx_hal_i2c.o(.ARM.exidx.text.HAL_I2C_Master_Receive_DMA) refers to stm32f0xx_hal_i2c.o(.text.HAL_I2C_Master_Receive_DMA) for [Anonymous Symbol]
    stm32f0xx_hal_i2c.o(.text.I2C_DMAMasterReceiveCplt) refers to stm32f0xx_hal_dma.o(.text.HAL_DMA_Start_IT) for HAL_DMA_Start_IT
    stm32f0xx_hal_i2c.o(.text.I2C_DMAMasterReceiveCplt) refers to stm32f0xx_hal_i2c.o(.text.I2C_ITError) for I2C_ITError
    stm32f0xx_hal_i2c.o(.text.I2C_DMAMasterReceiveCplt) refers to stm32f0xx_hal_i2c.o(.text.I2C_Slave_ISR_DMA) for I2C_Slave_ISR_DMA
    stm32f0xx_hal_i2c.o(.text.I2C_DMAMasterReceiveCplt) refers to stm32f0xx_hal_i2c.o(.text.I2C_Master_ISR_DMA) for I2C_Master_ISR_DMA
    stm32f0xx_hal_i2c.o(.text.I2C_DMAMasterReceiveCplt) refers to stm32f0xx_hal_i2c.o(.text.I2C_Mem_ISR_DMA) for I2C_Mem_ISR_DMA
    stm32f0xx_hal_i2c.o(.ARM.exidx.text.I2C_DMAMasterReceiveCplt) refers to stm32f0xx_hal_i2c.o(.text.I2C_DMAMasterReceiveCplt) for [Anonymous Symbol]
    stm32f0xx_hal_i2c.o(.text.HAL_I2C_Slave_Transmit_DMA) refers to stm32f0xx_hal_dma.o(.text.HAL_DMA_Start_IT) for HAL_DMA_Start_IT
    stm32f0xx_hal_i2c.o(.text.HAL_I2C_Slave_Transmit_DMA) refers to stm32f0xx_hal_i2c.o(.text.I2C_Slave_ISR_DMA) for I2C_Slave_ISR_DMA
    stm32f0xx_hal_i2c.o(.text.HAL_I2C_Slave_Transmit_DMA) refers to stm32f0xx_hal_i2c.o(.text.I2C_DMAError) for I2C_DMAError
    stm32f0xx_hal_i2c.o(.text.HAL_I2C_Slave_Transmit_DMA) refers to stm32f0xx_hal_i2c.o(.text.I2C_DMASlaveTransmitCplt) for I2C_DMASlaveTransmitCplt
    stm32f0xx_hal_i2c.o(.ARM.exidx.text.HAL_I2C_Slave_Transmit_DMA) refers to stm32f0xx_hal_i2c.o(.text.HAL_I2C_Slave_Transmit_DMA) for [Anonymous Symbol]
    stm32f0xx_hal_i2c.o(.text.I2C_Slave_ISR_DMA) refers to stm32f0xx_hal_i2c.o(.text.I2C_ITAddrCplt) for I2C_ITAddrCplt
    stm32f0xx_hal_i2c.o(.text.I2C_Slave_ISR_DMA) refers to stm32f0xx_hal_i2c.o(.text.I2C_ITSlaveCplt) for I2C_ITSlaveCplt
    stm32f0xx_hal_i2c.o(.text.I2C_Slave_ISR_DMA) refers to stm32f0xx_hal_i2c.o(.text.I2C_ITError) for I2C_ITError
    stm32f0xx_hal_i2c.o(.text.I2C_Slave_ISR_DMA) refers to stm32f0xx_hal_i2c.o(.text.I2C_ITListenCplt) for I2C_ITListenCplt
    stm32f0xx_hal_i2c.o(.text.I2C_Slave_ISR_DMA) refers to stm32f0xx_hal_i2c.o(.text.I2C_ITSlaveSeqCplt) for I2C_ITSlaveSeqCplt
    stm32f0xx_hal_i2c.o(.ARM.exidx.text.I2C_Slave_ISR_DMA) refers to stm32f0xx_hal_i2c.o(.text.I2C_Slave_ISR_DMA) for [Anonymous Symbol]
    stm32f0xx_hal_i2c.o(.text.I2C_DMASlaveTransmitCplt) refers to stm32f0xx_hal_i2c.o(.text.HAL_I2C_SlaveRxCpltCallback) for HAL_I2C_SlaveRxCpltCallback
    stm32f0xx_hal_i2c.o(.text.I2C_DMASlaveTransmitCplt) refers to stm32f0xx_hal_i2c.o(.text.HAL_I2C_SlaveTxCpltCallback) for HAL_I2C_SlaveTxCpltCallback
    stm32f0xx_hal_i2c.o(.ARM.exidx.text.I2C_DMASlaveTransmitCplt) refers to stm32f0xx_hal_i2c.o(.text.I2C_DMASlaveTransmitCplt) for [Anonymous Symbol]
    stm32f0xx_hal_i2c.o(.text.HAL_I2C_Slave_Receive_DMA) refers to stm32f0xx_hal_dma.o(.text.HAL_DMA_Start_IT) for HAL_DMA_Start_IT
    stm32f0xx_hal_i2c.o(.text.HAL_I2C_Slave_Receive_DMA) refers to stm32f0xx_hal_i2c.o(.text.I2C_Slave_ISR_DMA) for I2C_Slave_ISR_DMA
    stm32f0xx_hal_i2c.o(.text.HAL_I2C_Slave_Receive_DMA) refers to stm32f0xx_hal_i2c.o(.text.I2C_DMAError) for I2C_DMAError
    stm32f0xx_hal_i2c.o(.text.HAL_I2C_Slave_Receive_DMA) refers to stm32f0xx_hal_i2c.o(.text.I2C_DMASlaveReceiveCplt) for I2C_DMASlaveReceiveCplt
    stm32f0xx_hal_i2c.o(.ARM.exidx.text.HAL_I2C_Slave_Receive_DMA) refers to stm32f0xx_hal_i2c.o(.text.HAL_I2C_Slave_Receive_DMA) for [Anonymous Symbol]
    stm32f0xx_hal_i2c.o(.text.I2C_DMASlaveReceiveCplt) refers to stm32f0xx_hal_i2c.o(.text.HAL_I2C_SlaveRxCpltCallback) for HAL_I2C_SlaveRxCpltCallback
    stm32f0xx_hal_i2c.o(.text.I2C_DMASlaveReceiveCplt) refers to stm32f0xx_hal_i2c.o(.text.HAL_I2C_SlaveTxCpltCallback) for HAL_I2C_SlaveTxCpltCallback
    stm32f0xx_hal_i2c.o(.ARM.exidx.text.I2C_DMASlaveReceiveCplt) refers to stm32f0xx_hal_i2c.o(.text.I2C_DMASlaveReceiveCplt) for [Anonymous Symbol]
    stm32f0xx_hal_i2c.o(.text.HAL_I2C_Mem_Write) refers to stm32f0xx_hal.o(.text.HAL_GetTick) for HAL_GetTick
    stm32f0xx_hal_i2c.o(.text.HAL_I2C_Mem_Write) refers to stm32f0xx_hal_i2c.o(.text.I2C_WaitOnTXISFlagUntilTimeout) for I2C_WaitOnTXISFlagUntilTimeout
    stm32f0xx_hal_i2c.o(.text.HAL_I2C_Mem_Write) refers to stm32f0xx_hal_i2c.o(.text.I2C_WaitOnFlagUntilTimeout) for I2C_WaitOnFlagUntilTimeout
    stm32f0xx_hal_i2c.o(.text.HAL_I2C_Mem_Write) refers to stm32f0xx_hal_i2c.o(.text.I2C_IsErrorOccurred) for I2C_IsErrorOccurred
    stm32f0xx_hal_i2c.o(.text.HAL_I2C_Mem_Write) refers to stm32f0xx_hal_i2c.o(.text.I2C_WaitOnSTOPFlagUntilTimeout) for I2C_WaitOnSTOPFlagUntilTimeout
    stm32f0xx_hal_i2c.o(.ARM.exidx.text.HAL_I2C_Mem_Write) refers to stm32f0xx_hal_i2c.o(.text.HAL_I2C_Mem_Write) for [Anonymous Symbol]
    stm32f0xx_hal_i2c.o(.text.HAL_I2C_Mem_Read) refers to stm32f0xx_hal.o(.text.HAL_GetTick) for HAL_GetTick
    stm32f0xx_hal_i2c.o(.text.HAL_I2C_Mem_Read) refers to stm32f0xx_hal_i2c.o(.text.I2C_WaitOnTXISFlagUntilTimeout) for I2C_WaitOnTXISFlagUntilTimeout
    stm32f0xx_hal_i2c.o(.text.HAL_I2C_Mem_Read) refers to stm32f0xx_hal_i2c.o(.text.I2C_WaitOnFlagUntilTimeout) for I2C_WaitOnFlagUntilTimeout
    stm32f0xx_hal_i2c.o(.text.HAL_I2C_Mem_Read) refers to stm32f0xx_hal_i2c.o(.text.I2C_IsErrorOccurred) for I2C_IsErrorOccurred
    stm32f0xx_hal_i2c.o(.text.HAL_I2C_Mem_Read) refers to stm32f0xx_hal_i2c.o(.text.I2C_WaitOnSTOPFlagUntilTimeout) for I2C_WaitOnSTOPFlagUntilTimeout
    stm32f0xx_hal_i2c.o(.ARM.exidx.text.HAL_I2C_Mem_Read) refers to stm32f0xx_hal_i2c.o(.text.HAL_I2C_Mem_Read) for [Anonymous Symbol]
    stm32f0xx_hal_i2c.o(.text.HAL_I2C_Mem_Write_IT) refers to stm32f0xx_hal_i2c.o(.text.I2C_Mem_ISR_IT) for I2C_Mem_ISR_IT
    stm32f0xx_hal_i2c.o(.ARM.exidx.text.HAL_I2C_Mem_Write_IT) refers to stm32f0xx_hal_i2c.o(.text.HAL_I2C_Mem_Write_IT) for [Anonymous Symbol]
    stm32f0xx_hal_i2c.o(.text.I2C_Mem_ISR_IT) refers to stm32f0xx_hal_i2c.o(.text.I2C_ITError) for I2C_ITError
    stm32f0xx_hal_i2c.o(.text.I2C_Mem_ISR_IT) refers to stm32f0xx_hal_i2c.o(.text.I2C_ITMasterCplt) for I2C_ITMasterCplt
    stm32f0xx_hal_i2c.o(.ARM.exidx.text.I2C_Mem_ISR_IT) refers to stm32f0xx_hal_i2c.o(.text.I2C_Mem_ISR_IT) for [Anonymous Symbol]
    stm32f0xx_hal_i2c.o(.text.HAL_I2C_Mem_Read_IT) refers to stm32f0xx_hal_i2c.o(.text.I2C_Mem_ISR_IT) for I2C_Mem_ISR_IT
    stm32f0xx_hal_i2c.o(.ARM.exidx.text.HAL_I2C_Mem_Read_IT) refers to stm32f0xx_hal_i2c.o(.text.HAL_I2C_Mem_Read_IT) for [Anonymous Symbol]
    stm32f0xx_hal_i2c.o(.text.HAL_I2C_Mem_Write_DMA) refers to stm32f0xx_hal_dma.o(.text.HAL_DMA_Start_IT) for HAL_DMA_Start_IT
    stm32f0xx_hal_i2c.o(.text.HAL_I2C_Mem_Write_DMA) refers to stm32f0xx_hal_i2c.o(.text.I2C_Mem_ISR_DMA) for I2C_Mem_ISR_DMA
    stm32f0xx_hal_i2c.o(.text.HAL_I2C_Mem_Write_DMA) refers to stm32f0xx_hal_i2c.o(.text.I2C_DMAError) for I2C_DMAError
    stm32f0xx_hal_i2c.o(.text.HAL_I2C_Mem_Write_DMA) refers to stm32f0xx_hal_i2c.o(.text.I2C_DMAMasterTransmitCplt) for I2C_DMAMasterTransmitCplt
    stm32f0xx_hal_i2c.o(.ARM.exidx.text.HAL_I2C_Mem_Write_DMA) refers to stm32f0xx_hal_i2c.o(.text.HAL_I2C_Mem_Write_DMA) for [Anonymous Symbol]
    stm32f0xx_hal_i2c.o(.text.I2C_Mem_ISR_DMA) refers to stm32f0xx_hal_i2c.o(.text.I2C_ITMasterCplt) for I2C_ITMasterCplt
    stm32f0xx_hal_i2c.o(.text.I2C_Mem_ISR_DMA) refers to stm32f0xx_hal_i2c.o(.text.I2C_ITError) for I2C_ITError
    stm32f0xx_hal_i2c.o(.text.I2C_Mem_ISR_DMA) refers to stm32f0xx_hal_i2c.o(.text.I2C_Slave_ISR_DMA) for I2C_Slave_ISR_DMA
    stm32f0xx_hal_i2c.o(.text.I2C_Mem_ISR_DMA) refers to stm32f0xx_hal_i2c.o(.text.I2C_Master_ISR_DMA) for I2C_Master_ISR_DMA
    stm32f0xx_hal_i2c.o(.ARM.exidx.text.I2C_Mem_ISR_DMA) refers to stm32f0xx_hal_i2c.o(.text.I2C_Mem_ISR_DMA) for [Anonymous Symbol]
    stm32f0xx_hal_i2c.o(.text.HAL_I2C_Mem_Read_DMA) refers to stm32f0xx_hal_dma.o(.text.HAL_DMA_Start_IT) for HAL_DMA_Start_IT
    stm32f0xx_hal_i2c.o(.text.HAL_I2C_Mem_Read_DMA) refers to stm32f0xx_hal_i2c.o(.text.I2C_Mem_ISR_DMA) for I2C_Mem_ISR_DMA
    stm32f0xx_hal_i2c.o(.text.HAL_I2C_Mem_Read_DMA) refers to stm32f0xx_hal_i2c.o(.text.I2C_DMAError) for I2C_DMAError
    stm32f0xx_hal_i2c.o(.text.HAL_I2C_Mem_Read_DMA) refers to stm32f0xx_hal_i2c.o(.text.I2C_DMAMasterReceiveCplt) for I2C_DMAMasterReceiveCplt
    stm32f0xx_hal_i2c.o(.ARM.exidx.text.HAL_I2C_Mem_Read_DMA) refers to stm32f0xx_hal_i2c.o(.text.HAL_I2C_Mem_Read_DMA) for [Anonymous Symbol]
    stm32f0xx_hal_i2c.o(.text.HAL_I2C_IsDeviceReady) refers to stm32f0xx_hal.o(.text.HAL_GetTick) for HAL_GetTick
    stm32f0xx_hal_i2c.o(.text.HAL_I2C_IsDeviceReady) refers to stm32f0xx_hal_i2c.o(.text.I2C_WaitOnFlagUntilTimeout) for I2C_WaitOnFlagUntilTimeout
    stm32f0xx_hal_i2c.o(.ARM.exidx.text.HAL_I2C_IsDeviceReady) refers to stm32f0xx_hal_i2c.o(.text.HAL_I2C_IsDeviceReady) for [Anonymous Symbol]
    stm32f0xx_hal_i2c.o(.text.HAL_I2C_Master_Seq_Transmit_IT) refers to stm32f0xx_hal_i2c.o(.text.I2C_Master_ISR_IT) for I2C_Master_ISR_IT
    stm32f0xx_hal_i2c.o(.ARM.exidx.text.HAL_I2C_Master_Seq_Transmit_IT) refers to stm32f0xx_hal_i2c.o(.text.HAL_I2C_Master_Seq_Transmit_IT) for [Anonymous Symbol]
    stm32f0xx_hal_i2c.o(.text.HAL_I2C_Master_Seq_Transmit_DMA) refers to stm32f0xx_hal_dma.o(.text.HAL_DMA_Start_IT) for HAL_DMA_Start_IT
    stm32f0xx_hal_i2c.o(.text.HAL_I2C_Master_Seq_Transmit_DMA) refers to stm32f0xx_hal_i2c.o(.text.I2C_Master_ISR_DMA) for I2C_Master_ISR_DMA
    stm32f0xx_hal_i2c.o(.text.HAL_I2C_Master_Seq_Transmit_DMA) refers to stm32f0xx_hal_i2c.o(.text.I2C_DMAError) for I2C_DMAError
    stm32f0xx_hal_i2c.o(.text.HAL_I2C_Master_Seq_Transmit_DMA) refers to stm32f0xx_hal_i2c.o(.text.I2C_DMAMasterTransmitCplt) for I2C_DMAMasterTransmitCplt
    stm32f0xx_hal_i2c.o(.text.HAL_I2C_Master_Seq_Transmit_DMA) refers to stm32f0xx_hal_i2c.o(.text.I2C_Master_ISR_IT) for I2C_Master_ISR_IT
    stm32f0xx_hal_i2c.o(.ARM.exidx.text.HAL_I2C_Master_Seq_Transmit_DMA) refers to stm32f0xx_hal_i2c.o(.text.HAL_I2C_Master_Seq_Transmit_DMA) for [Anonymous Symbol]
    stm32f0xx_hal_i2c.o(.text.HAL_I2C_Master_Seq_Receive_IT) refers to stm32f0xx_hal_i2c.o(.text.I2C_Master_ISR_IT) for I2C_Master_ISR_IT
    stm32f0xx_hal_i2c.o(.ARM.exidx.text.HAL_I2C_Master_Seq_Receive_IT) refers to stm32f0xx_hal_i2c.o(.text.HAL_I2C_Master_Seq_Receive_IT) for [Anonymous Symbol]
    stm32f0xx_hal_i2c.o(.text.HAL_I2C_Master_Seq_Receive_DMA) refers to stm32f0xx_hal_dma.o(.text.HAL_DMA_Start_IT) for HAL_DMA_Start_IT
    stm32f0xx_hal_i2c.o(.text.HAL_I2C_Master_Seq_Receive_DMA) refers to stm32f0xx_hal_i2c.o(.text.I2C_Master_ISR_DMA) for I2C_Master_ISR_DMA
    stm32f0xx_hal_i2c.o(.text.HAL_I2C_Master_Seq_Receive_DMA) refers to stm32f0xx_hal_i2c.o(.text.I2C_DMAError) for I2C_DMAError
    stm32f0xx_hal_i2c.o(.text.HAL_I2C_Master_Seq_Receive_DMA) refers to stm32f0xx_hal_i2c.o(.text.I2C_DMAMasterReceiveCplt) for I2C_DMAMasterReceiveCplt
    stm32f0xx_hal_i2c.o(.text.HAL_I2C_Master_Seq_Receive_DMA) refers to stm32f0xx_hal_i2c.o(.text.I2C_Master_ISR_IT) for I2C_Master_ISR_IT
    stm32f0xx_hal_i2c.o(.ARM.exidx.text.HAL_I2C_Master_Seq_Receive_DMA) refers to stm32f0xx_hal_i2c.o(.text.HAL_I2C_Master_Seq_Receive_DMA) for [Anonymous Symbol]
    stm32f0xx_hal_i2c.o(.text.HAL_I2C_Slave_Seq_Transmit_IT) refers to stm32f0xx_hal_dma.o(.text.HAL_DMA_Abort_IT) for HAL_DMA_Abort_IT
    stm32f0xx_hal_i2c.o(.text.HAL_I2C_Slave_Seq_Transmit_IT) refers to stm32f0xx_hal_i2c.o(.text.I2C_DMAAbort) for I2C_DMAAbort
    stm32f0xx_hal_i2c.o(.text.HAL_I2C_Slave_Seq_Transmit_IT) refers to stm32f0xx_hal_i2c.o(.text.I2C_Slave_ISR_IT) for I2C_Slave_ISR_IT
    stm32f0xx_hal_i2c.o(.ARM.exidx.text.HAL_I2C_Slave_Seq_Transmit_IT) refers to stm32f0xx_hal_i2c.o(.text.HAL_I2C_Slave_Seq_Transmit_IT) for [Anonymous Symbol]
    stm32f0xx_hal_i2c.o(.text.I2C_DMAAbort) refers to stm32f0xx_hal_i2c.o(.text.HAL_I2C_AbortCpltCallback) for HAL_I2C_AbortCpltCallback
    stm32f0xx_hal_i2c.o(.text.I2C_DMAAbort) refers to stm32f0xx_hal_i2c.o(.text.HAL_I2C_ErrorCallback) for HAL_I2C_ErrorCallback
    stm32f0xx_hal_i2c.o(.ARM.exidx.text.I2C_DMAAbort) refers to stm32f0xx_hal_i2c.o(.text.I2C_DMAAbort) for [Anonymous Symbol]
    stm32f0xx_hal_i2c.o(.text.HAL_I2C_Slave_Seq_Transmit_DMA) refers to stm32f0xx_hal_dma.o(.text.HAL_DMA_Abort_IT) for HAL_DMA_Abort_IT
    stm32f0xx_hal_i2c.o(.text.HAL_I2C_Slave_Seq_Transmit_DMA) refers to stm32f0xx_hal_dma.o(.text.HAL_DMA_Start_IT) for HAL_DMA_Start_IT
    stm32f0xx_hal_i2c.o(.text.HAL_I2C_Slave_Seq_Transmit_DMA) refers to stm32f0xx_hal_i2c.o(.text.I2C_DMAAbort) for I2C_DMAAbort
    stm32f0xx_hal_i2c.o(.text.HAL_I2C_Slave_Seq_Transmit_DMA) refers to stm32f0xx_hal_i2c.o(.text.I2C_Slave_ISR_DMA) for I2C_Slave_ISR_DMA
    stm32f0xx_hal_i2c.o(.text.HAL_I2C_Slave_Seq_Transmit_DMA) refers to stm32f0xx_hal_i2c.o(.text.I2C_DMAError) for I2C_DMAError
    stm32f0xx_hal_i2c.o(.text.HAL_I2C_Slave_Seq_Transmit_DMA) refers to stm32f0xx_hal_i2c.o(.text.I2C_DMASlaveTransmitCplt) for I2C_DMASlaveTransmitCplt
    stm32f0xx_hal_i2c.o(.ARM.exidx.text.HAL_I2C_Slave_Seq_Transmit_DMA) refers to stm32f0xx_hal_i2c.o(.text.HAL_I2C_Slave_Seq_Transmit_DMA) for [Anonymous Symbol]
    stm32f0xx_hal_i2c.o(.text.HAL_I2C_Slave_Seq_Receive_IT) refers to stm32f0xx_hal_dma.o(.text.HAL_DMA_Abort_IT) for HAL_DMA_Abort_IT
    stm32f0xx_hal_i2c.o(.text.HAL_I2C_Slave_Seq_Receive_IT) refers to stm32f0xx_hal_i2c.o(.text.I2C_DMAAbort) for I2C_DMAAbort
    stm32f0xx_hal_i2c.o(.text.HAL_I2C_Slave_Seq_Receive_IT) refers to stm32f0xx_hal_i2c.o(.text.I2C_Slave_ISR_IT) for I2C_Slave_ISR_IT
    stm32f0xx_hal_i2c.o(.ARM.exidx.text.HAL_I2C_Slave_Seq_Receive_IT) refers to stm32f0xx_hal_i2c.o(.text.HAL_I2C_Slave_Seq_Receive_IT) for [Anonymous Symbol]
    stm32f0xx_hal_i2c.o(.text.HAL_I2C_Slave_Seq_Receive_DMA) refers to stm32f0xx_hal_dma.o(.text.HAL_DMA_Abort_IT) for HAL_DMA_Abort_IT
    stm32f0xx_hal_i2c.o(.text.HAL_I2C_Slave_Seq_Receive_DMA) refers to stm32f0xx_hal_dma.o(.text.HAL_DMA_Start_IT) for HAL_DMA_Start_IT
    stm32f0xx_hal_i2c.o(.text.HAL_I2C_Slave_Seq_Receive_DMA) refers to stm32f0xx_hal_i2c.o(.text.I2C_DMAAbort) for I2C_DMAAbort
    stm32f0xx_hal_i2c.o(.text.HAL_I2C_Slave_Seq_Receive_DMA) refers to stm32f0xx_hal_i2c.o(.text.I2C_Slave_ISR_DMA) for I2C_Slave_ISR_DMA
    stm32f0xx_hal_i2c.o(.text.HAL_I2C_Slave_Seq_Receive_DMA) refers to stm32f0xx_hal_i2c.o(.text.I2C_DMAError) for I2C_DMAError
    stm32f0xx_hal_i2c.o(.text.HAL_I2C_Slave_Seq_Receive_DMA) refers to stm32f0xx_hal_i2c.o(.text.I2C_DMASlaveReceiveCplt) for I2C_DMASlaveReceiveCplt
    stm32f0xx_hal_i2c.o(.ARM.exidx.text.HAL_I2C_Slave_Seq_Receive_DMA) refers to stm32f0xx_hal_i2c.o(.text.HAL_I2C_Slave_Seq_Receive_DMA) for [Anonymous Symbol]
    stm32f0xx_hal_i2c.o(.text.HAL_I2C_EnableListen_IT) refers to stm32f0xx_hal_i2c.o(.text.I2C_Slave_ISR_IT) for I2C_Slave_ISR_IT
    stm32f0xx_hal_i2c.o(.ARM.exidx.text.HAL_I2C_EnableListen_IT) refers to stm32f0xx_hal_i2c.o(.text.HAL_I2C_EnableListen_IT) for [Anonymous Symbol]
    stm32f0xx_hal_i2c.o(.ARM.exidx.text.HAL_I2C_DisableListen_IT) refers to stm32f0xx_hal_i2c.o(.text.HAL_I2C_DisableListen_IT) for [Anonymous Symbol]
    stm32f0xx_hal_i2c.o(.text.HAL_I2C_Master_Abort_IT) refers to stm32f0xx_hal_i2c.o(.text.I2C_Slave_ISR_DMA) for I2C_Slave_ISR_DMA
    stm32f0xx_hal_i2c.o(.text.HAL_I2C_Master_Abort_IT) refers to stm32f0xx_hal_i2c.o(.text.I2C_Master_ISR_DMA) for I2C_Master_ISR_DMA
    stm32f0xx_hal_i2c.o(.text.HAL_I2C_Master_Abort_IT) refers to stm32f0xx_hal_i2c.o(.text.I2C_Mem_ISR_DMA) for I2C_Mem_ISR_DMA
    stm32f0xx_hal_i2c.o(.ARM.exidx.text.HAL_I2C_Master_Abort_IT) refers to stm32f0xx_hal_i2c.o(.text.HAL_I2C_Master_Abort_IT) for [Anonymous Symbol]
    stm32f0xx_hal_i2c.o(.ARM.exidx.text.HAL_I2C_EV_IRQHandler) refers to stm32f0xx_hal_i2c.o(.text.HAL_I2C_EV_IRQHandler) for [Anonymous Symbol]
    stm32f0xx_hal_i2c.o(.text.HAL_I2C_ER_IRQHandler) refers to stm32f0xx_hal_i2c.o(.text.I2C_ITError) for I2C_ITError
    stm32f0xx_hal_i2c.o(.ARM.exidx.text.HAL_I2C_ER_IRQHandler) refers to stm32f0xx_hal_i2c.o(.text.HAL_I2C_ER_IRQHandler) for [Anonymous Symbol]
    stm32f0xx_hal_i2c.o(.text.I2C_ITError) refers to stm32f0xx_hal_dma.o(.text.HAL_DMA_GetState) for HAL_DMA_GetState
    stm32f0xx_hal_i2c.o(.text.I2C_ITError) refers to stm32f0xx_hal_dma.o(.text.HAL_DMA_Abort_IT) for HAL_DMA_Abort_IT
    stm32f0xx_hal_i2c.o(.text.I2C_ITError) refers to stm32f0xx_hal_i2c.o(.text.HAL_I2C_AbortCpltCallback) for HAL_I2C_AbortCpltCallback
    stm32f0xx_hal_i2c.o(.text.I2C_ITError) refers to stm32f0xx_hal_i2c.o(.text.HAL_I2C_ErrorCallback) for HAL_I2C_ErrorCallback
    stm32f0xx_hal_i2c.o(.text.I2C_ITError) refers to stm32f0xx_hal_i2c.o(.text.I2C_Slave_ISR_IT) for I2C_Slave_ISR_IT
    stm32f0xx_hal_i2c.o(.text.I2C_ITError) refers to stm32f0xx_hal_i2c.o(.text.I2C_DMAAbort) for I2C_DMAAbort
    stm32f0xx_hal_i2c.o(.ARM.exidx.text.I2C_ITError) refers to stm32f0xx_hal_i2c.o(.text.I2C_ITError) for [Anonymous Symbol]
    stm32f0xx_hal_i2c.o(.ARM.exidx.text.HAL_I2C_MasterTxCpltCallback) refers to stm32f0xx_hal_i2c.o(.text.HAL_I2C_MasterTxCpltCallback) for [Anonymous Symbol]
    stm32f0xx_hal_i2c.o(.ARM.exidx.text.HAL_I2C_MasterRxCpltCallback) refers to stm32f0xx_hal_i2c.o(.text.HAL_I2C_MasterRxCpltCallback) for [Anonymous Symbol]
    stm32f0xx_hal_i2c.o(.ARM.exidx.text.HAL_I2C_SlaveTxCpltCallback) refers to stm32f0xx_hal_i2c.o(.text.HAL_I2C_SlaveTxCpltCallback) for [Anonymous Symbol]
    stm32f0xx_hal_i2c.o(.ARM.exidx.text.HAL_I2C_SlaveRxCpltCallback) refers to stm32f0xx_hal_i2c.o(.text.HAL_I2C_SlaveRxCpltCallback) for [Anonymous Symbol]
    stm32f0xx_hal_i2c.o(.ARM.exidx.text.HAL_I2C_AddrCallback) refers to stm32f0xx_hal_i2c.o(.text.HAL_I2C_AddrCallback) for [Anonymous Symbol]
    stm32f0xx_hal_i2c.o(.ARM.exidx.text.HAL_I2C_ListenCpltCallback) refers to stm32f0xx_hal_i2c.o(.text.HAL_I2C_ListenCpltCallback) for [Anonymous Symbol]
    stm32f0xx_hal_i2c.o(.ARM.exidx.text.HAL_I2C_MemTxCpltCallback) refers to stm32f0xx_hal_i2c.o(.text.HAL_I2C_MemTxCpltCallback) for [Anonymous Symbol]
    stm32f0xx_hal_i2c.o(.ARM.exidx.text.HAL_I2C_MemRxCpltCallback) refers to stm32f0xx_hal_i2c.o(.text.HAL_I2C_MemRxCpltCallback) for [Anonymous Symbol]
    stm32f0xx_hal_i2c.o(.ARM.exidx.text.HAL_I2C_ErrorCallback) refers to stm32f0xx_hal_i2c.o(.text.HAL_I2C_ErrorCallback) for [Anonymous Symbol]
    stm32f0xx_hal_i2c.o(.ARM.exidx.text.HAL_I2C_AbortCpltCallback) refers to stm32f0xx_hal_i2c.o(.text.HAL_I2C_AbortCpltCallback) for [Anonymous Symbol]
    stm32f0xx_hal_i2c.o(.ARM.exidx.text.HAL_I2C_GetState) refers to stm32f0xx_hal_i2c.o(.text.HAL_I2C_GetState) for [Anonymous Symbol]
    stm32f0xx_hal_i2c.o(.ARM.exidx.text.HAL_I2C_GetMode) refers to stm32f0xx_hal_i2c.o(.text.HAL_I2C_GetMode) for [Anonymous Symbol]
    stm32f0xx_hal_i2c.o(.ARM.exidx.text.HAL_I2C_GetError) refers to stm32f0xx_hal_i2c.o(.text.HAL_I2C_GetError) for [Anonymous Symbol]
    stm32f0xx_hal_i2c.o(.text.I2C_ITMasterSeqCplt) refers to stm32f0xx_hal_i2c.o(.text.HAL_I2C_MasterRxCpltCallback) for HAL_I2C_MasterRxCpltCallback
    stm32f0xx_hal_i2c.o(.text.I2C_ITMasterSeqCplt) refers to stm32f0xx_hal_i2c.o(.text.HAL_I2C_MasterTxCpltCallback) for HAL_I2C_MasterTxCpltCallback
    stm32f0xx_hal_i2c.o(.ARM.exidx.text.I2C_ITMasterSeqCplt) refers to stm32f0xx_hal_i2c.o(.text.I2C_ITMasterSeqCplt) for [Anonymous Symbol]
    stm32f0xx_hal_i2c.o(.text.I2C_ITMasterCplt) refers to stm32f0xx_hal_i2c.o(.text.HAL_I2C_MemTxCpltCallback) for HAL_I2C_MemTxCpltCallback
    stm32f0xx_hal_i2c.o(.text.I2C_ITMasterCplt) refers to stm32f0xx_hal_i2c.o(.text.I2C_ITError) for I2C_ITError
    stm32f0xx_hal_i2c.o(.text.I2C_ITMasterCplt) refers to stm32f0xx_hal_i2c.o(.text.HAL_I2C_MemRxCpltCallback) for HAL_I2C_MemRxCpltCallback
    stm32f0xx_hal_i2c.o(.text.I2C_ITMasterCplt) refers to stm32f0xx_hal_i2c.o(.text.HAL_I2C_MasterTxCpltCallback) for HAL_I2C_MasterTxCpltCallback
    stm32f0xx_hal_i2c.o(.text.I2C_ITMasterCplt) refers to stm32f0xx_hal_i2c.o(.text.HAL_I2C_MasterRxCpltCallback) for HAL_I2C_MasterRxCpltCallback
    stm32f0xx_hal_i2c.o(.ARM.exidx.text.I2C_ITMasterCplt) refers to stm32f0xx_hal_i2c.o(.text.I2C_ITMasterCplt) for [Anonymous Symbol]
    stm32f0xx_hal_i2c.o(.text.I2C_ITSlaveCplt) refers to stm32f0xx_hal_i2c.o(.text.I2C_ITError) for I2C_ITError
    stm32f0xx_hal_i2c.o(.text.I2C_ITSlaveCplt) refers to stm32f0xx_hal_i2c.o(.text.HAL_I2C_ListenCpltCallback) for HAL_I2C_ListenCpltCallback
    stm32f0xx_hal_i2c.o(.text.I2C_ITSlaveCplt) refers to stm32f0xx_hal_i2c.o(.text.HAL_I2C_SlaveRxCpltCallback) for HAL_I2C_SlaveRxCpltCallback
    stm32f0xx_hal_i2c.o(.text.I2C_ITSlaveCplt) refers to stm32f0xx_hal_i2c.o(.text.HAL_I2C_SlaveTxCpltCallback) for HAL_I2C_SlaveTxCpltCallback
    stm32f0xx_hal_i2c.o(.ARM.exidx.text.I2C_ITSlaveCplt) refers to stm32f0xx_hal_i2c.o(.text.I2C_ITSlaveCplt) for [Anonymous Symbol]
    stm32f0xx_hal_i2c.o(.text.I2C_ITListenCplt) refers to stm32f0xx_hal_i2c.o(.text.HAL_I2C_ListenCpltCallback) for HAL_I2C_ListenCpltCallback
    stm32f0xx_hal_i2c.o(.ARM.exidx.text.I2C_ITListenCplt) refers to stm32f0xx_hal_i2c.o(.text.I2C_ITListenCplt) for [Anonymous Symbol]
    stm32f0xx_hal_i2c.o(.text.I2C_ITSlaveSeqCplt) refers to stm32f0xx_hal_i2c.o(.text.HAL_I2C_SlaveRxCpltCallback) for HAL_I2C_SlaveRxCpltCallback
    stm32f0xx_hal_i2c.o(.text.I2C_ITSlaveSeqCplt) refers to stm32f0xx_hal_i2c.o(.text.HAL_I2C_SlaveTxCpltCallback) for HAL_I2C_SlaveTxCpltCallback
    stm32f0xx_hal_i2c.o(.ARM.exidx.text.I2C_ITSlaveSeqCplt) refers to stm32f0xx_hal_i2c.o(.text.I2C_ITSlaveSeqCplt) for [Anonymous Symbol]
    stm32f0xx_hal_i2c.o(.text.I2C_ITAddrCplt) refers to stm32f0xx_hal_i2c.o(.text.HAL_I2C_AddrCallback) for HAL_I2C_AddrCallback
    stm32f0xx_hal_i2c.o(.ARM.exidx.text.I2C_ITAddrCplt) refers to stm32f0xx_hal_i2c.o(.text.I2C_ITAddrCplt) for [Anonymous Symbol]
    stm32f0xx_hal_i2c.o(.text.I2C_IsErrorOccurred) refers to stm32f0xx_hal.o(.text.HAL_GetTick) for HAL_GetTick
    stm32f0xx_hal_i2c.o(.ARM.exidx.text.I2C_IsErrorOccurred) refers to stm32f0xx_hal_i2c.o(.text.I2C_IsErrorOccurred) for [Anonymous Symbol]
    stm32f0xx_hal_i2c_ex.o(.ARM.exidx.text.HAL_I2CEx_ConfigAnalogFilter) refers to stm32f0xx_hal_i2c_ex.o(.text.HAL_I2CEx_ConfigAnalogFilter) for [Anonymous Symbol]
    stm32f0xx_hal_i2c_ex.o(.ARM.exidx.text.HAL_I2CEx_ConfigDigitalFilter) refers to stm32f0xx_hal_i2c_ex.o(.text.HAL_I2CEx_ConfigDigitalFilter) for [Anonymous Symbol]
    stm32f0xx_hal_i2c_ex.o(.ARM.exidx.text.HAL_I2CEx_EnableFastModePlus) refers to stm32f0xx_hal_i2c_ex.o(.text.HAL_I2CEx_EnableFastModePlus) for [Anonymous Symbol]
    stm32f0xx_hal_i2c_ex.o(.ARM.exidx.text.HAL_I2CEx_DisableFastModePlus) refers to stm32f0xx_hal_i2c_ex.o(.text.HAL_I2CEx_DisableFastModePlus) for [Anonymous Symbol]
    stm32f0xx_hal_rcc.o(.text.HAL_RCC_DeInit) refers to stm32f0xx_hal.o(.text.HAL_GetTick) for HAL_GetTick
    stm32f0xx_hal_rcc.o(.text.HAL_RCC_DeInit) refers to stm32f0xx_hal.o(.text.HAL_InitTick) for HAL_InitTick
    stm32f0xx_hal_rcc.o(.text.HAL_RCC_DeInit) refers to system_stm32f0xx.o(.data.SystemCoreClock) for SystemCoreClock
    stm32f0xx_hal_rcc.o(.text.HAL_RCC_DeInit) refers to stm32f0xx_hal.o(.data..L_MergedGlobals) for uwTickPrio
    stm32f0xx_hal_rcc.o(.ARM.exidx.text.HAL_RCC_DeInit) refers to stm32f0xx_hal_rcc.o(.text.HAL_RCC_DeInit) for [Anonymous Symbol]
    stm32f0xx_hal_rcc.o(.text.HAL_RCC_OscConfig) refers to stm32f0xx_hal.o(.text.HAL_GetTick) for HAL_GetTick
    stm32f0xx_hal_rcc.o(.ARM.exidx.text.HAL_RCC_OscConfig) refers to stm32f0xx_hal_rcc.o(.text.HAL_RCC_OscConfig) for [Anonymous Symbol]
    stm32f0xx_hal_rcc.o(.text.HAL_RCC_ClockConfig) refers to aeabi_sdivfast.o(.text_divfast) for __aeabi_uidiv
    stm32f0xx_hal_rcc.o(.text.HAL_RCC_ClockConfig) refers to stm32f0xx_hal.o(.text.HAL_InitTick) for HAL_InitTick
    stm32f0xx_hal_rcc.o(.text.HAL_RCC_ClockConfig) refers to stm32f0xx_hal.o(.text.HAL_GetTick) for HAL_GetTick
    stm32f0xx_hal_rcc.o(.text.HAL_RCC_ClockConfig) refers to stm32f0xx_hal_rcc.o(.rodata.cst16) for [Anonymous Symbol]
    stm32f0xx_hal_rcc.o(.text.HAL_RCC_ClockConfig) refers to system_stm32f0xx.o(.rodata.AHBPrescTable) for AHBPrescTable
    stm32f0xx_hal_rcc.o(.text.HAL_RCC_ClockConfig) refers to system_stm32f0xx.o(.data.SystemCoreClock) for SystemCoreClock
    stm32f0xx_hal_rcc.o(.ARM.exidx.text.HAL_RCC_ClockConfig) refers to stm32f0xx_hal_rcc.o(.text.HAL_RCC_ClockConfig) for [Anonymous Symbol]
    stm32f0xx_hal_rcc.o(.text.HAL_RCC_GetSysClockFreq) refers to aeabi_sdivfast.o(.text_divfast) for __aeabi_uidiv
    stm32f0xx_hal_rcc.o(.text.HAL_RCC_GetSysClockFreq) refers to stm32f0xx_hal_rcc.o(.rodata.cst16) for [Anonymous Symbol]
    stm32f0xx_hal_rcc.o(.ARM.exidx.text.HAL_RCC_GetSysClockFreq) refers to stm32f0xx_hal_rcc.o(.text.HAL_RCC_GetSysClockFreq) for [Anonymous Symbol]
    stm32f0xx_hal_rcc.o(.text.HAL_RCC_MCOConfig) refers to stm32f0xx_hal_gpio.o(.text.HAL_GPIO_Init) for HAL_GPIO_Init
    stm32f0xx_hal_rcc.o(.ARM.exidx.text.HAL_RCC_MCOConfig) refers to stm32f0xx_hal_rcc.o(.text.HAL_RCC_MCOConfig) for [Anonymous Symbol]
    stm32f0xx_hal_rcc.o(.ARM.exidx.text.HAL_RCC_EnableCSS) refers to stm32f0xx_hal_rcc.o(.text.HAL_RCC_EnableCSS) for [Anonymous Symbol]
    stm32f0xx_hal_rcc.o(.ARM.exidx.text.HAL_RCC_DisableCSS) refers to stm32f0xx_hal_rcc.o(.text.HAL_RCC_DisableCSS) for [Anonymous Symbol]
    stm32f0xx_hal_rcc.o(.text.HAL_RCC_GetHCLKFreq) refers to system_stm32f0xx.o(.data.SystemCoreClock) for SystemCoreClock
    stm32f0xx_hal_rcc.o(.ARM.exidx.text.HAL_RCC_GetHCLKFreq) refers to stm32f0xx_hal_rcc.o(.text.HAL_RCC_GetHCLKFreq) for [Anonymous Symbol]
    stm32f0xx_hal_rcc.o(.text.HAL_RCC_GetPCLK1Freq) refers to system_stm32f0xx.o(.data.SystemCoreClock) for SystemCoreClock
    stm32f0xx_hal_rcc.o(.text.HAL_RCC_GetPCLK1Freq) refers to system_stm32f0xx.o(.rodata.APBPrescTable) for APBPrescTable
    stm32f0xx_hal_rcc.o(.ARM.exidx.text.HAL_RCC_GetPCLK1Freq) refers to stm32f0xx_hal_rcc.o(.text.HAL_RCC_GetPCLK1Freq) for [Anonymous Symbol]
    stm32f0xx_hal_rcc.o(.ARM.exidx.text.HAL_RCC_GetOscConfig) refers to stm32f0xx_hal_rcc.o(.text.HAL_RCC_GetOscConfig) for [Anonymous Symbol]
    stm32f0xx_hal_rcc.o(.ARM.exidx.text.HAL_RCC_GetClockConfig) refers to stm32f0xx_hal_rcc.o(.text.HAL_RCC_GetClockConfig) for [Anonymous Symbol]
    stm32f0xx_hal_rcc.o(.text.HAL_RCC_NMI_IRQHandler) refers to stm32f0xx_hal_rcc.o(.text.HAL_RCC_CSSCallback) for HAL_RCC_CSSCallback
    stm32f0xx_hal_rcc.o(.ARM.exidx.text.HAL_RCC_NMI_IRQHandler) refers to stm32f0xx_hal_rcc.o(.text.HAL_RCC_NMI_IRQHandler) for [Anonymous Symbol]
    stm32f0xx_hal_rcc.o(.ARM.exidx.text.HAL_RCC_CSSCallback) refers to stm32f0xx_hal_rcc.o(.text.HAL_RCC_CSSCallback) for [Anonymous Symbol]
    stm32f0xx_hal_rcc_ex.o(.text.HAL_RCCEx_PeriphCLKConfig) refers to stm32f0xx_hal.o(.text.HAL_GetTick) for HAL_GetTick
    stm32f0xx_hal_rcc_ex.o(.ARM.exidx.text.HAL_RCCEx_PeriphCLKConfig) refers to stm32f0xx_hal_rcc_ex.o(.text.HAL_RCCEx_PeriphCLKConfig) for [Anonymous Symbol]
    stm32f0xx_hal_rcc_ex.o(.ARM.exidx.text.HAL_RCCEx_GetPeriphCLKConfig) refers to stm32f0xx_hal_rcc_ex.o(.text.HAL_RCCEx_GetPeriphCLKConfig) for [Anonymous Symbol]
    stm32f0xx_hal_rcc_ex.o(.text.HAL_RCCEx_GetPeriphCLKFreq) refers to stm32f0xx_hal_rcc.o(.text.HAL_RCC_GetPCLK1Freq) for HAL_RCC_GetPCLK1Freq
    stm32f0xx_hal_rcc_ex.o(.text.HAL_RCCEx_GetPeriphCLKFreq) refers to stm32f0xx_hal_rcc.o(.text.HAL_RCC_GetSysClockFreq) for HAL_RCC_GetSysClockFreq
    stm32f0xx_hal_rcc_ex.o(.ARM.exidx.text.HAL_RCCEx_GetPeriphCLKFreq) refers to stm32f0xx_hal_rcc_ex.o(.text.HAL_RCCEx_GetPeriphCLKFreq) for [Anonymous Symbol]
    stm32f0xx_hal.o(.text.HAL_Init) refers to stm32f0xx_hal.o(.text.HAL_InitTick) for HAL_InitTick
    stm32f0xx_hal.o(.text.HAL_Init) refers to stm32f0xx_hal_msp.o(.text.HAL_MspInit) for HAL_MspInit
    stm32f0xx_hal.o(.ARM.exidx.text.HAL_Init) refers to stm32f0xx_hal.o(.text.HAL_Init) for [Anonymous Symbol]
    stm32f0xx_hal.o(.text.HAL_InitTick) refers to aeabi_sdivfast.o(.text_divfast) for __aeabi_uidiv
    stm32f0xx_hal.o(.text.HAL_InitTick) refers to stm32f0xx_hal_cortex.o(.text.HAL_SYSTICK_Config) for HAL_SYSTICK_Config
    stm32f0xx_hal.o(.text.HAL_InitTick) refers to stm32f0xx_hal_cortex.o(.text.HAL_NVIC_SetPriority) for HAL_NVIC_SetPriority
    stm32f0xx_hal.o(.text.HAL_InitTick) refers to stm32f0xx_hal.o(.data..L_MergedGlobals) for [Anonymous Symbol]
    stm32f0xx_hal.o(.text.HAL_InitTick) refers to system_stm32f0xx.o(.data.SystemCoreClock) for SystemCoreClock
    stm32f0xx_hal.o(.ARM.exidx.text.HAL_InitTick) refers to stm32f0xx_hal.o(.text.HAL_InitTick) for [Anonymous Symbol]
    stm32f0xx_hal.o(.ARM.exidx.text.HAL_MspInit) refers to stm32f0xx_hal.o(.text.HAL_MspInit) for [Anonymous Symbol]
    stm32f0xx_hal.o(.text.HAL_DeInit) refers to stm32f0xx_hal.o(.text.HAL_MspDeInit) for HAL_MspDeInit
    stm32f0xx_hal.o(.ARM.exidx.text.HAL_DeInit) refers to stm32f0xx_hal.o(.text.HAL_DeInit) for [Anonymous Symbol]
    stm32f0xx_hal.o(.ARM.exidx.text.HAL_MspDeInit) refers to stm32f0xx_hal.o(.text.HAL_MspDeInit) for [Anonymous Symbol]
    stm32f0xx_hal.o(.text.HAL_IncTick) refers to stm32f0xx_hal.o(.data..L_MergedGlobals) for [Anonymous Symbol]
    stm32f0xx_hal.o(.text.HAL_IncTick) refers to stm32f0xx_hal.o(.bss.uwTick) for uwTick
    stm32f0xx_hal.o(.ARM.exidx.text.HAL_IncTick) refers to stm32f0xx_hal.o(.text.HAL_IncTick) for [Anonymous Symbol]
    stm32f0xx_hal.o(.text.HAL_GetTick) refers to stm32f0xx_hal.o(.bss.uwTick) for uwTick
    stm32f0xx_hal.o(.ARM.exidx.text.HAL_GetTick) refers to stm32f0xx_hal.o(.text.HAL_GetTick) for [Anonymous Symbol]
    stm32f0xx_hal.o(.text.HAL_GetTickPrio) refers to stm32f0xx_hal.o(.data..L_MergedGlobals) for [Anonymous Symbol]
    stm32f0xx_hal.o(.ARM.exidx.text.HAL_GetTickPrio) refers to stm32f0xx_hal.o(.text.HAL_GetTickPrio) for [Anonymous Symbol]
    stm32f0xx_hal.o(.text.HAL_SetTickFreq) refers to stm32f0xx_hal.o(.text.HAL_InitTick) for HAL_InitTick
    stm32f0xx_hal.o(.text.HAL_SetTickFreq) refers to stm32f0xx_hal.o(.data..L_MergedGlobals) for [Anonymous Symbol]
    stm32f0xx_hal.o(.ARM.exidx.text.HAL_SetTickFreq) refers to stm32f0xx_hal.o(.text.HAL_SetTickFreq) for [Anonymous Symbol]
    stm32f0xx_hal.o(.text.HAL_GetTickFreq) refers to stm32f0xx_hal.o(.data..L_MergedGlobals) for [Anonymous Symbol]
    stm32f0xx_hal.o(.ARM.exidx.text.HAL_GetTickFreq) refers to stm32f0xx_hal.o(.text.HAL_GetTickFreq) for [Anonymous Symbol]
    stm32f0xx_hal.o(.text.HAL_Delay) refers to stm32f0xx_hal.o(.text.HAL_GetTick) for HAL_GetTick
    stm32f0xx_hal.o(.text.HAL_Delay) refers to stm32f0xx_hal.o(.data..L_MergedGlobals) for [Anonymous Symbol]
    stm32f0xx_hal.o(.ARM.exidx.text.HAL_Delay) refers to stm32f0xx_hal.o(.text.HAL_Delay) for [Anonymous Symbol]
    stm32f0xx_hal.o(.ARM.exidx.text.HAL_SuspendTick) refers to stm32f0xx_hal.o(.text.HAL_SuspendTick) for [Anonymous Symbol]
    stm32f0xx_hal.o(.ARM.exidx.text.HAL_ResumeTick) refers to stm32f0xx_hal.o(.text.HAL_ResumeTick) for [Anonymous Symbol]
    stm32f0xx_hal.o(.ARM.exidx.text.HAL_GetHalVersion) refers to stm32f0xx_hal.o(.text.HAL_GetHalVersion) for [Anonymous Symbol]
    stm32f0xx_hal.o(.ARM.exidx.text.HAL_GetREVID) refers to stm32f0xx_hal.o(.text.HAL_GetREVID) for [Anonymous Symbol]
    stm32f0xx_hal.o(.ARM.exidx.text.HAL_GetDEVID) refers to stm32f0xx_hal.o(.text.HAL_GetDEVID) for [Anonymous Symbol]
    stm32f0xx_hal.o(.ARM.exidx.text.HAL_GetUIDw0) refers to stm32f0xx_hal.o(.text.HAL_GetUIDw0) for [Anonymous Symbol]
    stm32f0xx_hal.o(.ARM.exidx.text.HAL_GetUIDw1) refers to stm32f0xx_hal.o(.text.HAL_GetUIDw1) for [Anonymous Symbol]
    stm32f0xx_hal.o(.ARM.exidx.text.HAL_GetUIDw2) refers to stm32f0xx_hal.o(.text.HAL_GetUIDw2) for [Anonymous Symbol]
    stm32f0xx_hal.o(.ARM.exidx.text.HAL_DBGMCU_EnableDBGStopMode) refers to stm32f0xx_hal.o(.text.HAL_DBGMCU_EnableDBGStopMode) for [Anonymous Symbol]
    stm32f0xx_hal.o(.ARM.exidx.text.HAL_DBGMCU_DisableDBGStopMode) refers to stm32f0xx_hal.o(.text.HAL_DBGMCU_DisableDBGStopMode) for [Anonymous Symbol]
    stm32f0xx_hal.o(.ARM.exidx.text.HAL_DBGMCU_EnableDBGStandbyMode) refers to stm32f0xx_hal.o(.text.HAL_DBGMCU_EnableDBGStandbyMode) for [Anonymous Symbol]
    stm32f0xx_hal.o(.ARM.exidx.text.HAL_DBGMCU_DisableDBGStandbyMode) refers to stm32f0xx_hal.o(.text.HAL_DBGMCU_DisableDBGStandbyMode) for [Anonymous Symbol]
    stm32f0xx_hal_gpio.o(.ARM.exidx.text.HAL_GPIO_Init) refers to stm32f0xx_hal_gpio.o(.text.HAL_GPIO_Init) for [Anonymous Symbol]
    stm32f0xx_hal_gpio.o(.ARM.exidx.text.HAL_GPIO_DeInit) refers to stm32f0xx_hal_gpio.o(.text.HAL_GPIO_DeInit) for [Anonymous Symbol]
    stm32f0xx_hal_gpio.o(.ARM.exidx.text.HAL_GPIO_ReadPin) refers to stm32f0xx_hal_gpio.o(.text.HAL_GPIO_ReadPin) for [Anonymous Symbol]
    stm32f0xx_hal_gpio.o(.ARM.exidx.text.HAL_GPIO_WritePin) refers to stm32f0xx_hal_gpio.o(.text.HAL_GPIO_WritePin) for [Anonymous Symbol]
    stm32f0xx_hal_gpio.o(.ARM.exidx.text.HAL_GPIO_TogglePin) refers to stm32f0xx_hal_gpio.o(.text.HAL_GPIO_TogglePin) for [Anonymous Symbol]
    stm32f0xx_hal_gpio.o(.ARM.exidx.text.HAL_GPIO_LockPin) refers to stm32f0xx_hal_gpio.o(.text.HAL_GPIO_LockPin) for [Anonymous Symbol]
    stm32f0xx_hal_gpio.o(.text.HAL_GPIO_EXTI_IRQHandler) refers to stm32f0xx_hal_gpio.o(.text.HAL_GPIO_EXTI_Callback) for HAL_GPIO_EXTI_Callback
    stm32f0xx_hal_gpio.o(.ARM.exidx.text.HAL_GPIO_EXTI_IRQHandler) refers to stm32f0xx_hal_gpio.o(.text.HAL_GPIO_EXTI_IRQHandler) for [Anonymous Symbol]
    stm32f0xx_hal_gpio.o(.ARM.exidx.text.HAL_GPIO_EXTI_Callback) refers to stm32f0xx_hal_gpio.o(.text.HAL_GPIO_EXTI_Callback) for [Anonymous Symbol]
    stm32f0xx_hal_dma.o(.text.HAL_DMA_Init) refers to aeabi_sdivfast.o(.text_divfast) for __aeabi_uidiv
    stm32f0xx_hal_dma.o(.ARM.exidx.text.HAL_DMA_Init) refers to stm32f0xx_hal_dma.o(.text.HAL_DMA_Init) for [Anonymous Symbol]
    stm32f0xx_hal_dma.o(.text.HAL_DMA_DeInit) refers to aeabi_sdivfast.o(.text_divfast) for __aeabi_uidiv
    stm32f0xx_hal_dma.o(.ARM.exidx.text.HAL_DMA_DeInit) refers to stm32f0xx_hal_dma.o(.text.HAL_DMA_DeInit) for [Anonymous Symbol]
    stm32f0xx_hal_dma.o(.ARM.exidx.text.HAL_DMA_Start) refers to stm32f0xx_hal_dma.o(.text.HAL_DMA_Start) for [Anonymous Symbol]
    stm32f0xx_hal_dma.o(.ARM.exidx.text.HAL_DMA_Start_IT) refers to stm32f0xx_hal_dma.o(.text.HAL_DMA_Start_IT) for [Anonymous Symbol]
    stm32f0xx_hal_dma.o(.ARM.exidx.text.HAL_DMA_Abort) refers to stm32f0xx_hal_dma.o(.text.HAL_DMA_Abort) for [Anonymous Symbol]
    stm32f0xx_hal_dma.o(.ARM.exidx.text.HAL_DMA_Abort_IT) refers to stm32f0xx_hal_dma.o(.text.HAL_DMA_Abort_IT) for [Anonymous Symbol]
    stm32f0xx_hal_dma.o(.text.HAL_DMA_PollForTransfer) refers to stm32f0xx_hal.o(.text.HAL_GetTick) for HAL_GetTick
    stm32f0xx_hal_dma.o(.ARM.exidx.text.HAL_DMA_PollForTransfer) refers to stm32f0xx_hal_dma.o(.text.HAL_DMA_PollForTransfer) for [Anonymous Symbol]
    stm32f0xx_hal_dma.o(.ARM.exidx.text.HAL_DMA_IRQHandler) refers to stm32f0xx_hal_dma.o(.text.HAL_DMA_IRQHandler) for [Anonymous Symbol]
    stm32f0xx_hal_dma.o(.ARM.exidx.text.HAL_DMA_RegisterCallback) refers to stm32f0xx_hal_dma.o(.text.HAL_DMA_RegisterCallback) for [Anonymous Symbol]
    stm32f0xx_hal_dma.o(.ARM.exidx.text.HAL_DMA_UnRegisterCallback) refers to stm32f0xx_hal_dma.o(.text.HAL_DMA_UnRegisterCallback) for [Anonymous Symbol]
    stm32f0xx_hal_dma.o(.ARM.exidx.text.HAL_DMA_GetState) refers to stm32f0xx_hal_dma.o(.text.HAL_DMA_GetState) for [Anonymous Symbol]
    stm32f0xx_hal_dma.o(.ARM.exidx.text.HAL_DMA_GetError) refers to stm32f0xx_hal_dma.o(.text.HAL_DMA_GetError) for [Anonymous Symbol]
    stm32f0xx_hal_cortex.o(.ARM.exidx.text.HAL_NVIC_SetPriority) refers to stm32f0xx_hal_cortex.o(.text.HAL_NVIC_SetPriority) for [Anonymous Symbol]
    stm32f0xx_hal_cortex.o(.ARM.exidx.text.HAL_NVIC_EnableIRQ) refers to stm32f0xx_hal_cortex.o(.text.HAL_NVIC_EnableIRQ) for [Anonymous Symbol]
    stm32f0xx_hal_cortex.o(.ARM.exidx.text.HAL_NVIC_DisableIRQ) refers to stm32f0xx_hal_cortex.o(.text.HAL_NVIC_DisableIRQ) for [Anonymous Symbol]
    stm32f0xx_hal_cortex.o(.ARM.exidx.text.HAL_NVIC_SystemReset) refers to stm32f0xx_hal_cortex.o(.text.HAL_NVIC_SystemReset) for [Anonymous Symbol]
    stm32f0xx_hal_cortex.o(.ARM.exidx.text.HAL_SYSTICK_Config) refers to stm32f0xx_hal_cortex.o(.text.HAL_SYSTICK_Config) for [Anonymous Symbol]
    stm32f0xx_hal_cortex.o(.ARM.exidx.text.HAL_NVIC_GetPriority) refers to stm32f0xx_hal_cortex.o(.text.HAL_NVIC_GetPriority) for [Anonymous Symbol]
    stm32f0xx_hal_cortex.o(.ARM.exidx.text.HAL_NVIC_SetPendingIRQ) refers to stm32f0xx_hal_cortex.o(.text.HAL_NVIC_SetPendingIRQ) for [Anonymous Symbol]
    stm32f0xx_hal_cortex.o(.ARM.exidx.text.HAL_NVIC_GetPendingIRQ) refers to stm32f0xx_hal_cortex.o(.text.HAL_NVIC_GetPendingIRQ) for [Anonymous Symbol]
    stm32f0xx_hal_cortex.o(.ARM.exidx.text.HAL_NVIC_ClearPendingIRQ) refers to stm32f0xx_hal_cortex.o(.text.HAL_NVIC_ClearPendingIRQ) for [Anonymous Symbol]
    stm32f0xx_hal_cortex.o(.ARM.exidx.text.HAL_SYSTICK_CLKSourceConfig) refers to stm32f0xx_hal_cortex.o(.text.HAL_SYSTICK_CLKSourceConfig) for [Anonymous Symbol]
    stm32f0xx_hal_cortex.o(.text.HAL_SYSTICK_IRQHandler) refers to stm32f0xx_hal_cortex.o(.text.HAL_SYSTICK_Callback) for HAL_SYSTICK_Callback
    stm32f0xx_hal_cortex.o(.ARM.exidx.text.HAL_SYSTICK_IRQHandler) refers to stm32f0xx_hal_cortex.o(.text.HAL_SYSTICK_IRQHandler) for [Anonymous Symbol]
    stm32f0xx_hal_cortex.o(.ARM.exidx.text.HAL_SYSTICK_Callback) refers to stm32f0xx_hal_cortex.o(.text.HAL_SYSTICK_Callback) for [Anonymous Symbol]
    stm32f0xx_hal_pwr.o(.ARM.exidx.text.HAL_PWR_DeInit) refers to stm32f0xx_hal_pwr.o(.text.HAL_PWR_DeInit) for [Anonymous Symbol]
    stm32f0xx_hal_pwr.o(.ARM.exidx.text.HAL_PWR_EnableBkUpAccess) refers to stm32f0xx_hal_pwr.o(.text.HAL_PWR_EnableBkUpAccess) for [Anonymous Symbol]
    stm32f0xx_hal_pwr.o(.ARM.exidx.text.HAL_PWR_DisableBkUpAccess) refers to stm32f0xx_hal_pwr.o(.text.HAL_PWR_DisableBkUpAccess) for [Anonymous Symbol]
    stm32f0xx_hal_pwr.o(.ARM.exidx.text.HAL_PWR_EnableWakeUpPin) refers to stm32f0xx_hal_pwr.o(.text.HAL_PWR_EnableWakeUpPin) for [Anonymous Symbol]
    stm32f0xx_hal_pwr.o(.ARM.exidx.text.HAL_PWR_DisableWakeUpPin) refers to stm32f0xx_hal_pwr.o(.text.HAL_PWR_DisableWakeUpPin) for [Anonymous Symbol]
    stm32f0xx_hal_pwr.o(.ARM.exidx.text.HAL_PWR_EnterSLEEPMode) refers to stm32f0xx_hal_pwr.o(.text.HAL_PWR_EnterSLEEPMode) for [Anonymous Symbol]
    stm32f0xx_hal_pwr.o(.ARM.exidx.text.HAL_PWR_EnterSTOPMode) refers to stm32f0xx_hal_pwr.o(.text.HAL_PWR_EnterSTOPMode) for [Anonymous Symbol]
    stm32f0xx_hal_pwr.o(.ARM.exidx.text.HAL_PWR_EnterSTANDBYMode) refers to stm32f0xx_hal_pwr.o(.text.HAL_PWR_EnterSTANDBYMode) for [Anonymous Symbol]
    stm32f0xx_hal_pwr.o(.ARM.exidx.text.HAL_PWR_EnableSleepOnExit) refers to stm32f0xx_hal_pwr.o(.text.HAL_PWR_EnableSleepOnExit) for [Anonymous Symbol]
    stm32f0xx_hal_pwr.o(.ARM.exidx.text.HAL_PWR_DisableSleepOnExit) refers to stm32f0xx_hal_pwr.o(.text.HAL_PWR_DisableSleepOnExit) for [Anonymous Symbol]
    stm32f0xx_hal_pwr.o(.ARM.exidx.text.HAL_PWR_EnableSEVOnPend) refers to stm32f0xx_hal_pwr.o(.text.HAL_PWR_EnableSEVOnPend) for [Anonymous Symbol]
    stm32f0xx_hal_pwr.o(.ARM.exidx.text.HAL_PWR_DisableSEVOnPend) refers to stm32f0xx_hal_pwr.o(.text.HAL_PWR_DisableSEVOnPend) for [Anonymous Symbol]
    stm32f0xx_hal_flash.o(.text.HAL_FLASH_Program) refers to stm32f0xx_hal.o(.text.HAL_GetTick) for HAL_GetTick
    stm32f0xx_hal_flash.o(.text.HAL_FLASH_Program) refers to llushr.o(.text) for __aeabi_llsr
    stm32f0xx_hal_flash.o(.text.HAL_FLASH_Program) refers to stm32f0xx_hal_flash.o(.bss.pFlash) for pFlash
    stm32f0xx_hal_flash.o(.ARM.exidx.text.HAL_FLASH_Program) refers to stm32f0xx_hal_flash.o(.text.HAL_FLASH_Program) for [Anonymous Symbol]
    stm32f0xx_hal_flash.o(.text.FLASH_WaitForLastOperation) refers to stm32f0xx_hal.o(.text.HAL_GetTick) for HAL_GetTick
    stm32f0xx_hal_flash.o(.text.FLASH_WaitForLastOperation) refers to stm32f0xx_hal_flash.o(.bss.pFlash) for pFlash
    stm32f0xx_hal_flash.o(.ARM.exidx.text.FLASH_WaitForLastOperation) refers to stm32f0xx_hal_flash.o(.text.FLASH_WaitForLastOperation) for [Anonymous Symbol]
    stm32f0xx_hal_flash.o(.text.HAL_FLASH_Program_IT) refers to stm32f0xx_hal_flash.o(.bss.pFlash) for pFlash
    stm32f0xx_hal_flash.o(.ARM.exidx.text.HAL_FLASH_Program_IT) refers to stm32f0xx_hal_flash.o(.text.HAL_FLASH_Program_IT) for [Anonymous Symbol]
    stm32f0xx_hal_flash.o(.text.HAL_FLASH_IRQHandler) refers to stm32f0xx_hal_flash.o(.text.HAL_FLASH_OperationErrorCallback) for HAL_FLASH_OperationErrorCallback
    stm32f0xx_hal_flash.o(.text.HAL_FLASH_IRQHandler) refers to stm32f0xx_hal_flash.o(.text.HAL_FLASH_EndOfOperationCallback) for HAL_FLASH_EndOfOperationCallback
    stm32f0xx_hal_flash.o(.text.HAL_FLASH_IRQHandler) refers to stm32f0xx_hal_flash_ex.o(.text.FLASH_PageErase) for FLASH_PageErase
    stm32f0xx_hal_flash.o(.text.HAL_FLASH_IRQHandler) refers to stm32f0xx_hal_flash.o(.bss.pFlash) for pFlash
    stm32f0xx_hal_flash.o(.ARM.exidx.text.HAL_FLASH_IRQHandler) refers to stm32f0xx_hal_flash.o(.text.HAL_FLASH_IRQHandler) for [Anonymous Symbol]
    stm32f0xx_hal_flash.o(.ARM.exidx.text.HAL_FLASH_OperationErrorCallback) refers to stm32f0xx_hal_flash.o(.text.HAL_FLASH_OperationErrorCallback) for [Anonymous Symbol]
    stm32f0xx_hal_flash.o(.ARM.exidx.text.HAL_FLASH_EndOfOperationCallback) refers to stm32f0xx_hal_flash.o(.text.HAL_FLASH_EndOfOperationCallback) for [Anonymous Symbol]
    stm32f0xx_hal_flash.o(.ARM.exidx.text.HAL_FLASH_Unlock) refers to stm32f0xx_hal_flash.o(.text.HAL_FLASH_Unlock) for [Anonymous Symbol]
    stm32f0xx_hal_flash.o(.ARM.exidx.text.HAL_FLASH_Lock) refers to stm32f0xx_hal_flash.o(.text.HAL_FLASH_Lock) for [Anonymous Symbol]
    stm32f0xx_hal_flash.o(.ARM.exidx.text.HAL_FLASH_OB_Unlock) refers to stm32f0xx_hal_flash.o(.text.HAL_FLASH_OB_Unlock) for [Anonymous Symbol]
    stm32f0xx_hal_flash.o(.ARM.exidx.text.HAL_FLASH_OB_Lock) refers to stm32f0xx_hal_flash.o(.text.HAL_FLASH_OB_Lock) for [Anonymous Symbol]
    stm32f0xx_hal_flash.o(.text.HAL_FLASH_OB_Launch) refers to stm32f0xx_hal.o(.text.HAL_GetTick) for HAL_GetTick
    stm32f0xx_hal_flash.o(.text.HAL_FLASH_OB_Launch) refers to stm32f0xx_hal_flash.o(.bss.pFlash) for pFlash
    stm32f0xx_hal_flash.o(.ARM.exidx.text.HAL_FLASH_OB_Launch) refers to stm32f0xx_hal_flash.o(.text.HAL_FLASH_OB_Launch) for [Anonymous Symbol]
    stm32f0xx_hal_flash.o(.text.HAL_FLASH_GetError) refers to stm32f0xx_hal_flash.o(.bss.pFlash) for pFlash
    stm32f0xx_hal_flash.o(.ARM.exidx.text.HAL_FLASH_GetError) refers to stm32f0xx_hal_flash.o(.text.HAL_FLASH_GetError) for [Anonymous Symbol]
    stm32f0xx_hal_flash_ex.o(.text.HAL_FLASHEx_Erase) refers to stm32f0xx_hal_flash.o(.text.FLASH_WaitForLastOperation) for FLASH_WaitForLastOperation
    stm32f0xx_hal_flash_ex.o(.text.HAL_FLASHEx_Erase) refers to stm32f0xx_hal_flash.o(.bss.pFlash) for pFlash
    stm32f0xx_hal_flash_ex.o(.ARM.exidx.text.HAL_FLASHEx_Erase) refers to stm32f0xx_hal_flash_ex.o(.text.HAL_FLASHEx_Erase) for [Anonymous Symbol]
    stm32f0xx_hal_flash_ex.o(.text.FLASH_PageErase) refers to stm32f0xx_hal_flash.o(.bss.pFlash) for pFlash
    stm32f0xx_hal_flash_ex.o(.ARM.exidx.text.FLASH_PageErase) refers to stm32f0xx_hal_flash_ex.o(.text.FLASH_PageErase) for [Anonymous Symbol]
    stm32f0xx_hal_flash_ex.o(.text.HAL_FLASHEx_Erase_IT) refers to stm32f0xx_hal_flash.o(.bss.pFlash) for pFlash
    stm32f0xx_hal_flash_ex.o(.ARM.exidx.text.HAL_FLASHEx_Erase_IT) refers to stm32f0xx_hal_flash_ex.o(.text.HAL_FLASHEx_Erase_IT) for [Anonymous Symbol]
    stm32f0xx_hal_flash_ex.o(.text.HAL_FLASHEx_OBErase) refers to stm32f0xx_hal_flash.o(.text.FLASH_WaitForLastOperation) for FLASH_WaitForLastOperation
    stm32f0xx_hal_flash_ex.o(.text.HAL_FLASHEx_OBErase) refers to stm32f0xx_hal_flash.o(.bss.pFlash) for pFlash
    stm32f0xx_hal_flash_ex.o(.ARM.exidx.text.HAL_FLASHEx_OBErase) refers to stm32f0xx_hal_flash_ex.o(.text.HAL_FLASHEx_OBErase) for [Anonymous Symbol]
    stm32f0xx_hal_flash_ex.o(.text.HAL_FLASHEx_OBProgram) refers to stm32f0xx_hal_flash.o(.text.FLASH_WaitForLastOperation) for FLASH_WaitForLastOperation
    stm32f0xx_hal_flash_ex.o(.text.HAL_FLASHEx_OBProgram) refers to stm32f0xx_hal_flash_ex.o(.text.HAL_FLASHEx_OBErase) for HAL_FLASHEx_OBErase
    stm32f0xx_hal_flash_ex.o(.text.HAL_FLASHEx_OBProgram) refers to stm32f0xx_hal_flash.o(.bss.pFlash) for pFlash
    stm32f0xx_hal_flash_ex.o(.ARM.exidx.text.HAL_FLASHEx_OBProgram) refers to stm32f0xx_hal_flash_ex.o(.text.HAL_FLASHEx_OBProgram) for [Anonymous Symbol]
    stm32f0xx_hal_flash_ex.o(.ARM.exidx.text.HAL_FLASHEx_OBGetConfig) refers to stm32f0xx_hal_flash_ex.o(.text.HAL_FLASHEx_OBGetConfig) for [Anonymous Symbol]
    stm32f0xx_hal_flash_ex.o(.ARM.exidx.text.HAL_FLASHEx_OBGetUserData) refers to stm32f0xx_hal_flash_ex.o(.text.HAL_FLASHEx_OBGetUserData) for [Anonymous Symbol]
    stm32f0xx_hal_exti.o(.ARM.exidx.text.HAL_EXTI_SetConfigLine) refers to stm32f0xx_hal_exti.o(.text.HAL_EXTI_SetConfigLine) for [Anonymous Symbol]
    stm32f0xx_hal_exti.o(.ARM.exidx.text.HAL_EXTI_GetConfigLine) refers to stm32f0xx_hal_exti.o(.text.HAL_EXTI_GetConfigLine) for [Anonymous Symbol]
    stm32f0xx_hal_exti.o(.ARM.exidx.text.HAL_EXTI_ClearConfigLine) refers to stm32f0xx_hal_exti.o(.text.HAL_EXTI_ClearConfigLine) for [Anonymous Symbol]
    stm32f0xx_hal_exti.o(.ARM.exidx.text.HAL_EXTI_RegisterCallback) refers to stm32f0xx_hal_exti.o(.text.HAL_EXTI_RegisterCallback) for [Anonymous Symbol]
    stm32f0xx_hal_exti.o(.ARM.exidx.text.HAL_EXTI_GetHandle) refers to stm32f0xx_hal_exti.o(.text.HAL_EXTI_GetHandle) for [Anonymous Symbol]
    stm32f0xx_hal_exti.o(.ARM.exidx.text.HAL_EXTI_IRQHandler) refers to stm32f0xx_hal_exti.o(.text.HAL_EXTI_IRQHandler) for [Anonymous Symbol]
    stm32f0xx_hal_exti.o(.ARM.exidx.text.HAL_EXTI_GetPending) refers to stm32f0xx_hal_exti.o(.text.HAL_EXTI_GetPending) for [Anonymous Symbol]
    stm32f0xx_hal_exti.o(.ARM.exidx.text.HAL_EXTI_ClearPending) refers to stm32f0xx_hal_exti.o(.text.HAL_EXTI_ClearPending) for [Anonymous Symbol]
    stm32f0xx_hal_exti.o(.ARM.exidx.text.HAL_EXTI_GenerateSWI) refers to stm32f0xx_hal_exti.o(.text.HAL_EXTI_GenerateSWI) for [Anonymous Symbol]
    stm32f0xx_hal_rtc.o(.text.HAL_RTC_Init) refers to stm32f0xx_hal_msp.o(.text.HAL_RTC_MspInit) for HAL_RTC_MspInit
    stm32f0xx_hal_rtc.o(.text.HAL_RTC_Init) refers to stm32f0xx_hal.o(.text.HAL_GetTick) for HAL_GetTick
    stm32f0xx_hal_rtc.o(.ARM.exidx.text.HAL_RTC_Init) refers to stm32f0xx_hal_rtc.o(.text.HAL_RTC_Init) for [Anonymous Symbol]
    stm32f0xx_hal_rtc.o(.ARM.exidx.text.HAL_RTC_MspInit) refers to stm32f0xx_hal_rtc.o(.text.HAL_RTC_MspInit) for [Anonymous Symbol]
    stm32f0xx_hal_rtc.o(.text.RTC_EnterInitMode) refers to stm32f0xx_hal.o(.text.HAL_GetTick) for HAL_GetTick
    stm32f0xx_hal_rtc.o(.ARM.exidx.text.RTC_EnterInitMode) refers to stm32f0xx_hal_rtc.o(.text.RTC_EnterInitMode) for [Anonymous Symbol]
    stm32f0xx_hal_rtc.o(.text.RTC_ExitInitMode) refers to stm32f0xx_hal.o(.text.HAL_GetTick) for HAL_GetTick
    stm32f0xx_hal_rtc.o(.ARM.exidx.text.RTC_ExitInitMode) refers to stm32f0xx_hal_rtc.o(.text.RTC_ExitInitMode) for [Anonymous Symbol]
    stm32f0xx_hal_rtc.o(.text.HAL_RTC_DeInit) refers to stm32f0xx_hal.o(.text.HAL_GetTick) for HAL_GetTick
    stm32f0xx_hal_rtc.o(.text.HAL_RTC_DeInit) refers to stm32f0xx_hal_msp.o(.text.HAL_RTC_MspDeInit) for HAL_RTC_MspDeInit
    stm32f0xx_hal_rtc.o(.ARM.exidx.text.HAL_RTC_DeInit) refers to stm32f0xx_hal_rtc.o(.text.HAL_RTC_DeInit) for [Anonymous Symbol]
    stm32f0xx_hal_rtc.o(.ARM.exidx.text.HAL_RTC_MspDeInit) refers to stm32f0xx_hal_rtc.o(.text.HAL_RTC_MspDeInit) for [Anonymous Symbol]
    stm32f0xx_hal_rtc.o(.text.HAL_RTC_SetTime) refers to stm32f0xx_hal.o(.text.HAL_GetTick) for HAL_GetTick
    stm32f0xx_hal_rtc.o(.ARM.exidx.text.HAL_RTC_SetTime) refers to stm32f0xx_hal_rtc.o(.text.HAL_RTC_SetTime) for [Anonymous Symbol]
    stm32f0xx_hal_rtc.o(.ARM.exidx.text.RTC_ByteToBcd2) refers to stm32f0xx_hal_rtc.o(.text.RTC_ByteToBcd2) for [Anonymous Symbol]
    stm32f0xx_hal_rtc.o(.ARM.exidx.text.HAL_RTC_GetTime) refers to stm32f0xx_hal_rtc.o(.text.HAL_RTC_GetTime) for [Anonymous Symbol]
    stm32f0xx_hal_rtc.o(.ARM.exidx.text.RTC_Bcd2ToByte) refers to stm32f0xx_hal_rtc.o(.text.RTC_Bcd2ToByte) for [Anonymous Symbol]
    stm32f0xx_hal_rtc.o(.text.HAL_RTC_SetDate) refers to stm32f0xx_hal.o(.text.HAL_GetTick) for HAL_GetTick
    stm32f0xx_hal_rtc.o(.ARM.exidx.text.HAL_RTC_SetDate) refers to stm32f0xx_hal_rtc.o(.text.HAL_RTC_SetDate) for [Anonymous Symbol]
    stm32f0xx_hal_rtc.o(.ARM.exidx.text.HAL_RTC_GetDate) refers to stm32f0xx_hal_rtc.o(.text.HAL_RTC_GetDate) for [Anonymous Symbol]
    stm32f0xx_hal_rtc.o(.text.HAL_RTC_SetAlarm) refers to stm32f0xx_hal.o(.text.HAL_GetTick) for HAL_GetTick
    stm32f0xx_hal_rtc.o(.ARM.exidx.text.HAL_RTC_SetAlarm) refers to stm32f0xx_hal_rtc.o(.text.HAL_RTC_SetAlarm) for [Anonymous Symbol]
    stm32f0xx_hal_rtc.o(.text.HAL_RTC_SetAlarm_IT) refers to aeabi_sdivfast.o(.text_divfast) for __aeabi_uidiv
    stm32f0xx_hal_rtc.o(.text.HAL_RTC_SetAlarm_IT) refers to system_stm32f0xx.o(.data.SystemCoreClock) for SystemCoreClock
    stm32f0xx_hal_rtc.o(.ARM.exidx.text.HAL_RTC_SetAlarm_IT) refers to stm32f0xx_hal_rtc.o(.text.HAL_RTC_SetAlarm_IT) for [Anonymous Symbol]
    stm32f0xx_hal_rtc.o(.text.HAL_RTC_DeactivateAlarm) refers to stm32f0xx_hal.o(.text.HAL_GetTick) for HAL_GetTick
    stm32f0xx_hal_rtc.o(.ARM.exidx.text.HAL_RTC_DeactivateAlarm) refers to stm32f0xx_hal_rtc.o(.text.HAL_RTC_DeactivateAlarm) for [Anonymous Symbol]
    stm32f0xx_hal_rtc.o(.ARM.exidx.text.HAL_RTC_GetAlarm) refers to stm32f0xx_hal_rtc.o(.text.HAL_RTC_GetAlarm) for [Anonymous Symbol]
    stm32f0xx_hal_rtc.o(.text.HAL_RTC_AlarmIRQHandler) refers to stm32f0xx_hal_rtc.o(.text.HAL_RTC_AlarmAEventCallback) for HAL_RTC_AlarmAEventCallback
    stm32f0xx_hal_rtc.o(.ARM.exidx.text.HAL_RTC_AlarmIRQHandler) refers to stm32f0xx_hal_rtc.o(.text.HAL_RTC_AlarmIRQHandler) for [Anonymous Symbol]
    stm32f0xx_hal_rtc.o(.ARM.exidx.text.HAL_RTC_AlarmAEventCallback) refers to stm32f0xx_hal_rtc.o(.text.HAL_RTC_AlarmAEventCallback) for [Anonymous Symbol]
    stm32f0xx_hal_rtc.o(.text.HAL_RTC_PollForAlarmAEvent) refers to stm32f0xx_hal.o(.text.HAL_GetTick) for HAL_GetTick
    stm32f0xx_hal_rtc.o(.ARM.exidx.text.HAL_RTC_PollForAlarmAEvent) refers to stm32f0xx_hal_rtc.o(.text.HAL_RTC_PollForAlarmAEvent) for [Anonymous Symbol]
    stm32f0xx_hal_rtc.o(.text.HAL_RTC_WaitForSynchro) refers to stm32f0xx_hal.o(.text.HAL_GetTick) for HAL_GetTick
    stm32f0xx_hal_rtc.o(.ARM.exidx.text.HAL_RTC_WaitForSynchro) refers to stm32f0xx_hal_rtc.o(.text.HAL_RTC_WaitForSynchro) for [Anonymous Symbol]
    stm32f0xx_hal_rtc.o(.ARM.exidx.text.HAL_RTC_DST_Add1Hour) refers to stm32f0xx_hal_rtc.o(.text.HAL_RTC_DST_Add1Hour) for [Anonymous Symbol]
    stm32f0xx_hal_rtc.o(.ARM.exidx.text.HAL_RTC_DST_Sub1Hour) refers to stm32f0xx_hal_rtc.o(.text.HAL_RTC_DST_Sub1Hour) for [Anonymous Symbol]
    stm32f0xx_hal_rtc.o(.ARM.exidx.text.HAL_RTC_DST_SetStoreOperation) refers to stm32f0xx_hal_rtc.o(.text.HAL_RTC_DST_SetStoreOperation) for [Anonymous Symbol]
    stm32f0xx_hal_rtc.o(.ARM.exidx.text.HAL_RTC_DST_ClearStoreOperation) refers to stm32f0xx_hal_rtc.o(.text.HAL_RTC_DST_ClearStoreOperation) for [Anonymous Symbol]
    stm32f0xx_hal_rtc.o(.ARM.exidx.text.HAL_RTC_DST_ReadStoreOperation) refers to stm32f0xx_hal_rtc.o(.text.HAL_RTC_DST_ReadStoreOperation) for [Anonymous Symbol]
    stm32f0xx_hal_rtc.o(.ARM.exidx.text.HAL_RTC_GetState) refers to stm32f0xx_hal_rtc.o(.text.HAL_RTC_GetState) for [Anonymous Symbol]
    stm32f0xx_hal_rtc_ex.o(.ARM.exidx.text.HAL_RTCEx_SetTimeStamp) refers to stm32f0xx_hal_rtc_ex.o(.text.HAL_RTCEx_SetTimeStamp) for [Anonymous Symbol]
    stm32f0xx_hal_rtc_ex.o(.ARM.exidx.text.HAL_RTCEx_SetTimeStamp_IT) refers to stm32f0xx_hal_rtc_ex.o(.text.HAL_RTCEx_SetTimeStamp_IT) for [Anonymous Symbol]
    stm32f0xx_hal_rtc_ex.o(.ARM.exidx.text.HAL_RTCEx_DeactivateTimeStamp) refers to stm32f0xx_hal_rtc_ex.o(.text.HAL_RTCEx_DeactivateTimeStamp) for [Anonymous Symbol]
    stm32f0xx_hal_rtc_ex.o(.text.HAL_RTCEx_GetTimeStamp) refers to stm32f0xx_hal_rtc.o(.text.RTC_Bcd2ToByte) for RTC_Bcd2ToByte
    stm32f0xx_hal_rtc_ex.o(.ARM.exidx.text.HAL_RTCEx_GetTimeStamp) refers to stm32f0xx_hal_rtc_ex.o(.text.HAL_RTCEx_GetTimeStamp) for [Anonymous Symbol]
    stm32f0xx_hal_rtc_ex.o(.ARM.exidx.text.HAL_RTCEx_SetTamper) refers to stm32f0xx_hal_rtc_ex.o(.text.HAL_RTCEx_SetTamper) for [Anonymous Symbol]
    stm32f0xx_hal_rtc_ex.o(.ARM.exidx.text.HAL_RTCEx_SetTamper_IT) refers to stm32f0xx_hal_rtc_ex.o(.text.HAL_RTCEx_SetTamper_IT) for [Anonymous Symbol]
    stm32f0xx_hal_rtc_ex.o(.ARM.exidx.text.HAL_RTCEx_DeactivateTamper) refers to stm32f0xx_hal_rtc_ex.o(.text.HAL_RTCEx_DeactivateTamper) for [Anonymous Symbol]
    stm32f0xx_hal_rtc_ex.o(.text.HAL_RTCEx_TamperTimeStampIRQHandler) refers to stm32f0xx_hal_rtc_ex.o(.text.HAL_RTCEx_TimeStampEventCallback) for HAL_RTCEx_TimeStampEventCallback
    stm32f0xx_hal_rtc_ex.o(.text.HAL_RTCEx_TamperTimeStampIRQHandler) refers to stm32f0xx_hal_rtc_ex.o(.text.HAL_RTCEx_Tamper1EventCallback) for HAL_RTCEx_Tamper1EventCallback
    stm32f0xx_hal_rtc_ex.o(.text.HAL_RTCEx_TamperTimeStampIRQHandler) refers to stm32f0xx_hal_rtc_ex.o(.text.HAL_RTCEx_Tamper2EventCallback) for HAL_RTCEx_Tamper2EventCallback
    stm32f0xx_hal_rtc_ex.o(.ARM.exidx.text.HAL_RTCEx_TamperTimeStampIRQHandler) refers to stm32f0xx_hal_rtc_ex.o(.text.HAL_RTCEx_TamperTimeStampIRQHandler) for [Anonymous Symbol]
    stm32f0xx_hal_rtc_ex.o(.ARM.exidx.text.HAL_RTCEx_TimeStampEventCallback) refers to stm32f0xx_hal_rtc_ex.o(.text.HAL_RTCEx_TimeStampEventCallback) for [Anonymous Symbol]
    stm32f0xx_hal_rtc_ex.o(.ARM.exidx.text.HAL_RTCEx_Tamper1EventCallback) refers to stm32f0xx_hal_rtc_ex.o(.text.HAL_RTCEx_Tamper1EventCallback) for [Anonymous Symbol]
    stm32f0xx_hal_rtc_ex.o(.ARM.exidx.text.HAL_RTCEx_Tamper2EventCallback) refers to stm32f0xx_hal_rtc_ex.o(.text.HAL_RTCEx_Tamper2EventCallback) for [Anonymous Symbol]
    stm32f0xx_hal_rtc_ex.o(.text.HAL_RTCEx_PollForTimeStampEvent) refers to stm32f0xx_hal.o(.text.HAL_GetTick) for HAL_GetTick
    stm32f0xx_hal_rtc_ex.o(.ARM.exidx.text.HAL_RTCEx_PollForTimeStampEvent) refers to stm32f0xx_hal_rtc_ex.o(.text.HAL_RTCEx_PollForTimeStampEvent) for [Anonymous Symbol]
    stm32f0xx_hal_rtc_ex.o(.text.HAL_RTCEx_PollForTamper1Event) refers to stm32f0xx_hal.o(.text.HAL_GetTick) for HAL_GetTick
    stm32f0xx_hal_rtc_ex.o(.ARM.exidx.text.HAL_RTCEx_PollForTamper1Event) refers to stm32f0xx_hal_rtc_ex.o(.text.HAL_RTCEx_PollForTamper1Event) for [Anonymous Symbol]
    stm32f0xx_hal_rtc_ex.o(.text.HAL_RTCEx_PollForTamper2Event) refers to stm32f0xx_hal.o(.text.HAL_GetTick) for HAL_GetTick
    stm32f0xx_hal_rtc_ex.o(.ARM.exidx.text.HAL_RTCEx_PollForTamper2Event) refers to stm32f0xx_hal_rtc_ex.o(.text.HAL_RTCEx_PollForTamper2Event) for [Anonymous Symbol]
    stm32f0xx_hal_rtc_ex.o(.text.HAL_RTCEx_SetWakeUpTimer) refers to stm32f0xx_hal.o(.text.HAL_GetTick) for HAL_GetTick
    stm32f0xx_hal_rtc_ex.o(.ARM.exidx.text.HAL_RTCEx_SetWakeUpTimer) refers to stm32f0xx_hal_rtc_ex.o(.text.HAL_RTCEx_SetWakeUpTimer) for [Anonymous Symbol]
    stm32f0xx_hal_rtc_ex.o(.text.HAL_RTCEx_SetWakeUpTimer_IT) refers to aeabi_sdivfast.o(.text_divfast) for __aeabi_uidiv
    stm32f0xx_hal_rtc_ex.o(.text.HAL_RTCEx_SetWakeUpTimer_IT) refers to system_stm32f0xx.o(.data.SystemCoreClock) for SystemCoreClock
    stm32f0xx_hal_rtc_ex.o(.ARM.exidx.text.HAL_RTCEx_SetWakeUpTimer_IT) refers to stm32f0xx_hal_rtc_ex.o(.text.HAL_RTCEx_SetWakeUpTimer_IT) for [Anonymous Symbol]
    stm32f0xx_hal_rtc_ex.o(.text.HAL_RTCEx_DeactivateWakeUpTimer) refers to stm32f0xx_hal.o(.text.HAL_GetTick) for HAL_GetTick
    stm32f0xx_hal_rtc_ex.o(.ARM.exidx.text.HAL_RTCEx_DeactivateWakeUpTimer) refers to stm32f0xx_hal_rtc_ex.o(.text.HAL_RTCEx_DeactivateWakeUpTimer) for [Anonymous Symbol]
    stm32f0xx_hal_rtc_ex.o(.ARM.exidx.text.HAL_RTCEx_GetWakeUpTimer) refers to stm32f0xx_hal_rtc_ex.o(.text.HAL_RTCEx_GetWakeUpTimer) for [Anonymous Symbol]
    stm32f0xx_hal_rtc_ex.o(.text.HAL_RTCEx_WakeUpTimerIRQHandler) refers to stm32f0xx_hal_rtc_ex.o(.text.HAL_RTCEx_WakeUpTimerEventCallback) for HAL_RTCEx_WakeUpTimerEventCallback
    stm32f0xx_hal_rtc_ex.o(.ARM.exidx.text.HAL_RTCEx_WakeUpTimerIRQHandler) refers to stm32f0xx_hal_rtc_ex.o(.text.HAL_RTCEx_WakeUpTimerIRQHandler) for [Anonymous Symbol]
    stm32f0xx_hal_rtc_ex.o(.ARM.exidx.text.HAL_RTCEx_WakeUpTimerEventCallback) refers to stm32f0xx_hal_rtc_ex.o(.text.HAL_RTCEx_WakeUpTimerEventCallback) for [Anonymous Symbol]
    stm32f0xx_hal_rtc_ex.o(.text.HAL_RTCEx_PollForWakeUpTimerEvent) refers to stm32f0xx_hal.o(.text.HAL_GetTick) for HAL_GetTick
    stm32f0xx_hal_rtc_ex.o(.ARM.exidx.text.HAL_RTCEx_PollForWakeUpTimerEvent) refers to stm32f0xx_hal_rtc_ex.o(.text.HAL_RTCEx_PollForWakeUpTimerEvent) for [Anonymous Symbol]
    stm32f0xx_hal_rtc_ex.o(.text.HAL_RTCEx_SetSmoothCalib) refers to stm32f0xx_hal.o(.text.HAL_GetTick) for HAL_GetTick
    stm32f0xx_hal_rtc_ex.o(.ARM.exidx.text.HAL_RTCEx_SetSmoothCalib) refers to stm32f0xx_hal_rtc_ex.o(.text.HAL_RTCEx_SetSmoothCalib) for [Anonymous Symbol]
    stm32f0xx_hal_rtc_ex.o(.text.HAL_RTCEx_SetSynchroShift) refers to stm32f0xx_hal.o(.text.HAL_GetTick) for HAL_GetTick
    stm32f0xx_hal_rtc_ex.o(.text.HAL_RTCEx_SetSynchroShift) refers to stm32f0xx_hal_rtc.o(.text.HAL_RTC_WaitForSynchro) for HAL_RTC_WaitForSynchro
    stm32f0xx_hal_rtc_ex.o(.ARM.exidx.text.HAL_RTCEx_SetSynchroShift) refers to stm32f0xx_hal_rtc_ex.o(.text.HAL_RTCEx_SetSynchroShift) for [Anonymous Symbol]
    stm32f0xx_hal_rtc_ex.o(.ARM.exidx.text.HAL_RTCEx_SetCalibrationOutPut) refers to stm32f0xx_hal_rtc_ex.o(.text.HAL_RTCEx_SetCalibrationOutPut) for [Anonymous Symbol]
    stm32f0xx_hal_rtc_ex.o(.ARM.exidx.text.HAL_RTCEx_DeactivateCalibrationOutPut) refers to stm32f0xx_hal_rtc_ex.o(.text.HAL_RTCEx_DeactivateCalibrationOutPut) for [Anonymous Symbol]
    stm32f0xx_hal_rtc_ex.o(.text.HAL_RTCEx_SetRefClock) refers to stm32f0xx_hal_rtc.o(.text.RTC_EnterInitMode) for RTC_EnterInitMode
    stm32f0xx_hal_rtc_ex.o(.text.HAL_RTCEx_SetRefClock) refers to stm32f0xx_hal_rtc.o(.text.RTC_ExitInitMode) for RTC_ExitInitMode
    stm32f0xx_hal_rtc_ex.o(.ARM.exidx.text.HAL_RTCEx_SetRefClock) refers to stm32f0xx_hal_rtc_ex.o(.text.HAL_RTCEx_SetRefClock) for [Anonymous Symbol]
    stm32f0xx_hal_rtc_ex.o(.text.HAL_RTCEx_DeactivateRefClock) refers to stm32f0xx_hal_rtc.o(.text.RTC_EnterInitMode) for RTC_EnterInitMode
    stm32f0xx_hal_rtc_ex.o(.text.HAL_RTCEx_DeactivateRefClock) refers to stm32f0xx_hal_rtc.o(.text.RTC_ExitInitMode) for RTC_ExitInitMode
    stm32f0xx_hal_rtc_ex.o(.ARM.exidx.text.HAL_RTCEx_DeactivateRefClock) refers to stm32f0xx_hal_rtc_ex.o(.text.HAL_RTCEx_DeactivateRefClock) for [Anonymous Symbol]
    stm32f0xx_hal_rtc_ex.o(.ARM.exidx.text.HAL_RTCEx_EnableBypassShadow) refers to stm32f0xx_hal_rtc_ex.o(.text.HAL_RTCEx_EnableBypassShadow) for [Anonymous Symbol]
    stm32f0xx_hal_rtc_ex.o(.ARM.exidx.text.HAL_RTCEx_DisableBypassShadow) refers to stm32f0xx_hal_rtc_ex.o(.text.HAL_RTCEx_DisableBypassShadow) for [Anonymous Symbol]
    system_stm32f0xx.o(.ARM.exidx.text.SystemInit) refers to system_stm32f0xx.o(.text.SystemInit) for [Anonymous Symbol]
    system_stm32f0xx.o(.text.SystemCoreClockUpdate) refers to aeabi_sdivfast.o(.text_divfast) for __aeabi_uidiv
    system_stm32f0xx.o(.text.SystemCoreClockUpdate) refers to system_stm32f0xx.o(.data.SystemCoreClock) for SystemCoreClock
    system_stm32f0xx.o(.text.SystemCoreClockUpdate) refers to system_stm32f0xx.o(.rodata.AHBPrescTable) for AHBPrescTable
    system_stm32f0xx.o(.ARM.exidx.text.SystemCoreClockUpdate) refers to system_stm32f0xx.o(.text.SystemCoreClockUpdate) for [Anonymous Symbol]
    __2sprintf.o(.text) refers to _printf_char_common.o(.text) for _printf_char_common
    __2sprintf.o(.text) refers to _sputc.o(.text) for _sputc
    noretval__2sprintf.o(.text) refers to _printf_char_common.o(.text) for _printf_char_common
    noretval__2sprintf.o(.text) refers to _sputc.o(.text) for _sputc
    __printf.o(.text) refers to _printf_percent.o(.ARM.Collect$$_printf_percent$$00000000) for _printf_percent
    _printf_str.o(.text) refers (Special) to _printf_char.o(.text) for _printf_cs_common
    _printf_str.o(.text) refers (Weak) to _printf_pad.o(.text) for _printf_pre_padding
    _printf_str.o(.text) refers (Weak) to _printf_pad.o(.text) for _printf_post_padding
    _printf_hex_ll.o(.text) refers to _printf_intcommon.o(.text) for _printf_int_common
    _printf_hex_ll.o(.text) refers to _printf_hex_ll.o(.constdata) for .constdata
    _printf_hex_int.o(.text) refers to _printf_intcommon.o(.text) for _printf_int_common
    _printf_hex_int.o(.text) refers to _printf_hex_int.o(.constdata) for .constdata
    _printf_hex_int_ll.o(.text) refers to _printf_intcommon.o(.text) for _printf_int_common
    _printf_hex_int_ll.o(.text) refers to _printf_hex_int_ll.o(.constdata) for .constdata
    _printf_hex_ptr.o(.text) refers to _printf_intcommon.o(.text) for _printf_int_common
    _printf_hex_ptr.o(.text) refers to _printf_hex_ptr.o(.constdata) for .constdata
    _printf_hex_int_ptr.o(.text) refers to _printf_intcommon.o(.text) for _printf_int_common
    _printf_hex_int_ptr.o(.text) refers to _printf_hex_int_ptr.o(.constdata) for .constdata
    _printf_hex_ll_ptr.o(.text) refers to _printf_intcommon.o(.text) for _printf_int_common
    _printf_hex_ll_ptr.o(.text) refers to _printf_hex_ll_ptr.o(.constdata) for .constdata
    _printf_hex_int_ll_ptr.o(.text) refers to _printf_intcommon.o(.text) for _printf_int_common
    _printf_hex_int_ll_ptr.o(.text) refers to _printf_hex_int_ll_ptr.o(.constdata) for .constdata
    __printf_flags.o(.text) refers to _printf_percent.o(.ARM.Collect$$_printf_percent$$00000000) for _printf_percent
    __printf_flags.o(.text) refers to __printf_flags.o(.constdata) for .constdata
    __printf_ss.o(.text) refers to _printf_percent.o(.ARM.Collect$$_printf_percent$$00000000) for _printf_percent
    __printf_flags_ss.o(.text) refers to _printf_percent.o(.ARM.Collect$$_printf_percent$$00000000) for _printf_percent
    __printf_flags_ss.o(.text) refers to __printf_flags_ss.o(.constdata) for .constdata
    __printf_wp.o(.text) refers to __printf_wp.o(i._is_digit) for _is_digit
    __printf_wp.o(.text) refers to _printf_percent.o(.ARM.Collect$$_printf_percent$$00000000) for _printf_percent
    __printf_flags_wp.o(.text) refers to __printf_wp.o(i._is_digit) for _is_digit
    __printf_flags_wp.o(.text) refers to _printf_percent.o(.ARM.Collect$$_printf_percent$$00000000) for _printf_percent
    __printf_flags_wp.o(.text) refers to __printf_flags_wp.o(.constdata) for .constdata
    __printf_ss_wp.o(.text) refers to __printf_wp.o(i._is_digit) for _is_digit
    __printf_ss_wp.o(.text) refers to _printf_percent.o(.ARM.Collect$$_printf_percent$$00000000) for _printf_percent
    __printf_flags_ss_wp.o(.text) refers to __printf_wp.o(i._is_digit) for _is_digit
    __printf_flags_ss_wp.o(.text) refers to _printf_percent.o(.ARM.Collect$$_printf_percent$$00000000) for _printf_percent
    __printf_flags_ss_wp.o(.text) refers to __printf_flags_ss_wp.o(.constdata) for .constdata
    _printf_c.o(.ARM.Collect$$_printf_percent$$00000013) refers (Weak) to _printf_char.o(.text) for _printf_char
    _printf_s.o(.ARM.Collect$$_printf_percent$$00000014) refers (Weak) to _printf_char.o(.text) for _printf_string
    _printf_x.o(.ARM.Collect$$_printf_percent$$0000000C) refers (Weak) to _printf_hex_int.o(.text) for _printf_int_hex
    _printf_f.o(.ARM.Collect$$_printf_percent$$00000003) refers (Weak) to printf1.o(x$fpl$printf1) for _printf_fp_dec
    _printf_percent.o(.ARM.Collect$$_printf_percent$$00000000) refers (Special) to _printf_percent_end.o(.ARM.Collect$$_printf_percent$$00000017) for _printf_percent_end
    __main.o(!!!main) refers to __rtentry.o(.ARM.Collect$$rtentry$$00000000) for __rt_entry
    d2f.o(.text) refers (Special) to usenofp.o(x$fpl$usenofp) for __I$use$fp
    daddsub.o(.text) refers (Special) to usenofp.o(x$fpl$usenofp) for __I$use$fp
    ddiv.o(.text) refers (Special) to usenofp.o(x$fpl$usenofp) for __I$use$fp
    ddiv.o(.text) refers to ddiv.o(.constdata) for .constdata
    ddiv.o(.constdata) refers (Special) to usenofp.o(x$fpl$usenofp) for __I$use$fp
    dfixi.o(.text) refers (Special) to usenofp.o(x$fpl$usenofp) for __I$use$fp
    dflti.o(.text) refers (Special) to usenofp.o(x$fpl$usenofp) for __I$use$fp
    dmul.o(.text) refers (Special) to usenofp.o(x$fpl$usenofp) for __I$use$fp
    f2d.o(.text) refers (Special) to usenofp.o(x$fpl$usenofp) for __I$use$fp
    faddsub.o(x$fpl$fadd) refers (Special) to usenofp.o(x$fpl$usenofp) for __I$use$fp
    faddsub.o(x$fpl$fadd) refers to faddsub.o(x$fpl$fsub) for _fsub1
    faddsub.o(x$fpl$frsb) refers (Special) to usenofp.o(x$fpl$usenofp) for __I$use$fp
    faddsub.o(x$fpl$frsb) refers to faddsub.o(x$fpl$fsub) for _fsub1
    faddsub.o(x$fpl$frsb) refers to faddsub.o(x$fpl$fadd) for _fadd1
    faddsub.o(x$fpl$fsub) refers (Special) to usenofp.o(x$fpl$usenofp) for __I$use$fp
    faddsub.o(x$fpl$fsub) refers to faddsub.o(x$fpl$fadd) for _fadd1
    fflti.o(.text) refers (Special) to usenofp.o(x$fpl$usenofp) for __I$use$fp
    fmul.o(x$fpl$fmul) refers (Special) to usenofp.o(x$fpl$usenofp) for __I$use$fp
    printf1.o(x$fpl$printf1) refers to _printf_fp_dec.o(.text) for _printf_fp_dec_real
    pow.o(i.__softfp_pow) refers (Special) to usenofp.o(x$fpl$usenofp) for __I$use$fp
    pow.o(i.__softfp_pow) refers to pow.o(i.pow) for pow
    pow.o(i.pow) refers (Special) to usenofp.o(x$fpl$usenofp) for __I$use$fp
    pow.o(i.pow) refers to dunder.o(i.__mathlib_dbl_infnan2) for __mathlib_dbl_infnan2
    pow.o(i.pow) refers to _rserrno.o(.text) for __set_errno
    pow.o(i.pow) refers to dunder.o(i.__mathlib_dbl_divzero) for __mathlib_dbl_divzero
    pow.o(i.pow) refers to ddiv.o(.text) for __aeabi_ddiv
    pow.o(i.pow) refers to sqrt.o(i.sqrt) for sqrt
    pow.o(i.pow) refers to dflti.o(.text) for __aeabi_i2d
    pow.o(i.pow) refers to dunder.o(i.__mathlib_dbl_invalid) for __mathlib_dbl_invalid
    pow.o(i.pow) refers to dunder.o(i.__mathlib_dbl_overflow) for __mathlib_dbl_overflow
    pow.o(i.pow) refers to dmul.o(.text) for __aeabi_dmul
    pow.o(i.pow) refers to dunder.o(i.__mathlib_dbl_underflow) for __mathlib_dbl_underflow
    pow.o(i.pow) refers to daddsub.o(.text) for __aeabi_dsub
    pow.o(i.pow) refers to dscalbn.o(.text) for __ARM_scalbn
    pow.o(i.pow) refers to qnan.o(.constdata) for __mathlib_zero
    pow.o(i.pow) refers to poly.o(i.__kernel_poly) for __kernel_poly
    pow.o(i.pow) refers to drlef.o(x$fpl$drleqf) for __aeabi_cdrcmple
    pow.o(i.pow) refers to pow.o(.constdata) for .constdata
    pow.o(i.pow) refers to fpclassify.o(i.__ARM_fpclassify) for __ARM_fpclassify
    pow.o(.constdata) refers (Special) to usenofp.o(x$fpl$usenofp) for __I$use$fp
    __rtentry.o(.ARM.Collect$$rtentry$$00000000) refers (Special) to __rtentry2.o(.ARM.Collect$$rtentry$$0000000A) for __rt_entry_li
    __rtentry.o(.ARM.Collect$$rtentry$$00000000) refers (Special) to __rtentry2.o(.ARM.Collect$$rtentry$$0000000D) for __rt_entry_main
    __rtentry.o(.ARM.Collect$$rtentry$$00000000) refers (Special) to __rtentry2.o(.ARM.Collect$$rtentry$$0000000C) for __rt_entry_postli_1
    __rtentry.o(.ARM.Collect$$rtentry$$00000000) refers (Special) to __rtentry2.o(.ARM.Collect$$rtentry$$00000009) for __rt_entry_postsh_1
    __rtentry.o(.ARM.Collect$$rtentry$$00000000) refers (Special) to __rtentry2.o(.ARM.Collect$$rtentry$$00000002) for __rt_entry_presh_1
    __rtentry.o(.ARM.Collect$$rtentry$$00000000) refers (Special) to __rtentry4.o(.ARM.Collect$$rtentry$$00000004) for __rt_entry_sh
    aeabi_idiv0_sigfpe.o(.text) refers to rt_div0.o(.text) for __rt_div0
    _rserrno.o(.text) refers to rt_errno_addr_intlibspace.o(.text) for __aeabi_errno_addr
    _printf_intcommon.o(.text) refers (Weak) to _printf_pad.o(.text) for _printf_pre_padding
    _printf_intcommon.o(.text) refers (Weak) to _printf_pad.o(.text) for _printf_pre_padding
    _printf_intcommon.o(.text) refers (Weak) to _printf_pad.o(.text) for _printf_post_padding
    _printf_fp_dec.o(.text) refers (Special) to usenofp.o(x$fpl$usenofp) for __I$use$fp
    _printf_fp_dec.o(.text) refers (Special) to lc_numeric_c.o(locale$$code) for _get_lc_numeric
    _printf_fp_dec.o(.text) refers to bigflt0.o(.text) for _btod_etento
    _printf_fp_dec.o(.text) refers to btod.o(.text) for _btod_d2e
    _printf_fp_dec.o(.text) refers to lludiv10.o(.text) for _ll_udiv10
    _printf_fp_dec.o(.text) refers to fpclassify.o(i.__ARM_fpclassify) for __ARM_fpclassify
    _printf_fp_dec.o(.text) refers to _printf_fp_infnan.o(.text) for _printf_fp_infnan
    _printf_fp_dec.o(.text) refers to rtudiv10.o(.text) for __rt_udiv10
    _printf_fp_dec.o(.text) refers (Weak) to _printf_pad.o(.text) for _printf_pre_padding
    _printf_fp_dec.o(.text) refers (Weak) to _printf_pad.o(.text) for _printf_pre_padding
    _printf_fp_dec.o(.text) refers to rt_locale_intlibspace.o(.text) for __rt_locale
    _printf_fp_dec.o(.text) refers (Weak) to _printf_pad.o(.text) for _printf_post_padding
    _printf_fp_dec_accurate.o(.text) refers (Special) to usenofp.o(x$fpl$usenofp) for __I$use$fp
    _printf_fp_dec_accurate.o(.text) refers (Special) to lc_numeric_c.o(locale$$code) for _get_lc_numeric
    _printf_fp_dec_accurate.o(.text) refers to btod_accurate.o(.text) for _btod_main
    _printf_fp_dec_accurate.o(.text) refers to fpclassify.o(i.__ARM_fpclassify) for __ARM_fpclassify
    _printf_fp_dec_accurate.o(.text) refers to _printf_fp_infnan.o(.text) for _printf_fp_infnan
    _printf_fp_dec_accurate.o(.text) refers to rtudiv10.o(.text) for __rt_udiv10
    _printf_fp_dec_accurate.o(.text) refers (Weak) to _printf_pad.o(.text) for _printf_pre_padding
    _printf_fp_dec_accurate.o(.text) refers (Weak) to _printf_pad.o(.text) for _printf_pre_padding
    _printf_fp_dec_accurate.o(.text) refers to rt_locale_intlibspace.o(.text) for __rt_locale
    _printf_fp_dec_accurate.o(.text) refers (Weak) to _printf_pad.o(.text) for _printf_post_padding
    _printf_char_common.o(.text) refers to __printf_flags_wp.o(.text) for __printf
    _printf_char.o(.text) refers (Weak) to _printf_str.o(.text) for _printf_str
    drlef.o(x$fpl$drleqf) refers (Special) to usenofp.o(x$fpl$usenofp) for __I$use$fp
    drlef.o(x$fpl$drleqf) refers to dcmpin.o(.text) for __fpl_dcmp_InfNaN
    dscalbn.o(.text) refers (Special) to usenofp.o(x$fpl$usenofp) for __I$use$fp
    dunder.o(i.__mathlib_dbl_divzero) refers to ddiv.o(.text) for __aeabi_ddiv
    dunder.o(i.__mathlib_dbl_infnan) refers to dscalbn.o(.text) for __ARM_scalbn
    dunder.o(i.__mathlib_dbl_infnan2) refers to daddsub.o(.text) for __aeabi_dadd
    dunder.o(i.__mathlib_dbl_invalid) refers to ddiv.o(.text) for __aeabi_ddiv
    dunder.o(i.__mathlib_dbl_overflow) refers to dscalbn.o(.text) for __ARM_scalbn
    dunder.o(i.__mathlib_dbl_posinfnan) refers to dmul.o(.text) for __aeabi_dmul
    dunder.o(i.__mathlib_dbl_underflow) refers to dscalbn.o(.text) for __ARM_scalbn
    fpclassify.o(i.__ARM_fpclassify) refers (Special) to usenofp.o(x$fpl$usenofp) for __I$use$fp
    poly.o(i.__kernel_poly) refers (Special) to usenofp.o(x$fpl$usenofp) for __I$use$fp
    poly.o(i.__kernel_poly) refers to dmul.o(.text) for __aeabi_dmul
    poly.o(i.__kernel_poly) refers to daddsub.o(.text) for __aeabi_dadd
    qnan.o(.constdata) refers (Special) to usenofp.o(x$fpl$usenofp) for __I$use$fp
    sqrt.o(i.__softfp_sqrt) refers (Special) to usenofp.o(x$fpl$usenofp) for __I$use$fp
    sqrt.o(i.__softfp_sqrt) refers to dsqrt.o(.text) for _dsqrt
    sqrt.o(i.__softfp_sqrt) refers to _rserrno.o(.text) for __set_errno
    sqrt.o(i.sqrt) refers (Special) to usenofp.o(x$fpl$usenofp) for __I$use$fp
    sqrt.o(i.sqrt) refers to dsqrt.o(.text) for _dsqrt
    sqrt.o(i.sqrt) refers to _rserrno.o(.text) for __set_errno
    __rtentry2.o(.ARM.Collect$$rtentry$$00000008) refers to boardinit2.o(.text) for _platform_post_stackheap_init
    __rtentry2.o(.ARM.Collect$$rtentry$$0000000A) refers to libinit.o(.ARM.Collect$$libinit$$00000000) for __rt_lib_init
    __rtentry2.o(.ARM.Collect$$rtentry$$0000000B) refers to boardinit3.o(.text) for _platform_post_lib_init
    __rtentry2.o(.ARM.Collect$$rtentry$$0000000D) refers to main.o(.text.main) for main
    __rtentry2.o(.ARM.Collect$$rtentry$$0000000D) refers to exit.o(.text) for exit
    __rtentry2.o(.ARM.exidx) refers to __rtentry2.o(.ARM.Collect$$rtentry$$00000001) for .ARM.Collect$$rtentry$$00000001
    __rtentry2.o(.ARM.exidx) refers to __rtentry2.o(.ARM.Collect$$rtentry$$00000008) for .ARM.Collect$$rtentry$$00000008
    __rtentry2.o(.ARM.exidx) refers to __rtentry2.o(.ARM.Collect$$rtentry$$0000000A) for .ARM.Collect$$rtentry$$0000000A
    __rtentry2.o(.ARM.exidx) refers to __rtentry2.o(.ARM.Collect$$rtentry$$0000000B) for .ARM.Collect$$rtentry$$0000000B
    __rtentry2.o(.ARM.exidx) refers to __rtentry2.o(.ARM.Collect$$rtentry$$0000000D) for .ARM.Collect$$rtentry$$0000000D
    __rtentry4.o(.ARM.Collect$$rtentry$$00000004) refers to sys_stackheap_outer.o(.text) for __user_setup_stackheap
    __rtentry4.o(.ARM.exidx) refers to __rtentry4.o(.ARM.Collect$$rtentry$$00000004) for .ARM.Collect$$rtentry$$00000004
    rt_div0.o(.text) refers to defsig_fpe_outer.o(.text) for __rt_SIGFPE
    rt_locale.o(.text) refers to rt_locale.o(.bss) for __rt_locale_data
    rt_locale_intlibspace.o(.text) refers to libspace.o(.bss) for __libspace_start
    rt_errno_addr.o(.text) refers to rt_errno_addr.o(.bss) for __aeabi_errno_addr_data
    rt_errno_addr_intlibspace.o(.text) refers to libspace.o(.bss) for __libspace_start
    _printf_fp_infnan.o(.text) refers (Weak) to _printf_pad.o(.text) for _printf_pre_padding
    _printf_fp_infnan.o(.text) refers (Weak) to _printf_pad.o(.text) for _printf_post_padding
    bigflt0.o(.text) refers (Special) to usenofp.o(x$fpl$usenofp) for __I$use$fp
    bigflt0.o(.text) refers to aeabi_sdivfast.o(.text) for __aeabi_idivmod
    bigflt0.o(.text) refers to btod.o(.text) for _btod_emul
    bigflt0.o(.text) refers to bigflt0.o(.constdata) for .constdata
    bigflt0.o(.constdata) refers (Special) to usenofp.o(x$fpl$usenofp) for __I$use$fp
    btod.o(.text) refers to btod.o(i.__ARM_common_ll_muluu) for __ARM_common_ll_muluu
    btod_accurate.o(.text) refers to btod_accurate_common.o(.text) for _btod_common
    lc_numeric_c.o(locale$$data) refers (Special) to libinit2.o(.ARM.Collect$$libinit$$00000018) for __rt_lib_init_lc_numeric_2
    lc_numeric_c.o(locale$$code) refers (Special) to libinit2.o(.ARM.Collect$$libinit$$00000018) for __rt_lib_init_lc_numeric_2
    lc_numeric_c.o(locale$$code) refers to strcmpv6m.o(.text) for strcmp
    lc_numeric_c.o(locale$$code) refers to lc_numeric_c.o(locale$$data) for __lcnum_c_name
    dcmpin.o(.text) refers (Special) to usenofp.o(x$fpl$usenofp) for __I$use$fp
    dcmpin.o(.text) refers to cmpret.o(.text) for __fpl_cmpreturn
    dcmpin.o(.text) refers to dnan2.o(.text) for __fpl_dcheck_NaN2
    dsqrt.o(.text) refers (Special) to usenofp.o(x$fpl$usenofp) for __I$use$fp
    ieee_status.o(.text) refers (Special) to usenofp.o(x$fpl$usenofp) for __I$use$fp
    libspace.o(.text) refers to libspace.o(.bss) for __libspace_start
    sys_stackheap_outer.o(.text) refers to libspace.o(.text) for __user_perproc_libspace
    sys_stackheap_outer.o(.text) refers to startup_stm32f030xc.o(.text) for __user_initial_stackheap
    sys_stackheap_outer.o(__vectab_stack_and_reset_area) refers to tempstk.o(.text) for __temporary_stack_top
    sys_stackheap_outer.o(__vectab_stack_and_reset_area) refers to __main.o(!!!main) for __main
    btod_accurate_common.o(.text) refers to aeabi_sdivfast.o(.text) for __aeabi_uidivmod
    btod_accurate_common.o(.text) refers to llushr.o(.text) for __aeabi_llsr
    exit.o(.text) refers to rtexit.o(.ARM.Collect$$rtexit$$00000000) for __rt_exit
    defsig_fpe_outer.o(.text) refers to defsig_fpe_inner.o(.text) for __rt_SIGFPE_inner
    defsig_fpe_outer.o(.text) refers to defsig_exit.o(.text) for __sig_exit
    defsig_fpe_formal.o(.text) refers to rt_raise.o(.text) for __rt_raise
    libinit.o(.ARM.Collect$$libinit$$00000000) refers (Special) to libinit2.o(.ARM.Collect$$libinit$$00000030) for __rt_lib_init_alloca_1
    libinit.o(.ARM.Collect$$libinit$$00000000) refers (Special) to libinit2.o(.ARM.Collect$$libinit$$0000002E) for __rt_lib_init_argv_1
    libinit.o(.ARM.Collect$$libinit$$00000000) refers (Special) to libinit2.o(.ARM.Collect$$libinit$$0000001D) for __rt_lib_init_atexit_1
    libinit.o(.ARM.Collect$$libinit$$00000000) refers (Special) to libinit2.o(.ARM.Collect$$libinit$$00000023) for __rt_lib_init_clock_1
    libinit.o(.ARM.Collect$$libinit$$00000000) refers (Special) to libinit2.o(.ARM.Collect$$libinit$$00000034) for __rt_lib_init_cpp_1
    libinit.o(.ARM.Collect$$libinit$$00000000) refers (Special) to libinit2.o(.ARM.Collect$$libinit$$00000032) for __rt_lib_init_exceptions_1
    libinit.o(.ARM.Collect$$libinit$$00000000) refers (Special) to libinit2.o(.ARM.Collect$$libinit$$00000002) for __rt_lib_init_fp_1
    libinit.o(.ARM.Collect$$libinit$$00000000) refers (Special) to libinit2.o(.ARM.Collect$$libinit$$00000021) for __rt_lib_init_fp_trap_1
    libinit.o(.ARM.Collect$$libinit$$00000000) refers (Special) to libinit2.o(.ARM.Collect$$libinit$$00000025) for __rt_lib_init_getenv_1
    libinit.o(.ARM.Collect$$libinit$$00000000) refers (Special) to libinit2.o(.ARM.Collect$$libinit$$0000000C) for __rt_lib_init_heap_1
    libinit.o(.ARM.Collect$$libinit$$00000000) refers (Special) to libinit2.o(.ARM.Collect$$libinit$$00000013) for __rt_lib_init_lc_collate_1
    libinit.o(.ARM.Collect$$libinit$$00000000) refers (Special) to libinit2.o(.ARM.Collect$$libinit$$00000015) for __rt_lib_init_lc_ctype_1
    libinit.o(.ARM.Collect$$libinit$$00000000) refers (Special) to libinit2.o(.ARM.Collect$$libinit$$00000017) for __rt_lib_init_lc_monetary_1
    libinit.o(.ARM.Collect$$libinit$$00000000) refers (Special) to libinit2.o(.ARM.Collect$$libinit$$00000019) for __rt_lib_init_lc_numeric_1
    libinit.o(.ARM.Collect$$libinit$$00000000) refers (Special) to libinit2.o(.ARM.Collect$$libinit$$0000001B) for __rt_lib_init_lc_time_1
    libinit.o(.ARM.Collect$$libinit$$00000000) refers (Special) to libinit2.o(.ARM.Collect$$libinit$$00000006) for __rt_lib_init_preinit_1
    libinit.o(.ARM.Collect$$libinit$$00000000) refers (Special) to libinit2.o(.ARM.Collect$$libinit$$00000010) for __rt_lib_init_rand_1
    libinit.o(.ARM.Collect$$libinit$$00000000) refers (Special) to libinit2.o(.ARM.Collect$$libinit$$00000004) for __rt_lib_init_relocate_pie_1
    libinit.o(.ARM.Collect$$libinit$$00000000) refers (Special) to libinit2.o(.ARM.Collect$$libinit$$00000035) for __rt_lib_init_return
    libinit.o(.ARM.Collect$$libinit$$00000000) refers (Special) to libinit2.o(.ARM.Collect$$libinit$$0000001F) for __rt_lib_init_signal_1
    libinit.o(.ARM.Collect$$libinit$$00000000) refers (Special) to libinit2.o(.ARM.Collect$$libinit$$00000027) for __rt_lib_init_stdio_1
    libinit.o(.ARM.Collect$$libinit$$00000000) refers (Special) to libinit2.o(.ARM.Collect$$libinit$$0000000E) for __rt_lib_init_user_alloc_1
    libinit2.o(.ARM.Collect$$libinit$$00000011) refers (Weak) to rt_locale_intlibspace.o(.text) for __rt_locale
    libinit2.o(.ARM.Collect$$libinit$$00000012) refers to libinit2.o(.ARM.Collect$$libinit$$00000011) for .ARM.Collect$$libinit$$00000011
    libinit2.o(.ARM.Collect$$libinit$$00000014) refers to libinit2.o(.ARM.Collect$$libinit$$00000011) for .ARM.Collect$$libinit$$00000011
    libinit2.o(.ARM.Collect$$libinit$$00000016) refers to libinit2.o(.ARM.Collect$$libinit$$00000011) for .ARM.Collect$$libinit$$00000011
    libinit2.o(.ARM.Collect$$libinit$$00000018) refers to libinit2.o(.ARM.Collect$$libinit$$00000011) for .ARM.Collect$$libinit$$00000011
    libinit2.o(.ARM.Collect$$libinit$$00000018) refers (Weak) to lc_numeric_c.o(locale$$code) for _get_lc_numeric
    libinit2.o(.ARM.Collect$$libinit$$0000001A) refers to libinit2.o(.ARM.Collect$$libinit$$00000011) for .ARM.Collect$$libinit$$00000011
    libinit2.o(.ARM.Collect$$libinit$$00000028) refers to argv_veneer.o(.text) for __ARM_argv_veneer
    libinit2.o(.ARM.Collect$$libinit$$00000029) refers to argv_veneer.o(.text) for __ARM_argv_veneer
    cmpret.o(.text) refers (Special) to usenofp.o(x$fpl$usenofp) for __I$use$fp
    dnan2.o(.text) refers (Special) to usenofp.o(x$fpl$usenofp) for __I$use$fp
    dnan2.o(.text) refers to retnan.o(.text) for __fpl_return_NaN
    rtexit.o(.ARM.Collect$$rtexit$$00000000) refers (Special) to rtexit2.o(.ARM.Collect$$rtexit$$00000004) for __rt_exit_exit
    rtexit.o(.ARM.Collect$$rtexit$$00000000) refers (Special) to rtexit2.o(.ARM.Collect$$rtexit$$00000003) for __rt_exit_ls
    rtexit.o(.ARM.Collect$$rtexit$$00000000) refers (Special) to rtexit2.o(.ARM.Collect$$rtexit$$00000002) for __rt_exit_prels_1
    rtexit.o(.ARM.exidx) refers (Special) to rtexit2.o(.ARM.Collect$$rtexit$$00000004) for __rt_exit_exit
    rtexit.o(.ARM.exidx) refers (Special) to rtexit2.o(.ARM.Collect$$rtexit$$00000003) for __rt_exit_ls
    rtexit.o(.ARM.exidx) refers (Special) to rtexit2.o(.ARM.Collect$$rtexit$$00000002) for __rt_exit_prels_1
    rtexit.o(.ARM.exidx) refers to rtexit.o(.ARM.Collect$$rtexit$$00000000) for .ARM.Collect$$rtexit$$00000000
    rt_raise.o(.text) refers to __raise.o(.text) for __raise
    rt_raise.o(.text) refers to sys_exit.o(.text) for _sys_exit
    defsig_exit.o(.text) refers to sys_exit.o(.text) for _sys_exit
    defsig_fpe_inner.o(.text) refers to defsig_general.o(.text) for __default_signal_display
    retnan.o(.text) refers (Special) to usenofp.o(x$fpl$usenofp) for __I$use$fp
    retnan.o(.text) refers to cmpret.o(.text) for __fpl_cmpreturn
    sys_exit.o(.text) refers (Special) to use_no_semi.o(.text) for __I$use$semihosting
    sys_exit.o(.text) refers (Special) to indicate_semi.o(.text) for __semihosting_library_function
    sys_exit_hlt.o(.text) refers (Special) to use_no_semi.o(.text) for __I$use$semihosting
    sys_exit_hlt.o(.text) refers (Special) to indicate_semi.o(.text) for __semihosting_library_function
    rtexit2.o(.ARM.Collect$$rtexit$$00000003) refers to libshutdown.o(.ARM.Collect$$libshutdown$$00000000) for __rt_lib_shutdown
    rtexit2.o(.ARM.Collect$$rtexit$$00000004) refers to sys_exit.o(.text) for _sys_exit
    rtexit2.o(.ARM.exidx) refers to rtexit2.o(.ARM.Collect$$rtexit$$00000001) for .ARM.Collect$$rtexit$$00000001
    rtexit2.o(.ARM.exidx) refers to rtexit2.o(.ARM.Collect$$rtexit$$00000003) for .ARM.Collect$$rtexit$$00000003
    rtexit2.o(.ARM.exidx) refers to rtexit2.o(.ARM.Collect$$rtexit$$00000004) for .ARM.Collect$$rtexit$$00000004
    __raise.o(.text) refers to defsig.o(CL$$defsig) for __default_signal_handler
    defsig_general.o(.text) refers to sys_wrch.o(.text) for _ttywrch
    _get_argv_nomalloc.o(.text) refers (Special) to hrguard.o(.text) for __heap_region$guard
    _get_argv_nomalloc.o(.text) refers to defsig_rtmem_outer.o(.text) for __rt_SIGRTMEM
    _get_argv_nomalloc.o(.text) refers to sys_command.o(.text) for _sys_command_string
    sys_wrch.o(.text) refers (Special) to use_no_semi.o(.text) for __I$use$semihosting
    sys_wrch.o(.text) refers (Special) to indicate_semi.o(.text) for __semihosting_library_function
    sys_command.o(.text) refers (Special) to use_no_semi.o(.text) for __I$use$semihosting
    sys_command.o(.text) refers (Special) to indicate_semi.o(.text) for __semihosting_library_function
    sys_wrch_hlt.o(.text) refers (Special) to use_no_semi.o(.text) for __I$use$semihosting
    sys_wrch_hlt.o(.text) refers (Special) to indicate_semi.o(.text) for __semihosting_library_function
    sys_command_hlt.o(.text) refers (Special) to use_no_semi.o(.text) for __I$use$semihosting
    sys_command_hlt.o(.text) refers (Special) to indicate_semi.o(.text) for __semihosting_library_function
    defsig_rtmem_outer.o(.text) refers to defsig_rtmem_inner.o(.text) for __rt_SIGRTMEM_inner
    defsig_rtmem_outer.o(.text) refers to defsig_exit.o(.text) for __sig_exit
    defsig_rtmem_formal.o(.text) refers to rt_raise.o(.text) for __rt_raise
    defsig.o(CL$$defsig) refers to defsig_fpe_inner.o(.text) for __rt_SIGFPE_inner
    defsig.o(CL$$defsig) refers to defsig_rtmem_inner.o(.text) for __rt_SIGRTMEM_inner
    libshutdown.o(.ARM.Collect$$libshutdown$$00000000) refers (Special) to libshutdown2.o(.ARM.Collect$$libshutdown$$00000002) for __rt_lib_shutdown_cpp_1
    libshutdown.o(.ARM.Collect$$libshutdown$$00000000) refers (Special) to libshutdown2.o(.ARM.Collect$$libshutdown$$00000007) for __rt_lib_shutdown_fp_trap_1
    libshutdown.o(.ARM.Collect$$libshutdown$$00000000) refers (Special) to libshutdown2.o(.ARM.Collect$$libshutdown$$0000000F) for __rt_lib_shutdown_heap_1
    libshutdown.o(.ARM.Collect$$libshutdown$$00000000) refers (Special) to libshutdown2.o(.ARM.Collect$$libshutdown$$00000010) for __rt_lib_shutdown_return
    libshutdown.o(.ARM.Collect$$libshutdown$$00000000) refers (Special) to libshutdown2.o(.ARM.Collect$$libshutdown$$0000000A) for __rt_lib_shutdown_signal_1
    libshutdown.o(.ARM.Collect$$libshutdown$$00000000) refers (Special) to libshutdown2.o(.ARM.Collect$$libshutdown$$00000004) for __rt_lib_shutdown_stdio_1
    libshutdown.o(.ARM.Collect$$libshutdown$$00000000) refers (Special) to libshutdown2.o(.ARM.Collect$$libshutdown$$0000000C) for __rt_lib_shutdown_user_alloc_1
    defsig_abrt_inner.o(.text) refers to defsig_general.o(.text) for __default_signal_display
    defsig_rtred_inner.o(.text) refers to defsig_general.o(.text) for __default_signal_display
    defsig_rtmem_inner.o(.text) refers to defsig_general.o(.text) for __default_signal_display
    defsig_stak_inner.o(.text) refers to defsig_general.o(.text) for __default_signal_display
    defsig_pvfn_inner.o(.text) refers to defsig_general.o(.text) for __default_signal_display
    defsig_cppl_inner.o(.text) refers to defsig_general.o(.text) for __default_signal_display
    defsig_segv_inner.o(.text) refers to defsig_general.o(.text) for __default_signal_display
    defsig_other.o(.text) refers to defsig_general.o(.text) for __default_signal_display


==============================================================================

Removing Unused input sections from the image.

    Removing main.o(.text), (0 bytes).
    Removing main.o(.ARM.exidx.text.main), (8 bytes).
    Removing main.o(.ARM.exidx.text.SystemClock_Config), (8 bytes).
    Removing main.o(.text.Error_Handler), (8 bytes).
    Removing main.o(.ARM.exidx.text.Error_Handler), (8 bytes).
    Removing main.o(.ARM.use_no_argv), (4 bytes).
    Removing stm32f0xx_it.o(.text), (0 bytes).
    Removing stm32f0xx_it.o(.ARM.exidx.text.NMI_Handler), (8 bytes).
    Removing stm32f0xx_it.o(.ARM.exidx.text.HardFault_Handler), (8 bytes).
    Removing stm32f0xx_it.o(.ARM.exidx.text.SVC_Handler), (8 bytes).
    Removing stm32f0xx_it.o(.ARM.exidx.text.PendSV_Handler), (8 bytes).
    Removing stm32f0xx_it.o(.ARM.exidx.text.SysTick_Handler), (8 bytes).
    Removing stm32f0xx_hal_msp.o(.text), (0 bytes).
    Removing stm32f0xx_hal_msp.o(.ARM.exidx.text.HAL_MspInit), (8 bytes).
    Removing stm32f0xx_hal_msp.o(.ARM.exidx.text.HAL_I2C_MspInit), (8 bytes).
    Removing stm32f0xx_hal_msp.o(.text.HAL_I2C_MspDeInit), (56 bytes).
    Removing stm32f0xx_hal_msp.o(.ARM.exidx.text.HAL_I2C_MspDeInit), (8 bytes).
    Removing stm32f0xx_hal_msp.o(.ARM.exidx.text.HAL_RTC_MspInit), (8 bytes).
    Removing stm32f0xx_hal_msp.o(.text.HAL_RTC_MspDeInit), (32 bytes).
    Removing stm32f0xx_hal_msp.o(.ARM.exidx.text.HAL_RTC_MspDeInit), (8 bytes).
    Removing bmp280+aht20.o(.text), (0 bytes).
    Removing bmp280+aht20.o(.ARM.exidx.text.BMP280_init), (8 bytes).
    Removing bmp280+aht20.o(.text.BMP280_get_calib_values), (164 bytes).
    Removing bmp280+aht20.o(.ARM.exidx.text.BMP280_get_calib_values), (8 bytes).
    Removing bmp280+aht20.o(.ARM.exidx.text.BMP280_calc_values), (8 bytes).
    Removing bmp280+aht20.o(.text.AHT20_init), (36 bytes).
    Removing bmp280+aht20.o(.ARM.exidx.text.AHT20_init), (8 bytes).
    Removing bmp280+aht20.o(.ARM.exidx.text.AHT20_Read), (8 bytes).
    Removing ssd1306.o(.text), (0 bytes).
    Removing ssd1306.o(.ARM.exidx.text.init_OLED), (8 bytes).
    Removing ssd1306.o(.text.sendcommand), (40 bytes).
    Removing ssd1306.o(.ARM.exidx.text.sendcommand), (8 bytes).
    Removing ssd1306.o(.text.SendChar), (40 bytes).
    Removing ssd1306.o(.ARM.exidx.text.SendChar), (8 bytes).
    Removing ssd1306.o(.text.displayOn), (68 bytes).
    Removing ssd1306.o(.ARM.exidx.text.displayOn), (8 bytes).
    Removing ssd1306.o(.text.displayOff), (40 bytes).
    Removing ssd1306.o(.ARM.exidx.text.displayOff), (8 bytes).
    Removing ssd1306.o(.text.setXY), (108 bytes).
    Removing ssd1306.o(.ARM.exidx.text.setXY), (8 bytes).
    Removing ssd1306.o(.ARM.exidx.text.clear_display), (8 bytes).
    Removing ssd1306.o(.ARM.exidx.text.OLCD_write_string), (8 bytes).
    Removing stm32f0xx_hal_i2c.o(.text), (0 bytes).
    Removing stm32f0xx_hal_i2c.o(.ARM.exidx.text.HAL_I2C_Init), (8 bytes).
    Removing stm32f0xx_hal_i2c.o(.text.HAL_I2C_MspInit), (2 bytes).
    Removing stm32f0xx_hal_i2c.o(.ARM.exidx.text.HAL_I2C_MspInit), (8 bytes).
    Removing stm32f0xx_hal_i2c.o(.text.HAL_I2C_DeInit), (50 bytes).
    Removing stm32f0xx_hal_i2c.o(.ARM.exidx.text.HAL_I2C_DeInit), (8 bytes).
    Removing stm32f0xx_hal_i2c.o(.text.HAL_I2C_MspDeInit), (2 bytes).
    Removing stm32f0xx_hal_i2c.o(.ARM.exidx.text.HAL_I2C_MspDeInit), (8 bytes).
    Removing stm32f0xx_hal_i2c.o(.ARM.exidx.text.HAL_I2C_Master_Transmit), (8 bytes).
    Removing stm32f0xx_hal_i2c.o(.ARM.exidx.text.I2C_WaitOnFlagUntilTimeout), (8 bytes).
    Removing stm32f0xx_hal_i2c.o(.ARM.exidx.text.I2C_WaitOnTXISFlagUntilTimeout), (8 bytes).
    Removing stm32f0xx_hal_i2c.o(.ARM.exidx.text.I2C_WaitOnSTOPFlagUntilTimeout), (8 bytes).
    Removing stm32f0xx_hal_i2c.o(.ARM.exidx.text.HAL_I2C_Master_Receive), (8 bytes).
    Removing stm32f0xx_hal_i2c.o(.ARM.exidx.text.I2C_WaitOnRXNEFlagUntilTimeout), (8 bytes).
    Removing stm32f0xx_hal_i2c.o(.text.HAL_I2C_Slave_Transmit), (526 bytes).
    Removing stm32f0xx_hal_i2c.o(.ARM.exidx.text.HAL_I2C_Slave_Transmit), (8 bytes).
    Removing stm32f0xx_hal_i2c.o(.text.HAL_I2C_Slave_Receive), (370 bytes).
    Removing stm32f0xx_hal_i2c.o(.ARM.exidx.text.HAL_I2C_Slave_Receive), (8 bytes).
    Removing stm32f0xx_hal_i2c.o(.text.HAL_I2C_Master_Transmit_IT), (180 bytes).
    Removing stm32f0xx_hal_i2c.o(.ARM.exidx.text.HAL_I2C_Master_Transmit_IT), (8 bytes).
    Removing stm32f0xx_hal_i2c.o(.text.I2C_Master_ISR_IT), (428 bytes).
    Removing stm32f0xx_hal_i2c.o(.ARM.exidx.text.I2C_Master_ISR_IT), (8 bytes).
    Removing stm32f0xx_hal_i2c.o(.text.HAL_I2C_Master_Receive_IT), (132 bytes).
    Removing stm32f0xx_hal_i2c.o(.ARM.exidx.text.HAL_I2C_Master_Receive_IT), (8 bytes).
    Removing stm32f0xx_hal_i2c.o(.text.HAL_I2C_Slave_Transmit_IT), (124 bytes).
    Removing stm32f0xx_hal_i2c.o(.ARM.exidx.text.HAL_I2C_Slave_Transmit_IT), (8 bytes).
    Removing stm32f0xx_hal_i2c.o(.text.I2C_Slave_ISR_IT), (508 bytes).
    Removing stm32f0xx_hal_i2c.o(.ARM.exidx.text.I2C_Slave_ISR_IT), (8 bytes).
    Removing stm32f0xx_hal_i2c.o(.text.HAL_I2C_Slave_Receive_IT), (84 bytes).
    Removing stm32f0xx_hal_i2c.o(.ARM.exidx.text.HAL_I2C_Slave_Receive_IT), (8 bytes).
    Removing stm32f0xx_hal_i2c.o(.text.HAL_I2C_Master_Transmit_DMA), (352 bytes).
    Removing stm32f0xx_hal_i2c.o(.ARM.exidx.text.HAL_I2C_Master_Transmit_DMA), (8 bytes).
    Removing stm32f0xx_hal_i2c.o(.text.I2C_Master_ISR_DMA), (484 bytes).
    Removing stm32f0xx_hal_i2c.o(.ARM.exidx.text.I2C_Master_ISR_DMA), (8 bytes).
    Removing stm32f0xx_hal_i2c.o(.text.I2C_DMAMasterTransmitCplt), (180 bytes).
    Removing stm32f0xx_hal_i2c.o(.ARM.exidx.text.I2C_DMAMasterTransmitCplt), (8 bytes).
    Removing stm32f0xx_hal_i2c.o(.text.I2C_DMAError), (24 bytes).
    Removing stm32f0xx_hal_i2c.o(.ARM.exidx.text.I2C_DMAError), (8 bytes).
    Removing stm32f0xx_hal_i2c.o(.text.HAL_I2C_Master_Receive_DMA), (324 bytes).
    Removing stm32f0xx_hal_i2c.o(.ARM.exidx.text.HAL_I2C_Master_Receive_DMA), (8 bytes).
    Removing stm32f0xx_hal_i2c.o(.text.I2C_DMAMasterReceiveCplt), (188 bytes).
    Removing stm32f0xx_hal_i2c.o(.ARM.exidx.text.I2C_DMAMasterReceiveCplt), (8 bytes).
    Removing stm32f0xx_hal_i2c.o(.text.HAL_I2C_Slave_Transmit_DMA), (264 bytes).
    Removing stm32f0xx_hal_i2c.o(.ARM.exidx.text.HAL_I2C_Slave_Transmit_DMA), (8 bytes).
    Removing stm32f0xx_hal_i2c.o(.text.I2C_Slave_ISR_DMA), (288 bytes).
    Removing stm32f0xx_hal_i2c.o(.ARM.exidx.text.I2C_Slave_ISR_DMA), (8 bytes).
    Removing stm32f0xx_hal_i2c.o(.text.I2C_DMASlaveTransmitCplt), (152 bytes).
    Removing stm32f0xx_hal_i2c.o(.ARM.exidx.text.I2C_DMASlaveTransmitCplt), (8 bytes).
    Removing stm32f0xx_hal_i2c.o(.text.HAL_I2C_Slave_Receive_DMA), (208 bytes).
    Removing stm32f0xx_hal_i2c.o(.ARM.exidx.text.HAL_I2C_Slave_Receive_DMA), (8 bytes).
    Removing stm32f0xx_hal_i2c.o(.text.I2C_DMASlaveReceiveCplt), (164 bytes).
    Removing stm32f0xx_hal_i2c.o(.ARM.exidx.text.I2C_DMASlaveReceiveCplt), (8 bytes).
    Removing stm32f0xx_hal_i2c.o(.text.HAL_I2C_Mem_Write), (560 bytes).
    Removing stm32f0xx_hal_i2c.o(.ARM.exidx.text.HAL_I2C_Mem_Write), (8 bytes).
    Removing stm32f0xx_hal_i2c.o(.ARM.exidx.text.HAL_I2C_Mem_Read), (8 bytes).
    Removing stm32f0xx_hal_i2c.o(.text.HAL_I2C_Mem_Write_IT), (176 bytes).
    Removing stm32f0xx_hal_i2c.o(.ARM.exidx.text.HAL_I2C_Mem_Write_IT), (8 bytes).
    Removing stm32f0xx_hal_i2c.o(.text.I2C_Mem_ISR_IT), (500 bytes).
    Removing stm32f0xx_hal_i2c.o(.ARM.exidx.text.I2C_Mem_ISR_IT), (8 bytes).
    Removing stm32f0xx_hal_i2c.o(.text.HAL_I2C_Mem_Read_IT), (172 bytes).
    Removing stm32f0xx_hal_i2c.o(.ARM.exidx.text.HAL_I2C_Mem_Read_IT), (8 bytes).
    Removing stm32f0xx_hal_i2c.o(.text.HAL_I2C_Mem_Write_DMA), (296 bytes).
    Removing stm32f0xx_hal_i2c.o(.ARM.exidx.text.HAL_I2C_Mem_Write_DMA), (8 bytes).
    Removing stm32f0xx_hal_i2c.o(.text.I2C_Mem_ISR_DMA), (504 bytes).
    Removing stm32f0xx_hal_i2c.o(.ARM.exidx.text.I2C_Mem_ISR_DMA), (8 bytes).
    Removing stm32f0xx_hal_i2c.o(.text.HAL_I2C_Mem_Read_DMA), (292 bytes).
    Removing stm32f0xx_hal_i2c.o(.ARM.exidx.text.HAL_I2C_Mem_Read_DMA), (8 bytes).
    Removing stm32f0xx_hal_i2c.o(.text.HAL_I2C_IsDeviceReady), (500 bytes).
    Removing stm32f0xx_hal_i2c.o(.ARM.exidx.text.HAL_I2C_IsDeviceReady), (8 bytes).
    Removing stm32f0xx_hal_i2c.o(.text.HAL_I2C_Master_Seq_Transmit_IT), (296 bytes).
    Removing stm32f0xx_hal_i2c.o(.ARM.exidx.text.HAL_I2C_Master_Seq_Transmit_IT), (8 bytes).
    Removing stm32f0xx_hal_i2c.o(.text.HAL_I2C_Master_Seq_Transmit_DMA), (540 bytes).
    Removing stm32f0xx_hal_i2c.o(.ARM.exidx.text.HAL_I2C_Master_Seq_Transmit_DMA), (8 bytes).
    Removing stm32f0xx_hal_i2c.o(.text.HAL_I2C_Master_Seq_Receive_IT), (196 bytes).
    Removing stm32f0xx_hal_i2c.o(.ARM.exidx.text.HAL_I2C_Master_Seq_Receive_IT), (8 bytes).
    Removing stm32f0xx_hal_i2c.o(.text.HAL_I2C_Master_Seq_Receive_DMA), (400 bytes).
    Removing stm32f0xx_hal_i2c.o(.ARM.exidx.text.HAL_I2C_Master_Seq_Receive_DMA), (8 bytes).
    Removing stm32f0xx_hal_i2c.o(.text.HAL_I2C_Slave_Seq_Transmit_IT), (228 bytes).
    Removing stm32f0xx_hal_i2c.o(.ARM.exidx.text.HAL_I2C_Slave_Seq_Transmit_IT), (8 bytes).
    Removing stm32f0xx_hal_i2c.o(.text.I2C_DMAAbort), (62 bytes).
    Removing stm32f0xx_hal_i2c.o(.ARM.exidx.text.I2C_DMAAbort), (8 bytes).
    Removing stm32f0xx_hal_i2c.o(.text.HAL_I2C_Slave_Seq_Transmit_DMA), (388 bytes).
    Removing stm32f0xx_hal_i2c.o(.ARM.exidx.text.HAL_I2C_Slave_Seq_Transmit_DMA), (8 bytes).
    Removing stm32f0xx_hal_i2c.o(.text.HAL_I2C_Slave_Seq_Receive_IT), (224 bytes).
    Removing stm32f0xx_hal_i2c.o(.ARM.exidx.text.HAL_I2C_Slave_Seq_Receive_IT), (8 bytes).
    Removing stm32f0xx_hal_i2c.o(.text.HAL_I2C_Slave_Seq_Receive_DMA), (384 bytes).
    Removing stm32f0xx_hal_i2c.o(.ARM.exidx.text.HAL_I2C_Slave_Seq_Receive_DMA), (8 bytes).
    Removing stm32f0xx_hal_i2c.o(.text.HAL_I2C_EnableListen_IT), (44 bytes).
    Removing stm32f0xx_hal_i2c.o(.ARM.exidx.text.HAL_I2C_EnableListen_IT), (8 bytes).
    Removing stm32f0xx_hal_i2c.o(.text.HAL_I2C_DisableListen_IT), (54 bytes).
    Removing stm32f0xx_hal_i2c.o(.ARM.exidx.text.HAL_I2C_DisableListen_IT), (8 bytes).
    Removing stm32f0xx_hal_i2c.o(.text.HAL_I2C_Master_Abort_IT), (200 bytes).
    Removing stm32f0xx_hal_i2c.o(.ARM.exidx.text.HAL_I2C_Master_Abort_IT), (8 bytes).
    Removing stm32f0xx_hal_i2c.o(.text.HAL_I2C_EV_IRQHandler), (18 bytes).
    Removing stm32f0xx_hal_i2c.o(.ARM.exidx.text.HAL_I2C_EV_IRQHandler), (8 bytes).
    Removing stm32f0xx_hal_i2c.o(.text.HAL_I2C_ER_IRQHandler), (130 bytes).
    Removing stm32f0xx_hal_i2c.o(.ARM.exidx.text.HAL_I2C_ER_IRQHandler), (8 bytes).
    Removing stm32f0xx_hal_i2c.o(.text.I2C_ITError), (352 bytes).
    Removing stm32f0xx_hal_i2c.o(.ARM.exidx.text.I2C_ITError), (8 bytes).
    Removing stm32f0xx_hal_i2c.o(.text.HAL_I2C_MasterTxCpltCallback), (2 bytes).
    Removing stm32f0xx_hal_i2c.o(.ARM.exidx.text.HAL_I2C_MasterTxCpltCallback), (8 bytes).
    Removing stm32f0xx_hal_i2c.o(.text.HAL_I2C_MasterRxCpltCallback), (2 bytes).
    Removing stm32f0xx_hal_i2c.o(.ARM.exidx.text.HAL_I2C_MasterRxCpltCallback), (8 bytes).
    Removing stm32f0xx_hal_i2c.o(.text.HAL_I2C_SlaveTxCpltCallback), (2 bytes).
    Removing stm32f0xx_hal_i2c.o(.ARM.exidx.text.HAL_I2C_SlaveTxCpltCallback), (8 bytes).
    Removing stm32f0xx_hal_i2c.o(.text.HAL_I2C_SlaveRxCpltCallback), (2 bytes).
    Removing stm32f0xx_hal_i2c.o(.ARM.exidx.text.HAL_I2C_SlaveRxCpltCallback), (8 bytes).
    Removing stm32f0xx_hal_i2c.o(.text.HAL_I2C_AddrCallback), (2 bytes).
    Removing stm32f0xx_hal_i2c.o(.ARM.exidx.text.HAL_I2C_AddrCallback), (8 bytes).
    Removing stm32f0xx_hal_i2c.o(.text.HAL_I2C_ListenCpltCallback), (2 bytes).
    Removing stm32f0xx_hal_i2c.o(.ARM.exidx.text.HAL_I2C_ListenCpltCallback), (8 bytes).
    Removing stm32f0xx_hal_i2c.o(.text.HAL_I2C_MemTxCpltCallback), (2 bytes).
    Removing stm32f0xx_hal_i2c.o(.ARM.exidx.text.HAL_I2C_MemTxCpltCallback), (8 bytes).
    Removing stm32f0xx_hal_i2c.o(.text.HAL_I2C_MemRxCpltCallback), (2 bytes).
    Removing stm32f0xx_hal_i2c.o(.ARM.exidx.text.HAL_I2C_MemRxCpltCallback), (8 bytes).
    Removing stm32f0xx_hal_i2c.o(.text.HAL_I2C_ErrorCallback), (2 bytes).
    Removing stm32f0xx_hal_i2c.o(.ARM.exidx.text.HAL_I2C_ErrorCallback), (8 bytes).
    Removing stm32f0xx_hal_i2c.o(.text.HAL_I2C_AbortCpltCallback), (2 bytes).
    Removing stm32f0xx_hal_i2c.o(.ARM.exidx.text.HAL_I2C_AbortCpltCallback), (8 bytes).
    Removing stm32f0xx_hal_i2c.o(.text.HAL_I2C_GetState), (6 bytes).
    Removing stm32f0xx_hal_i2c.o(.ARM.exidx.text.HAL_I2C_GetState), (8 bytes).
    Removing stm32f0xx_hal_i2c.o(.text.HAL_I2C_GetMode), (6 bytes).
    Removing stm32f0xx_hal_i2c.o(.ARM.exidx.text.HAL_I2C_GetMode), (8 bytes).
    Removing stm32f0xx_hal_i2c.o(.text.HAL_I2C_GetError), (4 bytes).
    Removing stm32f0xx_hal_i2c.o(.ARM.exidx.text.HAL_I2C_GetError), (8 bytes).
    Removing stm32f0xx_hal_i2c.o(.text.I2C_ITMasterSeqCplt), (96 bytes).
    Removing stm32f0xx_hal_i2c.o(.ARM.exidx.text.I2C_ITMasterSeqCplt), (8 bytes).
    Removing stm32f0xx_hal_i2c.o(.text.I2C_ITMasterCplt), (264 bytes).
    Removing stm32f0xx_hal_i2c.o(.ARM.exidx.text.I2C_ITMasterCplt), (8 bytes).
    Removing stm32f0xx_hal_i2c.o(.text.I2C_ITSlaveCplt), (892 bytes).
    Removing stm32f0xx_hal_i2c.o(.ARM.exidx.text.I2C_ITSlaveCplt), (8 bytes).
    Removing stm32f0xx_hal_i2c.o(.text.I2C_ITListenCplt), (96 bytes).
    Removing stm32f0xx_hal_i2c.o(.ARM.exidx.text.I2C_ITListenCplt), (8 bytes).
    Removing stm32f0xx_hal_i2c.o(.text.I2C_ITSlaveSeqCplt), (132 bytes).
    Removing stm32f0xx_hal_i2c.o(.ARM.exidx.text.I2C_ITSlaveSeqCplt), (8 bytes).
    Removing stm32f0xx_hal_i2c.o(.text.I2C_ITAddrCplt), (168 bytes).
    Removing stm32f0xx_hal_i2c.o(.ARM.exidx.text.I2C_ITAddrCplt), (8 bytes).
    Removing stm32f0xx_hal_i2c.o(.ARM.exidx.text.I2C_IsErrorOccurred), (8 bytes).
    Removing stm32f0xx_hal_i2c_ex.o(.text), (0 bytes).
    Removing stm32f0xx_hal_i2c_ex.o(.ARM.exidx.text.HAL_I2CEx_ConfigAnalogFilter), (8 bytes).
    Removing stm32f0xx_hal_i2c_ex.o(.ARM.exidx.text.HAL_I2CEx_ConfigDigitalFilter), (8 bytes).
    Removing stm32f0xx_hal_i2c_ex.o(.text.HAL_I2CEx_EnableFastModePlus), (40 bytes).
    Removing stm32f0xx_hal_i2c_ex.o(.ARM.exidx.text.HAL_I2CEx_EnableFastModePlus), (8 bytes).
    Removing stm32f0xx_hal_i2c_ex.o(.text.HAL_I2CEx_DisableFastModePlus), (40 bytes).
    Removing stm32f0xx_hal_i2c_ex.o(.ARM.exidx.text.HAL_I2CEx_DisableFastModePlus), (8 bytes).
    Removing stm32f0xx_hal_rcc.o(.text), (0 bytes).
    Removing stm32f0xx_hal_rcc.o(.text.HAL_RCC_DeInit), (184 bytes).
    Removing stm32f0xx_hal_rcc.o(.ARM.exidx.text.HAL_RCC_DeInit), (8 bytes).
    Removing stm32f0xx_hal_rcc.o(.ARM.exidx.text.HAL_RCC_OscConfig), (8 bytes).
    Removing stm32f0xx_hal_rcc.o(.ARM.exidx.text.HAL_RCC_ClockConfig), (8 bytes).
    Removing stm32f0xx_hal_rcc.o(.text.HAL_RCC_GetSysClockFreq), (60 bytes).
    Removing stm32f0xx_hal_rcc.o(.ARM.exidx.text.HAL_RCC_GetSysClockFreq), (8 bytes).
    Removing stm32f0xx_hal_rcc.o(.text.HAL_RCC_MCOConfig), (80 bytes).
    Removing stm32f0xx_hal_rcc.o(.ARM.exidx.text.HAL_RCC_MCOConfig), (8 bytes).
    Removing stm32f0xx_hal_rcc.o(.text.HAL_RCC_EnableCSS), (20 bytes).
    Removing stm32f0xx_hal_rcc.o(.ARM.exidx.text.HAL_RCC_EnableCSS), (8 bytes).
    Removing stm32f0xx_hal_rcc.o(.text.HAL_RCC_DisableCSS), (20 bytes).
    Removing stm32f0xx_hal_rcc.o(.ARM.exidx.text.HAL_RCC_DisableCSS), (8 bytes).
    Removing stm32f0xx_hal_rcc.o(.text.HAL_RCC_GetHCLKFreq), (12 bytes).
    Removing stm32f0xx_hal_rcc.o(.ARM.exidx.text.HAL_RCC_GetHCLKFreq), (8 bytes).
    Removing stm32f0xx_hal_rcc.o(.text.HAL_RCC_GetPCLK1Freq), (32 bytes).
    Removing stm32f0xx_hal_rcc.o(.ARM.exidx.text.HAL_RCC_GetPCLK1Freq), (8 bytes).
    Removing stm32f0xx_hal_rcc.o(.text.HAL_RCC_GetOscConfig), (136 bytes).
    Removing stm32f0xx_hal_rcc.o(.ARM.exidx.text.HAL_RCC_GetOscConfig), (8 bytes).
    Removing stm32f0xx_hal_rcc.o(.text.HAL_RCC_GetClockConfig), (52 bytes).
    Removing stm32f0xx_hal_rcc.o(.ARM.exidx.text.HAL_RCC_GetClockConfig), (8 bytes).
    Removing stm32f0xx_hal_rcc.o(.text.HAL_RCC_NMI_IRQHandler), (24 bytes).
    Removing stm32f0xx_hal_rcc.o(.ARM.exidx.text.HAL_RCC_NMI_IRQHandler), (8 bytes).
    Removing stm32f0xx_hal_rcc.o(.text.HAL_RCC_CSSCallback), (2 bytes).
    Removing stm32f0xx_hal_rcc.o(.ARM.exidx.text.HAL_RCC_CSSCallback), (8 bytes).
    Removing stm32f0xx_hal_rcc_ex.o(.text), (0 bytes).
    Removing stm32f0xx_hal_rcc_ex.o(.ARM.exidx.text.HAL_RCCEx_PeriphCLKConfig), (8 bytes).
    Removing stm32f0xx_hal_rcc_ex.o(.text.HAL_RCCEx_GetPeriphCLKConfig), (48 bytes).
    Removing stm32f0xx_hal_rcc_ex.o(.ARM.exidx.text.HAL_RCCEx_GetPeriphCLKConfig), (8 bytes).
    Removing stm32f0xx_hal_rcc_ex.o(.text.HAL_RCCEx_GetPeriphCLKFreq), (164 bytes).
    Removing stm32f0xx_hal_rcc_ex.o(.ARM.exidx.text.HAL_RCCEx_GetPeriphCLKFreq), (8 bytes).
    Removing stm32f0xx_hal.o(.text), (0 bytes).
    Removing stm32f0xx_hal.o(.ARM.exidx.text.HAL_Init), (8 bytes).
    Removing stm32f0xx_hal.o(.ARM.exidx.text.HAL_InitTick), (8 bytes).
    Removing stm32f0xx_hal.o(.text.HAL_MspInit), (2 bytes).
    Removing stm32f0xx_hal.o(.ARM.exidx.text.HAL_MspInit), (8 bytes).
    Removing stm32f0xx_hal.o(.text.HAL_DeInit), (32 bytes).
    Removing stm32f0xx_hal.o(.ARM.exidx.text.HAL_DeInit), (8 bytes).
    Removing stm32f0xx_hal.o(.text.HAL_MspDeInit), (2 bytes).
    Removing stm32f0xx_hal.o(.ARM.exidx.text.HAL_MspDeInit), (8 bytes).
    Removing stm32f0xx_hal.o(.ARM.exidx.text.HAL_IncTick), (8 bytes).
    Removing stm32f0xx_hal.o(.ARM.exidx.text.HAL_GetTick), (8 bytes).
    Removing stm32f0xx_hal.o(.text.HAL_GetTickPrio), (12 bytes).
    Removing stm32f0xx_hal.o(.ARM.exidx.text.HAL_GetTickPrio), (8 bytes).
    Removing stm32f0xx_hal.o(.text.HAL_SetTickFreq), (36 bytes).
    Removing stm32f0xx_hal.o(.ARM.exidx.text.HAL_SetTickFreq), (8 bytes).
    Removing stm32f0xx_hal.o(.text.HAL_GetTickFreq), (12 bytes).
    Removing stm32f0xx_hal.o(.ARM.exidx.text.HAL_GetTickFreq), (8 bytes).
    Removing stm32f0xx_hal.o(.ARM.exidx.text.HAL_Delay), (8 bytes).
    Removing stm32f0xx_hal.o(.text.HAL_SuspendTick), (16 bytes).
    Removing stm32f0xx_hal.o(.ARM.exidx.text.HAL_SuspendTick), (8 bytes).
    Removing stm32f0xx_hal.o(.text.HAL_ResumeTick), (16 bytes).
    Removing stm32f0xx_hal.o(.ARM.exidx.text.HAL_ResumeTick), (8 bytes).
    Removing stm32f0xx_hal.o(.text.HAL_GetHalVersion), (8 bytes).
    Removing stm32f0xx_hal.o(.ARM.exidx.text.HAL_GetHalVersion), (8 bytes).
    Removing stm32f0xx_hal.o(.text.HAL_GetREVID), (12 bytes).
    Removing stm32f0xx_hal.o(.ARM.exidx.text.HAL_GetREVID), (8 bytes).
    Removing stm32f0xx_hal.o(.text.HAL_GetDEVID), (20 bytes).
    Removing stm32f0xx_hal.o(.ARM.exidx.text.HAL_GetDEVID), (8 bytes).
    Removing stm32f0xx_hal.o(.text.HAL_GetUIDw0), (12 bytes).
    Removing stm32f0xx_hal.o(.ARM.exidx.text.HAL_GetUIDw0), (8 bytes).
    Removing stm32f0xx_hal.o(.text.HAL_GetUIDw1), (12 bytes).
    Removing stm32f0xx_hal.o(.ARM.exidx.text.HAL_GetUIDw1), (8 bytes).
    Removing stm32f0xx_hal.o(.text.HAL_GetUIDw2), (12 bytes).
    Removing stm32f0xx_hal.o(.ARM.exidx.text.HAL_GetUIDw2), (8 bytes).
    Removing stm32f0xx_hal.o(.text.HAL_DBGMCU_EnableDBGStopMode), (16 bytes).
    Removing stm32f0xx_hal.o(.ARM.exidx.text.HAL_DBGMCU_EnableDBGStopMode), (8 bytes).
    Removing stm32f0xx_hal.o(.text.HAL_DBGMCU_DisableDBGStopMode), (16 bytes).
    Removing stm32f0xx_hal.o(.ARM.exidx.text.HAL_DBGMCU_DisableDBGStopMode), (8 bytes).
    Removing stm32f0xx_hal.o(.text.HAL_DBGMCU_EnableDBGStandbyMode), (16 bytes).
    Removing stm32f0xx_hal.o(.ARM.exidx.text.HAL_DBGMCU_EnableDBGStandbyMode), (8 bytes).
    Removing stm32f0xx_hal.o(.text.HAL_DBGMCU_DisableDBGStandbyMode), (16 bytes).
    Removing stm32f0xx_hal.o(.ARM.exidx.text.HAL_DBGMCU_DisableDBGStandbyMode), (8 bytes).
    Removing stm32f0xx_hal_gpio.o(.text), (0 bytes).
    Removing stm32f0xx_hal_gpio.o(.ARM.exidx.text.HAL_GPIO_Init), (8 bytes).
    Removing stm32f0xx_hal_gpio.o(.text.HAL_GPIO_DeInit), (252 bytes).
    Removing stm32f0xx_hal_gpio.o(.ARM.exidx.text.HAL_GPIO_DeInit), (8 bytes).
    Removing stm32f0xx_hal_gpio.o(.text.HAL_GPIO_ReadPin), (10 bytes).
    Removing stm32f0xx_hal_gpio.o(.ARM.exidx.text.HAL_GPIO_ReadPin), (8 bytes).
    Removing stm32f0xx_hal_gpio.o(.text.HAL_GPIO_WritePin), (16 bytes).
    Removing stm32f0xx_hal_gpio.o(.ARM.exidx.text.HAL_GPIO_WritePin), (8 bytes).
    Removing stm32f0xx_hal_gpio.o(.text.HAL_GPIO_TogglePin), (16 bytes).
    Removing stm32f0xx_hal_gpio.o(.ARM.exidx.text.HAL_GPIO_TogglePin), (8 bytes).
    Removing stm32f0xx_hal_gpio.o(.text.HAL_GPIO_LockPin), (40 bytes).
    Removing stm32f0xx_hal_gpio.o(.ARM.exidx.text.HAL_GPIO_LockPin), (8 bytes).
    Removing stm32f0xx_hal_gpio.o(.text.HAL_GPIO_EXTI_IRQHandler), (24 bytes).
    Removing stm32f0xx_hal_gpio.o(.ARM.exidx.text.HAL_GPIO_EXTI_IRQHandler), (8 bytes).
    Removing stm32f0xx_hal_gpio.o(.text.HAL_GPIO_EXTI_Callback), (2 bytes).
    Removing stm32f0xx_hal_gpio.o(.ARM.exidx.text.HAL_GPIO_EXTI_Callback), (8 bytes).
    Removing stm32f0xx_hal_dma.o(.text), (0 bytes).
    Removing stm32f0xx_hal_dma.o(.text.HAL_DMA_Init), (124 bytes).
    Removing stm32f0xx_hal_dma.o(.ARM.exidx.text.HAL_DMA_Init), (8 bytes).
    Removing stm32f0xx_hal_dma.o(.text.HAL_DMA_DeInit), (92 bytes).
    Removing stm32f0xx_hal_dma.o(.ARM.exidx.text.HAL_DMA_DeInit), (8 bytes).
    Removing stm32f0xx_hal_dma.o(.text.HAL_DMA_Start), (104 bytes).
    Removing stm32f0xx_hal_dma.o(.ARM.exidx.text.HAL_DMA_Start), (8 bytes).
    Removing stm32f0xx_hal_dma.o(.text.HAL_DMA_Start_IT), (130 bytes).
    Removing stm32f0xx_hal_dma.o(.ARM.exidx.text.HAL_DMA_Start_IT), (8 bytes).
    Removing stm32f0xx_hal_dma.o(.text.HAL_DMA_Abort), (62 bytes).
    Removing stm32f0xx_hal_dma.o(.ARM.exidx.text.HAL_DMA_Abort), (8 bytes).
    Removing stm32f0xx_hal_dma.o(.text.HAL_DMA_Abort_IT), (66 bytes).
    Removing stm32f0xx_hal_dma.o(.ARM.exidx.text.HAL_DMA_Abort_IT), (8 bytes).
    Removing stm32f0xx_hal_dma.o(.text.HAL_DMA_PollForTransfer), (278 bytes).
    Removing stm32f0xx_hal_dma.o(.ARM.exidx.text.HAL_DMA_PollForTransfer), (8 bytes).
    Removing stm32f0xx_hal_dma.o(.text.HAL_DMA_IRQHandler), (212 bytes).
    Removing stm32f0xx_hal_dma.o(.ARM.exidx.text.HAL_DMA_IRQHandler), (8 bytes).
    Removing stm32f0xx_hal_dma.o(.text.HAL_DMA_RegisterCallback), (70 bytes).
    Removing stm32f0xx_hal_dma.o(.ARM.exidx.text.HAL_DMA_RegisterCallback), (8 bytes).
    Removing stm32f0xx_hal_dma.o(.text.HAL_DMA_UnRegisterCallback), (102 bytes).
    Removing stm32f0xx_hal_dma.o(.ARM.exidx.text.HAL_DMA_UnRegisterCallback), (8 bytes).
    Removing stm32f0xx_hal_dma.o(.text.HAL_DMA_GetState), (6 bytes).
    Removing stm32f0xx_hal_dma.o(.ARM.exidx.text.HAL_DMA_GetState), (8 bytes).
    Removing stm32f0xx_hal_dma.o(.text.HAL_DMA_GetError), (4 bytes).
    Removing stm32f0xx_hal_dma.o(.ARM.exidx.text.HAL_DMA_GetError), (8 bytes).
    Removing stm32f0xx_hal_cortex.o(.text), (0 bytes).
    Removing stm32f0xx_hal_cortex.o(.ARM.exidx.text.HAL_NVIC_SetPriority), (8 bytes).
    Removing stm32f0xx_hal_cortex.o(.text.HAL_NVIC_EnableIRQ), (24 bytes).
    Removing stm32f0xx_hal_cortex.o(.ARM.exidx.text.HAL_NVIC_EnableIRQ), (8 bytes).
    Removing stm32f0xx_hal_cortex.o(.text.HAL_NVIC_DisableIRQ), (32 bytes).
    Removing stm32f0xx_hal_cortex.o(.ARM.exidx.text.HAL_NVIC_DisableIRQ), (8 bytes).
    Removing stm32f0xx_hal_cortex.o(.text.HAL_NVIC_SystemReset), (32 bytes).
    Removing stm32f0xx_hal_cortex.o(.ARM.exidx.text.HAL_NVIC_SystemReset), (8 bytes).
    Removing stm32f0xx_hal_cortex.o(.ARM.exidx.text.HAL_SYSTICK_Config), (8 bytes).
    Removing stm32f0xx_hal_cortex.o(.text.HAL_NVIC_GetPriority), (48 bytes).
    Removing stm32f0xx_hal_cortex.o(.ARM.exidx.text.HAL_NVIC_GetPriority), (8 bytes).
    Removing stm32f0xx_hal_cortex.o(.text.HAL_NVIC_SetPendingIRQ), (24 bytes).
    Removing stm32f0xx_hal_cortex.o(.ARM.exidx.text.HAL_NVIC_SetPendingIRQ), (8 bytes).
    Removing stm32f0xx_hal_cortex.o(.text.HAL_NVIC_GetPendingIRQ), (28 bytes).
    Removing stm32f0xx_hal_cortex.o(.ARM.exidx.text.HAL_NVIC_GetPendingIRQ), (8 bytes).
    Removing stm32f0xx_hal_cortex.o(.text.HAL_NVIC_ClearPendingIRQ), (24 bytes).
    Removing stm32f0xx_hal_cortex.o(.ARM.exidx.text.HAL_NVIC_ClearPendingIRQ), (8 bytes).
    Removing stm32f0xx_hal_cortex.o(.text.HAL_SYSTICK_CLKSourceConfig), (28 bytes).
    Removing stm32f0xx_hal_cortex.o(.ARM.exidx.text.HAL_SYSTICK_CLKSourceConfig), (8 bytes).
    Removing stm32f0xx_hal_cortex.o(.text.HAL_SYSTICK_IRQHandler), (8 bytes).
    Removing stm32f0xx_hal_cortex.o(.ARM.exidx.text.HAL_SYSTICK_IRQHandler), (8 bytes).
    Removing stm32f0xx_hal_cortex.o(.text.HAL_SYSTICK_Callback), (2 bytes).
    Removing stm32f0xx_hal_cortex.o(.ARM.exidx.text.HAL_SYSTICK_Callback), (8 bytes).
    Removing stm32f0xx_hal_pwr.o(.text), (0 bytes).
    Removing stm32f0xx_hal_pwr.o(.text.HAL_PWR_DeInit), (24 bytes).
    Removing stm32f0xx_hal_pwr.o(.ARM.exidx.text.HAL_PWR_DeInit), (8 bytes).
    Removing stm32f0xx_hal_pwr.o(.ARM.exidx.text.HAL_PWR_EnableBkUpAccess), (8 bytes).
    Removing stm32f0xx_hal_pwr.o(.text.HAL_PWR_DisableBkUpAccess), (20 bytes).
    Removing stm32f0xx_hal_pwr.o(.ARM.exidx.text.HAL_PWR_DisableBkUpAccess), (8 bytes).
    Removing stm32f0xx_hal_pwr.o(.text.HAL_PWR_EnableWakeUpPin), (16 bytes).
    Removing stm32f0xx_hal_pwr.o(.ARM.exidx.text.HAL_PWR_EnableWakeUpPin), (8 bytes).
    Removing stm32f0xx_hal_pwr.o(.text.HAL_PWR_DisableWakeUpPin), (16 bytes).
    Removing stm32f0xx_hal_pwr.o(.ARM.exidx.text.HAL_PWR_DisableWakeUpPin), (8 bytes).
    Removing stm32f0xx_hal_pwr.o(.text.HAL_PWR_EnterSLEEPMode), (32 bytes).
    Removing stm32f0xx_hal_pwr.o(.ARM.exidx.text.HAL_PWR_EnterSLEEPMode), (8 bytes).
    Removing stm32f0xx_hal_pwr.o(.text.HAL_PWR_EnterSTOPMode), (60 bytes).
    Removing stm32f0xx_hal_pwr.o(.ARM.exidx.text.HAL_PWR_EnterSTOPMode), (8 bytes).
    Removing stm32f0xx_hal_pwr.o(.text.HAL_PWR_EnterSTANDBYMode), (32 bytes).
    Removing stm32f0xx_hal_pwr.o(.ARM.exidx.text.HAL_PWR_EnterSTANDBYMode), (8 bytes).
    Removing stm32f0xx_hal_pwr.o(.text.HAL_PWR_EnableSleepOnExit), (16 bytes).
    Removing stm32f0xx_hal_pwr.o(.ARM.exidx.text.HAL_PWR_EnableSleepOnExit), (8 bytes).
    Removing stm32f0xx_hal_pwr.o(.text.HAL_PWR_DisableSleepOnExit), (16 bytes).
    Removing stm32f0xx_hal_pwr.o(.ARM.exidx.text.HAL_PWR_DisableSleepOnExit), (8 bytes).
    Removing stm32f0xx_hal_pwr.o(.text.HAL_PWR_EnableSEVOnPend), (16 bytes).
    Removing stm32f0xx_hal_pwr.o(.ARM.exidx.text.HAL_PWR_EnableSEVOnPend), (8 bytes).
    Removing stm32f0xx_hal_pwr.o(.text.HAL_PWR_DisableSEVOnPend), (16 bytes).
    Removing stm32f0xx_hal_pwr.o(.ARM.exidx.text.HAL_PWR_DisableSEVOnPend), (8 bytes).
    Removing stm32f0xx_hal_pwr_ex.o(.text), (0 bytes).
    Removing stm32f0xx_hal_flash.o(.text), (0 bytes).
    Removing stm32f0xx_hal_flash.o(.text.HAL_FLASH_Program), (340 bytes).
    Removing stm32f0xx_hal_flash.o(.ARM.exidx.text.HAL_FLASH_Program), (8 bytes).
    Removing stm32f0xx_hal_flash.o(.text.FLASH_WaitForLastOperation), (172 bytes).
    Removing stm32f0xx_hal_flash.o(.ARM.exidx.text.FLASH_WaitForLastOperation), (8 bytes).
    Removing stm32f0xx_hal_flash.o(.text.HAL_FLASH_Program_IT), (92 bytes).
    Removing stm32f0xx_hal_flash.o(.ARM.exidx.text.HAL_FLASH_Program_IT), (8 bytes).
    Removing stm32f0xx_hal_flash.o(.text.HAL_FLASH_IRQHandler), (348 bytes).
    Removing stm32f0xx_hal_flash.o(.ARM.exidx.text.HAL_FLASH_IRQHandler), (8 bytes).
    Removing stm32f0xx_hal_flash.o(.text.HAL_FLASH_OperationErrorCallback), (2 bytes).
    Removing stm32f0xx_hal_flash.o(.ARM.exidx.text.HAL_FLASH_OperationErrorCallback), (8 bytes).
    Removing stm32f0xx_hal_flash.o(.text.HAL_FLASH_EndOfOperationCallback), (2 bytes).
    Removing stm32f0xx_hal_flash.o(.ARM.exidx.text.HAL_FLASH_EndOfOperationCallback), (8 bytes).
    Removing stm32f0xx_hal_flash.o(.text.HAL_FLASH_Unlock), (40 bytes).
    Removing stm32f0xx_hal_flash.o(.ARM.exidx.text.HAL_FLASH_Unlock), (8 bytes).
    Removing stm32f0xx_hal_flash.o(.text.HAL_FLASH_Lock), (20 bytes).
    Removing stm32f0xx_hal_flash.o(.ARM.exidx.text.HAL_FLASH_Lock), (8 bytes).
    Removing stm32f0xx_hal_flash.o(.text.HAL_FLASH_OB_Unlock), (36 bytes).
    Removing stm32f0xx_hal_flash.o(.ARM.exidx.text.HAL_FLASH_OB_Unlock), (8 bytes).
    Removing stm32f0xx_hal_flash.o(.text.HAL_FLASH_OB_Lock), (20 bytes).
    Removing stm32f0xx_hal_flash.o(.ARM.exidx.text.HAL_FLASH_OB_Lock), (8 bytes).
    Removing stm32f0xx_hal_flash.o(.text.HAL_FLASH_OB_Launch), (152 bytes).
    Removing stm32f0xx_hal_flash.o(.ARM.exidx.text.HAL_FLASH_OB_Launch), (8 bytes).
    Removing stm32f0xx_hal_flash.o(.text.HAL_FLASH_GetError), (12 bytes).
    Removing stm32f0xx_hal_flash.o(.ARM.exidx.text.HAL_FLASH_GetError), (8 bytes).
    Removing stm32f0xx_hal_flash.o(.bss.pFlash), (32 bytes).
    Removing stm32f0xx_hal_flash_ex.o(.text), (0 bytes).
    Removing stm32f0xx_hal_flash_ex.o(.text.HAL_FLASHEx_Erase), (208 bytes).
    Removing stm32f0xx_hal_flash_ex.o(.ARM.exidx.text.HAL_FLASHEx_Erase), (8 bytes).
    Removing stm32f0xx_hal_flash_ex.o(.text.FLASH_PageErase), (36 bytes).
    Removing stm32f0xx_hal_flash_ex.o(.ARM.exidx.text.FLASH_PageErase), (8 bytes).
    Removing stm32f0xx_hal_flash_ex.o(.text.HAL_FLASHEx_Erase_IT), (112 bytes).
    Removing stm32f0xx_hal_flash_ex.o(.ARM.exidx.text.HAL_FLASHEx_Erase_IT), (8 bytes).
    Removing stm32f0xx_hal_flash_ex.o(.text.HAL_FLASHEx_OBErase), (184 bytes).
    Removing stm32f0xx_hal_flash_ex.o(.ARM.exidx.text.HAL_FLASHEx_OBErase), (8 bytes).
    Removing stm32f0xx_hal_flash_ex.o(.text.HAL_FLASHEx_OBProgram), (520 bytes).
    Removing stm32f0xx_hal_flash_ex.o(.ARM.exidx.text.HAL_FLASHEx_OBProgram), (8 bytes).
    Removing stm32f0xx_hal_flash_ex.o(.text.HAL_FLASHEx_OBGetConfig), (56 bytes).
    Removing stm32f0xx_hal_flash_ex.o(.ARM.exidx.text.HAL_FLASHEx_OBGetConfig), (8 bytes).
    Removing stm32f0xx_hal_flash_ex.o(.text.HAL_FLASHEx_OBGetUserData), (28 bytes).
    Removing stm32f0xx_hal_flash_ex.o(.ARM.exidx.text.HAL_FLASHEx_OBGetUserData), (8 bytes).
    Removing stm32f0xx_hal_exti.o(.text), (0 bytes).
    Removing stm32f0xx_hal_exti.o(.text.HAL_EXTI_SetConfigLine), (160 bytes).
    Removing stm32f0xx_hal_exti.o(.ARM.exidx.text.HAL_EXTI_SetConfigLine), (8 bytes).
    Removing stm32f0xx_hal_exti.o(.text.HAL_EXTI_GetConfigLine), (128 bytes).
    Removing stm32f0xx_hal_exti.o(.ARM.exidx.text.HAL_EXTI_GetConfigLine), (8 bytes).
    Removing stm32f0xx_hal_exti.o(.text.HAL_EXTI_ClearConfigLine), (96 bytes).
    Removing stm32f0xx_hal_exti.o(.ARM.exidx.text.HAL_EXTI_ClearConfigLine), (8 bytes).
    Removing stm32f0xx_hal_exti.o(.text.HAL_EXTI_RegisterCallback), (14 bytes).
    Removing stm32f0xx_hal_exti.o(.ARM.exidx.text.HAL_EXTI_RegisterCallback), (8 bytes).
    Removing stm32f0xx_hal_exti.o(.text.HAL_EXTI_GetHandle), (14 bytes).
    Removing stm32f0xx_hal_exti.o(.ARM.exidx.text.HAL_EXTI_GetHandle), (8 bytes).
    Removing stm32f0xx_hal_exti.o(.text.HAL_EXTI_IRQHandler), (36 bytes).
    Removing stm32f0xx_hal_exti.o(.ARM.exidx.text.HAL_EXTI_IRQHandler), (8 bytes).
    Removing stm32f0xx_hal_exti.o(.text.HAL_EXTI_GetPending), (24 bytes).
    Removing stm32f0xx_hal_exti.o(.ARM.exidx.text.HAL_EXTI_GetPending), (8 bytes).
    Removing stm32f0xx_hal_exti.o(.text.HAL_EXTI_ClearPending), (20 bytes).
    Removing stm32f0xx_hal_exti.o(.ARM.exidx.text.HAL_EXTI_ClearPending), (8 bytes).
    Removing stm32f0xx_hal_exti.o(.text.HAL_EXTI_GenerateSWI), (20 bytes).
    Removing stm32f0xx_hal_exti.o(.ARM.exidx.text.HAL_EXTI_GenerateSWI), (8 bytes).
    Removing stm32f0xx_hal_rtc.o(.text), (0 bytes).
    Removing stm32f0xx_hal_rtc.o(.ARM.exidx.text.HAL_RTC_Init), (8 bytes).
    Removing stm32f0xx_hal_rtc.o(.text.HAL_RTC_MspInit), (2 bytes).
    Removing stm32f0xx_hal_rtc.o(.ARM.exidx.text.HAL_RTC_MspInit), (8 bytes).
    Removing stm32f0xx_hal_rtc.o(.text.RTC_EnterInitMode), (84 bytes).
    Removing stm32f0xx_hal_rtc.o(.ARM.exidx.text.RTC_EnterInitMode), (8 bytes).
    Removing stm32f0xx_hal_rtc.o(.text.RTC_ExitInitMode), (76 bytes).
    Removing stm32f0xx_hal_rtc.o(.ARM.exidx.text.RTC_ExitInitMode), (8 bytes).
    Removing stm32f0xx_hal_rtc.o(.text.HAL_RTC_DeInit), (208 bytes).
    Removing stm32f0xx_hal_rtc.o(.ARM.exidx.text.HAL_RTC_DeInit), (8 bytes).
    Removing stm32f0xx_hal_rtc.o(.text.HAL_RTC_MspDeInit), (2 bytes).
    Removing stm32f0xx_hal_rtc.o(.ARM.exidx.text.HAL_RTC_MspDeInit), (8 bytes).
    Removing stm32f0xx_hal_rtc.o(.ARM.exidx.text.HAL_RTC_SetTime), (8 bytes).
    Removing stm32f0xx_hal_rtc.o(.text.RTC_ByteToBcd2), (38 bytes).
    Removing stm32f0xx_hal_rtc.o(.ARM.exidx.text.RTC_ByteToBcd2), (8 bytes).
    Removing stm32f0xx_hal_rtc.o(.ARM.exidx.text.HAL_RTC_GetTime), (8 bytes).
    Removing stm32f0xx_hal_rtc.o(.text.RTC_Bcd2ToByte), (16 bytes).
    Removing stm32f0xx_hal_rtc.o(.ARM.exidx.text.RTC_Bcd2ToByte), (8 bytes).
    Removing stm32f0xx_hal_rtc.o(.ARM.exidx.text.HAL_RTC_SetDate), (8 bytes).
    Removing stm32f0xx_hal_rtc.o(.ARM.exidx.text.HAL_RTC_GetDate), (8 bytes).
    Removing stm32f0xx_hal_rtc.o(.text.HAL_RTC_SetAlarm), (376 bytes).
    Removing stm32f0xx_hal_rtc.o(.ARM.exidx.text.HAL_RTC_SetAlarm), (8 bytes).
    Removing stm32f0xx_hal_rtc.o(.text.HAL_RTC_SetAlarm_IT), (452 bytes).
    Removing stm32f0xx_hal_rtc.o(.ARM.exidx.text.HAL_RTC_SetAlarm_IT), (8 bytes).
    Removing stm32f0xx_hal_rtc.o(.text.HAL_RTC_DeactivateAlarm), (112 bytes).
    Removing stm32f0xx_hal_rtc.o(.ARM.exidx.text.HAL_RTC_DeactivateAlarm), (8 bytes).
    Removing stm32f0xx_hal_rtc.o(.text.HAL_RTC_GetAlarm), (164 bytes).
    Removing stm32f0xx_hal_rtc.o(.ARM.exidx.text.HAL_RTC_GetAlarm), (8 bytes).
    Removing stm32f0xx_hal_rtc.o(.text.HAL_RTC_AlarmIRQHandler), (56 bytes).
    Removing stm32f0xx_hal_rtc.o(.ARM.exidx.text.HAL_RTC_AlarmIRQHandler), (8 bytes).
    Removing stm32f0xx_hal_rtc.o(.text.HAL_RTC_AlarmAEventCallback), (2 bytes).
    Removing stm32f0xx_hal_rtc.o(.ARM.exidx.text.HAL_RTC_AlarmAEventCallback), (8 bytes).
    Removing stm32f0xx_hal_rtc.o(.text.HAL_RTC_PollForAlarmAEvent), (128 bytes).
    Removing stm32f0xx_hal_rtc.o(.ARM.exidx.text.HAL_RTC_PollForAlarmAEvent), (8 bytes).
    Removing stm32f0xx_hal_rtc.o(.text.HAL_RTC_WaitForSynchro), (52 bytes).
    Removing stm32f0xx_hal_rtc.o(.ARM.exidx.text.HAL_RTC_WaitForSynchro), (8 bytes).
    Removing stm32f0xx_hal_rtc.o(.text.HAL_RTC_DST_Add1Hour), (26 bytes).
    Removing stm32f0xx_hal_rtc.o(.ARM.exidx.text.HAL_RTC_DST_Add1Hour), (8 bytes).
    Removing stm32f0xx_hal_rtc.o(.text.HAL_RTC_DST_Sub1Hour), (26 bytes).
    Removing stm32f0xx_hal_rtc.o(.ARM.exidx.text.HAL_RTC_DST_Sub1Hour), (8 bytes).
    Removing stm32f0xx_hal_rtc.o(.text.HAL_RTC_DST_SetStoreOperation), (26 bytes).
    Removing stm32f0xx_hal_rtc.o(.ARM.exidx.text.HAL_RTC_DST_SetStoreOperation), (8 bytes).
    Removing stm32f0xx_hal_rtc.o(.text.HAL_RTC_DST_ClearStoreOperation), (26 bytes).
    Removing stm32f0xx_hal_rtc.o(.ARM.exidx.text.HAL_RTC_DST_ClearStoreOperation), (8 bytes).
    Removing stm32f0xx_hal_rtc.o(.text.HAL_RTC_DST_ReadStoreOperation), (12 bytes).
    Removing stm32f0xx_hal_rtc.o(.ARM.exidx.text.HAL_RTC_DST_ReadStoreOperation), (8 bytes).
    Removing stm32f0xx_hal_rtc.o(.text.HAL_RTC_GetState), (4 bytes).
    Removing stm32f0xx_hal_rtc.o(.ARM.exidx.text.HAL_RTC_GetState), (8 bytes).
    Removing stm32f0xx_hal_rtc_ex.o(.text), (0 bytes).
    Removing stm32f0xx_hal_rtc_ex.o(.text.HAL_RTCEx_SetTimeStamp), (92 bytes).
    Removing stm32f0xx_hal_rtc_ex.o(.ARM.exidx.text.HAL_RTCEx_SetTimeStamp), (8 bytes).
    Removing stm32f0xx_hal_rtc_ex.o(.text.HAL_RTCEx_SetTimeStamp_IT), (120 bytes).
    Removing stm32f0xx_hal_rtc_ex.o(.ARM.exidx.text.HAL_RTCEx_SetTimeStamp_IT), (8 bytes).
    Removing stm32f0xx_hal_rtc_ex.o(.text.HAL_RTCEx_DeactivateTimeStamp), (64 bytes).
    Removing stm32f0xx_hal_rtc_ex.o(.ARM.exidx.text.HAL_RTCEx_DeactivateTimeStamp), (8 bytes).
    Removing stm32f0xx_hal_rtc_ex.o(.text.HAL_RTCEx_GetTimeStamp), (144 bytes).
    Removing stm32f0xx_hal_rtc_ex.o(.ARM.exidx.text.HAL_RTCEx_GetTimeStamp), (8 bytes).
    Removing stm32f0xx_hal_rtc_ex.o(.text.HAL_RTCEx_SetTamper), (84 bytes).
    Removing stm32f0xx_hal_rtc_ex.o(.ARM.exidx.text.HAL_RTCEx_SetTamper), (8 bytes).
    Removing stm32f0xx_hal_rtc_ex.o(.text.HAL_RTCEx_SetTamper_IT), (104 bytes).
    Removing stm32f0xx_hal_rtc_ex.o(.ARM.exidx.text.HAL_RTCEx_SetTamper_IT), (8 bytes).
    Removing stm32f0xx_hal_rtc_ex.o(.text.HAL_RTCEx_DeactivateTamper), (34 bytes).
    Removing stm32f0xx_hal_rtc_ex.o(.ARM.exidx.text.HAL_RTCEx_DeactivateTamper), (8 bytes).
    Removing stm32f0xx_hal_rtc_ex.o(.text.HAL_RTCEx_TamperTimeStampIRQHandler), (128 bytes).
    Removing stm32f0xx_hal_rtc_ex.o(.ARM.exidx.text.HAL_RTCEx_TamperTimeStampIRQHandler), (8 bytes).
    Removing stm32f0xx_hal_rtc_ex.o(.text.HAL_RTCEx_TimeStampEventCallback), (2 bytes).
    Removing stm32f0xx_hal_rtc_ex.o(.ARM.exidx.text.HAL_RTCEx_TimeStampEventCallback), (8 bytes).
    Removing stm32f0xx_hal_rtc_ex.o(.text.HAL_RTCEx_Tamper1EventCallback), (2 bytes).
    Removing stm32f0xx_hal_rtc_ex.o(.ARM.exidx.text.HAL_RTCEx_Tamper1EventCallback), (8 bytes).
    Removing stm32f0xx_hal_rtc_ex.o(.text.HAL_RTCEx_Tamper2EventCallback), (2 bytes).
    Removing stm32f0xx_hal_rtc_ex.o(.ARM.exidx.text.HAL_RTCEx_Tamper2EventCallback), (8 bytes).
    Removing stm32f0xx_hal_rtc_ex.o(.text.HAL_RTCEx_PollForTimeStampEvent), (184 bytes).
    Removing stm32f0xx_hal_rtc_ex.o(.ARM.exidx.text.HAL_RTCEx_PollForTimeStampEvent), (8 bytes).
    Removing stm32f0xx_hal_rtc_ex.o(.text.HAL_RTCEx_PollForTamper1Event), (128 bytes).
    Removing stm32f0xx_hal_rtc_ex.o(.ARM.exidx.text.HAL_RTCEx_PollForTamper1Event), (8 bytes).
    Removing stm32f0xx_hal_rtc_ex.o(.text.HAL_RTCEx_PollForTamper2Event), (128 bytes).
    Removing stm32f0xx_hal_rtc_ex.o(.ARM.exidx.text.HAL_RTCEx_PollForTamper2Event), (8 bytes).
    Removing stm32f0xx_hal_rtc_ex.o(.text.HAL_RTCEx_SetWakeUpTimer), (184 bytes).
    Removing stm32f0xx_hal_rtc_ex.o(.ARM.exidx.text.HAL_RTCEx_SetWakeUpTimer), (8 bytes).
    Removing stm32f0xx_hal_rtc_ex.o(.text.HAL_RTCEx_SetWakeUpTimer_IT), (332 bytes).
    Removing stm32f0xx_hal_rtc_ex.o(.ARM.exidx.text.HAL_RTCEx_SetWakeUpTimer_IT), (8 bytes).
    Removing stm32f0xx_hal_rtc_ex.o(.text.HAL_RTCEx_DeactivateWakeUpTimer), (112 bytes).
    Removing stm32f0xx_hal_rtc_ex.o(.ARM.exidx.text.HAL_RTCEx_DeactivateWakeUpTimer), (8 bytes).
    Removing stm32f0xx_hal_rtc_ex.o(.text.HAL_RTCEx_GetWakeUpTimer), (8 bytes).
    Removing stm32f0xx_hal_rtc_ex.o(.ARM.exidx.text.HAL_RTCEx_GetWakeUpTimer), (8 bytes).
    Removing stm32f0xx_hal_rtc_ex.o(.text.HAL_RTCEx_WakeUpTimerIRQHandler), (56 bytes).
    Removing stm32f0xx_hal_rtc_ex.o(.ARM.exidx.text.HAL_RTCEx_WakeUpTimerIRQHandler), (8 bytes).
    Removing stm32f0xx_hal_rtc_ex.o(.text.HAL_RTCEx_WakeUpTimerEventCallback), (2 bytes).
    Removing stm32f0xx_hal_rtc_ex.o(.ARM.exidx.text.HAL_RTCEx_WakeUpTimerEventCallback), (8 bytes).
    Removing stm32f0xx_hal_rtc_ex.o(.text.HAL_RTCEx_PollForWakeUpTimerEvent), (128 bytes).
    Removing stm32f0xx_hal_rtc_ex.o(.ARM.exidx.text.HAL_RTCEx_PollForWakeUpTimerEvent), (8 bytes).
    Removing stm32f0xx_hal_rtc_ex.o(.text.HAL_RTCEx_SetSmoothCalib), (124 bytes).
    Removing stm32f0xx_hal_rtc_ex.o(.ARM.exidx.text.HAL_RTCEx_SetSmoothCalib), (8 bytes).
    Removing stm32f0xx_hal_rtc_ex.o(.text.HAL_RTCEx_SetSynchroShift), (136 bytes).
    Removing stm32f0xx_hal_rtc_ex.o(.ARM.exidx.text.HAL_RTCEx_SetSynchroShift), (8 bytes).
    Removing stm32f0xx_hal_rtc_ex.o(.text.HAL_RTCEx_SetCalibrationOutPut), (64 bytes).
    Removing stm32f0xx_hal_rtc_ex.o(.ARM.exidx.text.HAL_RTCEx_SetCalibrationOutPut), (8 bytes).
    Removing stm32f0xx_hal_rtc_ex.o(.text.HAL_RTCEx_DeactivateCalibrationOutPut), (50 bytes).
    Removing stm32f0xx_hal_rtc_ex.o(.ARM.exidx.text.HAL_RTCEx_DeactivateCalibrationOutPut), (8 bytes).
    Removing stm32f0xx_hal_rtc_ex.o(.text.HAL_RTCEx_SetRefClock), (78 bytes).
    Removing stm32f0xx_hal_rtc_ex.o(.ARM.exidx.text.HAL_RTCEx_SetRefClock), (8 bytes).
    Removing stm32f0xx_hal_rtc_ex.o(.text.HAL_RTCEx_DeactivateRefClock), (78 bytes).
    Removing stm32f0xx_hal_rtc_ex.o(.ARM.exidx.text.HAL_RTCEx_DeactivateRefClock), (8 bytes).
    Removing stm32f0xx_hal_rtc_ex.o(.text.HAL_RTCEx_EnableBypassShadow), (48 bytes).
    Removing stm32f0xx_hal_rtc_ex.o(.ARM.exidx.text.HAL_RTCEx_EnableBypassShadow), (8 bytes).
    Removing stm32f0xx_hal_rtc_ex.o(.text.HAL_RTCEx_DisableBypassShadow), (48 bytes).
    Removing stm32f0xx_hal_rtc_ex.o(.ARM.exidx.text.HAL_RTCEx_DisableBypassShadow), (8 bytes).
    Removing stm32f0xx_hal_tim.o(.text), (0 bytes).
    Removing stm32f0xx_hal_tim_ex.o(.text), (0 bytes).
    Removing system_stm32f0xx.o(.text), (0 bytes).
    Removing system_stm32f0xx.o(.ARM.exidx.text.SystemInit), (8 bytes).
    Removing system_stm32f0xx.o(.text.SystemCoreClockUpdate), (80 bytes).
    Removing system_stm32f0xx.o(.ARM.exidx.text.SystemCoreClockUpdate), (8 bytes).
    Removing system_stm32f0xx.o(.rodata.APBPrescTable), (8 bytes).

523 unused section(s) (total 26868 bytes) removed from the image.

==============================================================================

Image Symbol Table

    Local Symbols

    Symbol Name                              Value     Ov Type        Size  Object(Section)

    ../clib/../cmprslib/zerorunl2.c          0x00000000   Number         0  __dczerorl2.o ABSOLUTE
    ../clib/angel/boardlib.s                 0x00000000   Number         0  boardinit1.o ABSOLUTE
    ../clib/angel/boardlib.s                 0x00000000   Number         0  boardinit2.o ABSOLUTE
    ../clib/angel/boardlib.s                 0x00000000   Number         0  boardinit3.o ABSOLUTE
    ../clib/angel/boardlib.s                 0x00000000   Number         0  boardshut.o ABSOLUTE
    ../clib/angel/handlers.s                 0x00000000   Number         0  __scatter_zi.o ABSOLUTE
    ../clib/angel/kernel.s                   0x00000000   Number         0  __rtentry.o ABSOLUTE
    ../clib/angel/kernel.s                   0x00000000   Number         0  __rtentry2.o ABSOLUTE
    ../clib/angel/kernel.s                   0x00000000   Number         0  __rtentry4.o ABSOLUTE
    ../clib/angel/kernel.s                   0x00000000   Number         0  rtexit.o ABSOLUTE
    ../clib/angel/kernel.s                   0x00000000   Number         0  rtexit2.o ABSOLUTE
    ../clib/angel/rt.s                       0x00000000   Number         0  aeabi_idiv0.o ABSOLUTE
    ../clib/angel/rt.s                       0x00000000   Number         0  aeabi_idiv0_sigfpe.o ABSOLUTE
    ../clib/angel/rt.s                       0x00000000   Number         0  rt_div0.o ABSOLUTE
    ../clib/angel/rt.s                       0x00000000   Number         0  rt_locale.o ABSOLUTE
    ../clib/angel/rt.s                       0x00000000   Number         0  rt_locale_intlibspace.o ABSOLUTE
    ../clib/angel/rt.s                       0x00000000   Number         0  rt_errno_addr.o ABSOLUTE
    ../clib/angel/rt.s                       0x00000000   Number         0  rt_errno_addr_intlibspace.o ABSOLUTE
    ../clib/angel/rt.s                       0x00000000   Number         0  rt_raise.o ABSOLUTE
    ../clib/angel/scatterp.s                 0x00000000   Number         0  __scatter.o ABSOLUTE
    ../clib/angel/startup.s                  0x00000000   Number         0  __main.o ABSOLUTE
    ../clib/angel/sys.s                      0x00000000   Number         0  libspace.o ABSOLUTE
    ../clib/angel/sys.s                      0x00000000   Number         0  sys_stackheap_outer.o ABSOLUTE
    ../clib/angel/sys.s                      0x00000000   Number         0  tempstk.o ABSOLUTE
    ../clib/angel/sys.s                      0x00000000   Number         0  use_no_semi.o ABSOLUTE
    ../clib/angel/sys.s                      0x00000000   Number         0  indicate_semi.o ABSOLUTE
    ../clib/angel/sysapp.c                   0x00000000   Number         0  sys_exit.o ABSOLUTE
    ../clib/angel/sysapp.c                   0x00000000   Number         0  sys_exit_hlt.o ABSOLUTE
    ../clib/angel/sysapp.c                   0x00000000   Number         0  sys_wrch.o ABSOLUTE
    ../clib/angel/sysapp.c                   0x00000000   Number         0  sys_command.o ABSOLUTE
    ../clib/angel/sysapp.c                   0x00000000   Number         0  sys_wrch_hlt.o ABSOLUTE
    ../clib/angel/sysapp.c                   0x00000000   Number         0  sys_command_hlt.o ABSOLUTE
    ../clib/armsys.c                         0x00000000   Number         0  argv_veneer.o ABSOLUTE
    ../clib/armsys.c                         0x00000000   Number         0  _get_argv_nomalloc.o ABSOLUTE
    ../clib/armsys.c                         0x00000000   Number         0  no_argv.o ABSOLUTE
    ../clib/bigflt.c                         0x00000000   Number         0  bigflt0.o ABSOLUTE
    ../clib/btod.c                           0x00000000   Number         0  btod.o ABSOLUTE
    ../clib/btod_accurate.c                  0x00000000   Number         0  btod_accurate.o ABSOLUTE
    ../clib/btod_accurate.c                  0x00000000   Number         0  btod_accurate_common.o ABSOLUTE
    ../clib/division.c                       0x00000000   Number         0  lludiv10.o ABSOLUTE
    ../clib/division.c                       0x00000000   Number         0  rtudiv10.o ABSOLUTE
    ../clib/division.s                       0x00000000   Number         0  aeabi_sdivfast.o ABSOLUTE
    ../clib/division.s                       0x00000000   Number         0  aeabi_sdivfast_div0.o ABSOLUTE
    ../clib/fenv.c                           0x00000000   Number         0  _rserrno.o ABSOLUTE
    ../clib/heapalloc.c                      0x00000000   Number         0  hrguard.o ABSOLUTE
    ../clib/heapaux.c                        0x00000000   Number         0  heapauxi.o ABSOLUTE
    ../clib/libinit.s                        0x00000000   Number         0  libinit.o ABSOLUTE
    ../clib/libinit.s                        0x00000000   Number         0  libinit2.o ABSOLUTE
    ../clib/libinit.s                        0x00000000   Number         0  libshutdown.o ABSOLUTE
    ../clib/libinit.s                        0x00000000   Number         0  libshutdown2.o ABSOLUTE
    ../clib/locale.s                         0x00000000   Number         0  lc_numeric_c.o ABSOLUTE
    ../clib/longlong.c                       0x00000000   Number         0  llushr.o ABSOLUTE
    ../clib/memcpset.s                       0x00000000   Number         0  strcmpv6m.o ABSOLUTE
    ../clib/misc.s                           0x00000000   Number         0  printf_stubs.o ABSOLUTE
    ../clib/printf.c                         0x00000000   Number         0  __2sprintf.o ABSOLUTE
    ../clib/printf.c                         0x00000000   Number         0  noretval__2sprintf.o ABSOLUTE
    ../clib/printf.c                         0x00000000   Number         0  __printf.o ABSOLUTE
    ../clib/printf.c                         0x00000000   Number         0  _printf_pad.o ABSOLUTE
    ../clib/printf.c                         0x00000000   Number         0  _printf_str.o ABSOLUTE
    ../clib/printf.c                         0x00000000   Number         0  _printf_hex_ll.o ABSOLUTE
    ../clib/printf.c                         0x00000000   Number         0  _printf_hex_int.o ABSOLUTE
    ../clib/printf.c                         0x00000000   Number         0  _printf_hex_int_ll.o ABSOLUTE
    ../clib/printf.c                         0x00000000   Number         0  _printf_hex_ptr.o ABSOLUTE
    ../clib/printf.c                         0x00000000   Number         0  _printf_hex_int_ptr.o ABSOLUTE
    ../clib/printf.c                         0x00000000   Number         0  _printf_hex_ll_ptr.o ABSOLUTE
    ../clib/printf.c                         0x00000000   Number         0  _printf_hex_int_ll_ptr.o ABSOLUTE
    ../clib/printf.c                         0x00000000   Number         0  __printf_flags.o ABSOLUTE
    ../clib/printf.c                         0x00000000   Number         0  __printf_ss.o ABSOLUTE
    ../clib/printf.c                         0x00000000   Number         0  __printf_flags_ss.o ABSOLUTE
    ../clib/printf.c                         0x00000000   Number         0  __printf_wp.o ABSOLUTE
    ../clib/printf.c                         0x00000000   Number         0  __printf_flags_wp.o ABSOLUTE
    ../clib/printf.c                         0x00000000   Number         0  __printf_ss_wp.o ABSOLUTE
    ../clib/printf.c                         0x00000000   Number         0  __printf_flags_ss_wp.o ABSOLUTE
    ../clib/printf.c                         0x00000000   Number         0  _printf_intcommon.o ABSOLUTE
    ../clib/printf.c                         0x00000000   Number         0  _printf_fp_dec.o ABSOLUTE
    ../clib/printf.c                         0x00000000   Number         0  _printf_fp_dec_accurate.o ABSOLUTE
    ../clib/printf.c                         0x00000000   Number         0  _printf_char_common.o ABSOLUTE
    ../clib/printf.c                         0x00000000   Number         0  _sputc.o ABSOLUTE
    ../clib/printf.c                         0x00000000   Number         0  _printf_char.o ABSOLUTE
    ../clib/printf.c                         0x00000000   Number         0  _printf_fp_infnan.o ABSOLUTE
    ../clib/printf.c                         0x00000000   Number         0  __printf_nopercent.o ABSOLUTE
    ../clib/printf_percent.s                 0x00000000   Number         0  _printf_c.o ABSOLUTE
    ../clib/printf_percent.s                 0x00000000   Number         0  _printf_s.o ABSOLUTE
    ../clib/printf_percent.s                 0x00000000   Number         0  _printf_x.o ABSOLUTE
    ../clib/printf_percent.s                 0x00000000   Number         0  _printf_f.o ABSOLUTE
    ../clib/printf_percent.s                 0x00000000   Number         0  _printf_percent.o ABSOLUTE
    ../clib/printf_percent.s                 0x00000000   Number         0  _printf_percent_end.o ABSOLUTE
    ../clib/signal.c                         0x00000000   Number         0  defsig_fpe_outer.o ABSOLUTE
    ../clib/signal.c                         0x00000000   Number         0  defsig_fpe_formal.o ABSOLUTE
    ../clib/signal.c                         0x00000000   Number         0  defsig_exit.o ABSOLUTE
    ../clib/signal.c                         0x00000000   Number         0  defsig_fpe_inner.o ABSOLUTE
    ../clib/signal.c                         0x00000000   Number         0  __raise.o ABSOLUTE
    ../clib/signal.c                         0x00000000   Number         0  defsig_general.o ABSOLUTE
    ../clib/signal.c                         0x00000000   Number         0  defsig_rtmem_outer.o ABSOLUTE
    ../clib/signal.c                         0x00000000   Number         0  defsig_rtmem_formal.o ABSOLUTE
    ../clib/signal.c                         0x00000000   Number         0  defsig_abrt_inner.o ABSOLUTE
    ../clib/signal.c                         0x00000000   Number         0  defsig_rtred_inner.o ABSOLUTE
    ../clib/signal.c                         0x00000000   Number         0  defsig_rtmem_inner.o ABSOLUTE
    ../clib/signal.c                         0x00000000   Number         0  defsig_stak_inner.o ABSOLUTE
    ../clib/signal.c                         0x00000000   Number         0  defsig_pvfn_inner.o ABSOLUTE
    ../clib/signal.c                         0x00000000   Number         0  defsig_cppl_inner.o ABSOLUTE
    ../clib/signal.c                         0x00000000   Number         0  defsig_segv_inner.o ABSOLUTE
    ../clib/signal.c                         0x00000000   Number         0  defsig_other.o ABSOLUTE
    ../clib/signal.s                         0x00000000   Number         0  defsig.o ABSOLUTE
    ../clib/stdlib.c                         0x00000000   Number         0  exit.o ABSOLUTE
    ../fplib/cfplib/cmpret.c                 0x00000000   Number         0  cmpret.o ABSOLUTE
    ../fplib/cfplib/d2f.c                    0x00000000   Number         0  d2f.o ABSOLUTE
    ../fplib/cfplib/daddsub.c                0x00000000   Number         0  daddsub.o ABSOLUTE
    ../fplib/cfplib/dcmpin.c                 0x00000000   Number         0  dcmpin.o ABSOLUTE
    ../fplib/cfplib/ddiv.c                   0x00000000   Number         0  ddiv.o ABSOLUTE
    ../fplib/cfplib/dmul.c                   0x00000000   Number         0  dmul.o ABSOLUTE
    ../fplib/cfplib/dsqrt.c                  0x00000000   Number         0  dsqrt.o ABSOLUTE
    ../fplib/cfplib/f2d.c                    0x00000000   Number         0  f2d.o ABSOLUTE
    ../fplib/cfplib/ffix.c                   0x00000000   Number         0  dfixi.o ABSOLUTE
    ../fplib/cfplib/fflt.c                   0x00000000   Number         0  dflti.o ABSOLUTE
    ../fplib/cfplib/fflt.c                   0x00000000   Number         0  fflti.o ABSOLUTE
    ../fplib/cfplib/fpinit.c                 0x00000000   Number         0  fpinit.o ABSOLUTE
    ../fplib/cfplib/ieee_status.c            0x00000000   Number         0  ieee_status.o ABSOLUTE
    ../fplib/cfplib/nan2.c                   0x00000000   Number         0  dnan2.o ABSOLUTE
    ../fplib/cfplib/retnan.c                 0x00000000   Number         0  retnan.o ABSOLUTE
    ../fplib/cfplib/scalbn.c                 0x00000000   Number         0  dscalbn.o ABSOLUTE
    ../fplib/drleqf6m.s                      0x00000000   Number         0  drlef.o ABSOLUTE
    ../fplib/faddsub6m.s                     0x00000000   Number         0  faddsub.o ABSOLUTE
    ../fplib/fmul6m.s                        0x00000000   Number         0  fmul.o ABSOLUTE
    ../fplib/printf1.s                       0x00000000   Number         0  printf1.o ABSOLUTE
    ../fplib/usenofp.s                       0x00000000   Number         0  usenofp.o ABSOLUTE
    ../mathlib/dunder.c                      0x00000000   Number         0  dunder.o ABSOLUTE
    ../mathlib/fpclassify.c                  0x00000000   Number         0  fpclassify.o ABSOLUTE
    ../mathlib/poly.c                        0x00000000   Number         0  poly.o ABSOLUTE
    ../mathlib/pow.c                         0x00000000   Number         0  pow.o ABSOLUTE
    ../mathlib/qnan.c                        0x00000000   Number         0  qnan.o ABSOLUTE
    ../mathlib/sqrt.c                        0x00000000   Number         0  sqrt.o ABSOLUTE
    BMP280+AHT20.c                           0x00000000   Number         0  bmp280+aht20.o ABSOLUTE
    dc.s                                     0x00000000   Number         0  dc.o ABSOLUTE
    main.c                                   0x00000000   Number         0  main.o ABSOLUTE
    ssd1306.c                                0x00000000   Number         0  ssd1306.o ABSOLUTE
    startup_stm32f030xc.s                    0x00000000   Number         0  startup_stm32f030xc.o ABSOLUTE
    stm32f0xx_hal.c                          0x00000000   Number         0  stm32f0xx_hal.o ABSOLUTE
    stm32f0xx_hal_cortex.c                   0x00000000   Number         0  stm32f0xx_hal_cortex.o ABSOLUTE
    stm32f0xx_hal_dma.c                      0x00000000   Number         0  stm32f0xx_hal_dma.o ABSOLUTE
    stm32f0xx_hal_exti.c                     0x00000000   Number         0  stm32f0xx_hal_exti.o ABSOLUTE
    stm32f0xx_hal_flash.c                    0x00000000   Number         0  stm32f0xx_hal_flash.o ABSOLUTE
    stm32f0xx_hal_flash_ex.c                 0x00000000   Number         0  stm32f0xx_hal_flash_ex.o ABSOLUTE
    stm32f0xx_hal_gpio.c                     0x00000000   Number         0  stm32f0xx_hal_gpio.o ABSOLUTE
    stm32f0xx_hal_i2c.c                      0x00000000   Number         0  stm32f0xx_hal_i2c.o ABSOLUTE
    stm32f0xx_hal_i2c_ex.c                   0x00000000   Number         0  stm32f0xx_hal_i2c_ex.o ABSOLUTE
    stm32f0xx_hal_msp.c                      0x00000000   Number         0  stm32f0xx_hal_msp.o ABSOLUTE
    stm32f0xx_hal_pwr.c                      0x00000000   Number         0  stm32f0xx_hal_pwr.o ABSOLUTE
    stm32f0xx_hal_pwr_ex.c                   0x00000000   Number         0  stm32f0xx_hal_pwr_ex.o ABSOLUTE
    stm32f0xx_hal_rcc.c                      0x00000000   Number         0  stm32f0xx_hal_rcc.o ABSOLUTE
    stm32f0xx_hal_rcc_ex.c                   0x00000000   Number         0  stm32f0xx_hal_rcc_ex.o ABSOLUTE
    stm32f0xx_hal_rtc.c                      0x00000000   Number         0  stm32f0xx_hal_rtc.o ABSOLUTE
    stm32f0xx_hal_rtc_ex.c                   0x00000000   Number         0  stm32f0xx_hal_rtc_ex.o ABSOLUTE
    stm32f0xx_hal_tim.c                      0x00000000   Number         0  stm32f0xx_hal_tim.o ABSOLUTE
    stm32f0xx_hal_tim_ex.c                   0x00000000   Number         0  stm32f0xx_hal_tim_ex.o ABSOLUTE
    stm32f0xx_it.c                           0x00000000   Number         0  stm32f0xx_it.o ABSOLUTE
    system_stm32f0xx.c                       0x00000000   Number         0  system_stm32f0xx.o ABSOLUTE
    RESET                                    0x08000000   Section      184  startup_stm32f030xc.o(RESET)
    !!!main                                  0x080000b8   Section        8  __main.o(!!!main)
    !!!scatter                               0x080000c0   Section       84  __scatter.o(!!!scatter)
    !!handler_null                           0x08000114   Section        2  __scatter.o(!!handler_null)
    !!handler_zi                             0x08000118   Section       28  __scatter_zi.o(!!handler_zi)
    .ARM.Collect$$_printf_percent$$00000000  0x08000134   Section        2  _printf_percent.o(.ARM.Collect$$_printf_percent$$00000000)
    .ARM.Collect$$_printf_percent$$00000003  0x08000136   Section       10  _printf_f.o(.ARM.Collect$$_printf_percent$$00000003)
    .ARM.Collect$$_printf_percent$$0000000C  0x08000140   Section       10  _printf_x.o(.ARM.Collect$$_printf_percent$$0000000C)
    .ARM.Collect$$_printf_percent$$00000013  0x0800014a   Section       10  _printf_c.o(.ARM.Collect$$_printf_percent$$00000013)
    .ARM.Collect$$_printf_percent$$00000014  0x08000154   Section       10  _printf_s.o(.ARM.Collect$$_printf_percent$$00000014)
    .ARM.Collect$$_printf_percent$$00000017  0x0800015e   Section        4  _printf_percent_end.o(.ARM.Collect$$_printf_percent$$00000017)
    .ARM.Collect$$libinit$$00000000          0x08000162   Section        2  libinit.o(.ARM.Collect$$libinit$$00000000)
    .ARM.Collect$$libinit$$00000002          0x08000164   Section        0  libinit2.o(.ARM.Collect$$libinit$$00000002)
    .ARM.Collect$$libinit$$00000004          0x08000164   Section        0  libinit2.o(.ARM.Collect$$libinit$$00000004)
    .ARM.Collect$$libinit$$00000006          0x08000164   Section        0  libinit2.o(.ARM.Collect$$libinit$$00000006)
    .ARM.Collect$$libinit$$0000000C          0x08000164   Section        0  libinit2.o(.ARM.Collect$$libinit$$0000000C)
    .ARM.Collect$$libinit$$0000000E          0x08000164   Section        0  libinit2.o(.ARM.Collect$$libinit$$0000000E)
    .ARM.Collect$$libinit$$00000010          0x08000164   Section        0  libinit2.o(.ARM.Collect$$libinit$$00000010)
    .ARM.Collect$$libinit$$00000011          0x08000164   Section        6  libinit2.o(.ARM.Collect$$libinit$$00000011)
    .ARM.Collect$$libinit$$00000013          0x0800016a   Section        0  libinit2.o(.ARM.Collect$$libinit$$00000013)
    .ARM.Collect$$libinit$$00000015          0x0800016a   Section        0  libinit2.o(.ARM.Collect$$libinit$$00000015)
    .ARM.Collect$$libinit$$00000017          0x0800016a   Section        0  libinit2.o(.ARM.Collect$$libinit$$00000017)
    .ARM.Collect$$libinit$$00000018          0x0800016a   Section       10  libinit2.o(.ARM.Collect$$libinit$$00000018)
    .ARM.Collect$$libinit$$00000019          0x08000174   Section        0  libinit2.o(.ARM.Collect$$libinit$$00000019)
    .ARM.Collect$$libinit$$0000001B          0x08000174   Section        0  libinit2.o(.ARM.Collect$$libinit$$0000001B)
    .ARM.Collect$$libinit$$0000001D          0x08000174   Section        0  libinit2.o(.ARM.Collect$$libinit$$0000001D)
    .ARM.Collect$$libinit$$0000001F          0x08000174   Section        0  libinit2.o(.ARM.Collect$$libinit$$0000001F)
    .ARM.Collect$$libinit$$00000021          0x08000174   Section        0  libinit2.o(.ARM.Collect$$libinit$$00000021)
    .ARM.Collect$$libinit$$00000023          0x08000174   Section        0  libinit2.o(.ARM.Collect$$libinit$$00000023)
    .ARM.Collect$$libinit$$00000025          0x08000174   Section        0  libinit2.o(.ARM.Collect$$libinit$$00000025)
    .ARM.Collect$$libinit$$00000027          0x08000174   Section        0  libinit2.o(.ARM.Collect$$libinit$$00000027)
    .ARM.Collect$$libinit$$0000002E          0x08000174   Section        0  libinit2.o(.ARM.Collect$$libinit$$0000002E)
    .ARM.Collect$$libinit$$00000030          0x08000174   Section        0  libinit2.o(.ARM.Collect$$libinit$$00000030)
    .ARM.Collect$$libinit$$00000032          0x08000174   Section        0  libinit2.o(.ARM.Collect$$libinit$$00000032)
    .ARM.Collect$$libinit$$00000034          0x08000174   Section        0  libinit2.o(.ARM.Collect$$libinit$$00000034)
    .ARM.Collect$$libinit$$00000035          0x08000174   Section        2  libinit2.o(.ARM.Collect$$libinit$$00000035)
    .ARM.Collect$$libshutdown$$00000000      0x08000176   Section        2  libshutdown.o(.ARM.Collect$$libshutdown$$00000000)
    .ARM.Collect$$libshutdown$$00000002      0x08000178   Section        0  libshutdown2.o(.ARM.Collect$$libshutdown$$00000002)
    .ARM.Collect$$libshutdown$$00000004      0x08000178   Section        0  libshutdown2.o(.ARM.Collect$$libshutdown$$00000004)
    .ARM.Collect$$libshutdown$$00000007      0x08000178   Section        0  libshutdown2.o(.ARM.Collect$$libshutdown$$00000007)
    .ARM.Collect$$libshutdown$$0000000A      0x08000178   Section        0  libshutdown2.o(.ARM.Collect$$libshutdown$$0000000A)
    .ARM.Collect$$libshutdown$$0000000C      0x08000178   Section        0  libshutdown2.o(.ARM.Collect$$libshutdown$$0000000C)
    .ARM.Collect$$libshutdown$$0000000F      0x08000178   Section        0  libshutdown2.o(.ARM.Collect$$libshutdown$$0000000F)
    .ARM.Collect$$libshutdown$$00000010      0x08000178   Section        2  libshutdown2.o(.ARM.Collect$$libshutdown$$00000010)
    .ARM.Collect$$rtentry$$00000000          0x0800017a   Section        0  __rtentry.o(.ARM.Collect$$rtentry$$00000000)
    .ARM.Collect$$rtentry$$00000002          0x0800017a   Section        0  __rtentry2.o(.ARM.Collect$$rtentry$$00000002)
    .ARM.Collect$$rtentry$$00000004          0x0800017a   Section        6  __rtentry4.o(.ARM.Collect$$rtentry$$00000004)
    .ARM.Collect$$rtentry$$00000009          0x08000180   Section        0  __rtentry2.o(.ARM.Collect$$rtentry$$00000009)
    .ARM.Collect$$rtentry$$0000000A          0x08000180   Section        4  __rtentry2.o(.ARM.Collect$$rtentry$$0000000A)
    .ARM.Collect$$rtentry$$0000000C          0x08000184   Section        0  __rtentry2.o(.ARM.Collect$$rtentry$$0000000C)
    .ARM.Collect$$rtentry$$0000000D          0x08000184   Section        8  __rtentry2.o(.ARM.Collect$$rtentry$$0000000D)
    .ARM.Collect$$rtexit$$00000000           0x0800018c   Section        2  rtexit.o(.ARM.Collect$$rtexit$$00000000)
    .ARM.Collect$$rtexit$$00000002           0x0800018e   Section        0  rtexit2.o(.ARM.Collect$$rtexit$$00000002)
    .ARM.Collect$$rtexit$$00000003           0x0800018e   Section        4  rtexit2.o(.ARM.Collect$$rtexit$$00000003)
    .ARM.Collect$$rtexit$$00000004           0x08000192   Section        6  rtexit2.o(.ARM.Collect$$rtexit$$00000004)
    .text                                    0x08000198   Section       56  startup_stm32f030xc.o(.text)
    .text                                    0x080001d0   Section        0  noretval__2sprintf.o(.text)
    .text                                    0x080001f8   Section        0  _printf_pad.o(.text)
    .text                                    0x08000246   Section        0  _printf_str.o(.text)
    .text                                    0x08000298   Section        0  _printf_hex_int.o(.text)
    .text                                    0x080002f0   Section        0  __printf_flags_wp.o(.text)
    .text                                    0x08000428   Section      504  aeabi_sdivfast.o(.text)
    .text                                    0x08000620   Section        0  heapauxi.o(.text)
    .text                                    0x08000628   Section        0  d2f.o(.text)
    _dadd1                                   0x080006a5   Thumb Code   290  daddsub.o(.text)
    .text                                    0x080006a4   Section        0  daddsub.o(.text)
    _dsub1                                   0x080007c7   Thumb Code   470  daddsub.o(.text)
    .text                                    0x080009fc   Section        0  ddiv.o(.text)
    .text                                    0x08000e44   Section        0  dfixi.o(.text)
    .text                                    0x08000eb0   Section        0  dflti.o(.text)
    .text                                    0x08000f08   Section        0  dmul.o(.text)
    .text                                    0x08001150   Section        0  f2d.o(.text)
    .text                                    0x080011a4   Section        0  fflti.o(.text)
    .text                                    0x08001202   Section        0  _rserrno.o(.text)
    .text                                    0x08001218   Section        0  _printf_intcommon.o(.text)
    _fp_digits                               0x080012c9   Thumb Code   412  _printf_fp_dec.o(.text)
    .text                                    0x080012c8   Section        0  _printf_fp_dec.o(.text)
    _printf_input_char                       0x080016dd   Thumb Code    10  _printf_char_common.o(.text)
    .text                                    0x080016dc   Section        0  _printf_char_common.o(.text)
    .text                                    0x0800170c   Section        0  _sputc.o(.text)
    .text                                    0x08001716   Section        0  _printf_char.o(.text)
    .text                                    0x08001744   Section        0  dscalbn.o(.text)
    .text                                    0x080017a4   Section        8  rt_locale_intlibspace.o(.text)
    .text                                    0x080017ac   Section        8  rt_errno_addr_intlibspace.o(.text)
    .text                                    0x080017b4   Section        0  lludiv10.o(.text)
    .text                                    0x08001830   Section        0  _printf_fp_infnan.o(.text)
    .text                                    0x080018b8   Section        0  bigflt0.o(.text)
    .text                                    0x08001990   Section        0  btod.o(.text)
    btod_internal_mul                        0x080019d1   Thumb Code   492  btod.o(.text)
    btod_internal_div                        0x08001bbd   Thumb Code   520  btod.o(.text)
    .text                                    0x08001f10   Section        0  rtudiv10.o(.text)
    .text                                    0x08001f38   Section        0  dcmpin.o(.text)
    .text                                    0x08001fd8   Section        0  dsqrt.o(.text)
    .text                                    0x080020d8   Section        8  libspace.o(.text)
    .text                                    0x080020e0   Section       62  sys_stackheap_outer.o(.text)
    .text                                    0x0800211e   Section        0  exit.o(.text)
    .text                                    0x08002130   Section      176  strcmpv6m.o(.text)
    .text                                    0x080021e0   Section        0  cmpret.o(.text)
    .text                                    0x08002210   Section        0  dnan2.o(.text)
    .text                                    0x08002224   Section        0  retnan.o(.text)
    .text                                    0x08002284   Section        0  sys_exit.o(.text)
    .text                                    0x08002290   Section        2  use_no_semi.o(.text)
    .text                                    0x08002292   Section        0  indicate_semi.o(.text)
    .text                                    0x08002292   Section        0  __dczerorl2.o(.text)
    [Anonymous Symbol]                       0x080022e8   Section        0  bmp280+aht20.o(.text.AHT20_Read)
    __arm_cp.4_0                             0x0800236c   Number         4  bmp280+aht20.o(.text.AHT20_Read)
    __arm_cp.4_1                             0x08002370   Number         4  bmp280+aht20.o(.text.AHT20_Read)
    __arm_cp.4_2                             0x08002374   Number         4  bmp280+aht20.o(.text.AHT20_Read)
    __arm_cp.4_4                             0x08002378   Number         4  bmp280+aht20.o(.text.AHT20_Read)
    __arm_cp.4_5                             0x0800237c   Number         4  bmp280+aht20.o(.text.AHT20_Read)
    [Anonymous Symbol]                       0x08002380   Section        0  bmp280+aht20.o(.text.BMP280_calc_values)
    __arm_cp.2_0                             0x080026f8   Number         4  bmp280+aht20.o(.text.BMP280_calc_values)
    __arm_cp.2_1                             0x080026fc   Number         4  bmp280+aht20.o(.text.BMP280_calc_values)
    __arm_cp.2_2                             0x08002700   Number         4  bmp280+aht20.o(.text.BMP280_calc_values)
    __arm_cp.2_3                             0x08002704   Number         4  bmp280+aht20.o(.text.BMP280_calc_values)
    __arm_cp.2_4                             0x08002708   Number         4  bmp280+aht20.o(.text.BMP280_calc_values)
    __arm_cp.2_5                             0x0800270c   Number         4  bmp280+aht20.o(.text.BMP280_calc_values)
    __arm_cp.2_6                             0x08002710   Number         4  bmp280+aht20.o(.text.BMP280_calc_values)
    __arm_cp.2_7                             0x08002714   Number         4  bmp280+aht20.o(.text.BMP280_calc_values)
    __arm_cp.2_8                             0x08002718   Number         4  bmp280+aht20.o(.text.BMP280_calc_values)
    __arm_cp.2_9                             0x0800271c   Number         4  bmp280+aht20.o(.text.BMP280_calc_values)
    __arm_cp.2_10                            0x08002720   Number         4  bmp280+aht20.o(.text.BMP280_calc_values)
    __arm_cp.2_11                            0x08002724   Number         4  bmp280+aht20.o(.text.BMP280_calc_values)
    __arm_cp.2_12                            0x08002728   Number         4  bmp280+aht20.o(.text.BMP280_calc_values)
    __arm_cp.2_13                            0x0800272c   Number         4  bmp280+aht20.o(.text.BMP280_calc_values)
    __arm_cp.2_14                            0x08002730   Number         4  bmp280+aht20.o(.text.BMP280_calc_values)
    __arm_cp.2_15                            0x08002734   Number         4  bmp280+aht20.o(.text.BMP280_calc_values)
    __arm_cp.2_16                            0x08002738   Number         4  bmp280+aht20.o(.text.BMP280_calc_values)
    __arm_cp.2_17                            0x0800273c   Number         4  bmp280+aht20.o(.text.BMP280_calc_values)
    __arm_cp.2_18                            0x08002740   Number         4  bmp280+aht20.o(.text.BMP280_calc_values)
    __arm_cp.2_19                            0x08002744   Number         4  bmp280+aht20.o(.text.BMP280_calc_values)
    [Anonymous Symbol]                       0x08002748   Section        0  bmp280+aht20.o(.text.BMP280_init)
    __arm_cp.0_0                             0x08002844   Number         4  bmp280+aht20.o(.text.BMP280_init)
    __arm_cp.0_1                             0x08002848   Number         4  bmp280+aht20.o(.text.BMP280_init)
    [Anonymous Symbol]                       0x0800284c   Section        0  stm32f0xx_hal.o(.text.HAL_Delay)
    __arm_cp.10_0                            0x0800286c   Number         4  stm32f0xx_hal.o(.text.HAL_Delay)
    [Anonymous Symbol]                       0x08002870   Section        0  stm32f0xx_hal_gpio.o(.text.HAL_GPIO_Init)
    __arm_cp.0_0                             0x08002a18   Number         4  stm32f0xx_hal_gpio.o(.text.HAL_GPIO_Init)
    __arm_cp.0_1                             0x08002a1c   Number         4  stm32f0xx_hal_gpio.o(.text.HAL_GPIO_Init)
    __arm_cp.0_2                             0x08002a20   Number         4  stm32f0xx_hal_gpio.o(.text.HAL_GPIO_Init)
    __arm_cp.0_3                             0x08002a24   Number         4  stm32f0xx_hal_gpio.o(.text.HAL_GPIO_Init)
    __arm_cp.0_4                             0x08002a28   Number         4  stm32f0xx_hal_gpio.o(.text.HAL_GPIO_Init)
    __arm_cp.0_5                             0x08002a2c   Number         4  stm32f0xx_hal_gpio.o(.text.HAL_GPIO_Init)
    [Anonymous Symbol]                       0x08002a30   Section        0  stm32f0xx_hal.o(.text.HAL_GetTick)
    __arm_cp.6_0                             0x08002a38   Number         4  stm32f0xx_hal.o(.text.HAL_GetTick)
    [Anonymous Symbol]                       0x08002a3c   Section        0  stm32f0xx_hal_i2c_ex.o(.text.HAL_I2CEx_ConfigAnalogFilter)
    [Anonymous Symbol]                       0x08002a7e   Section        0  stm32f0xx_hal_i2c_ex.o(.text.HAL_I2CEx_ConfigDigitalFilter)
    [Anonymous Symbol]                       0x08002ac0   Section        0  stm32f0xx_hal_i2c.o(.text.HAL_I2C_Init)
    __arm_cp.0_0                             0x08002b6c   Number         4  stm32f0xx_hal_i2c.o(.text.HAL_I2C_Init)
    __arm_cp.0_1                             0x08002b70   Number         4  stm32f0xx_hal_i2c.o(.text.HAL_I2C_Init)
    [Anonymous Symbol]                       0x08002b74   Section        0  stm32f0xx_hal_i2c.o(.text.HAL_I2C_Master_Receive)
    __arm_cp.8_2                             0x08002d04   Number         4  stm32f0xx_hal_i2c.o(.text.HAL_I2C_Master_Receive)
    __arm_cp.8_3                             0x08002d08   Number         4  stm32f0xx_hal_i2c.o(.text.HAL_I2C_Master_Receive)
    [Anonymous Symbol]                       0x08002d0c   Section        0  stm32f0xx_hal_i2c.o(.text.HAL_I2C_Master_Transmit)
    __arm_cp.4_0                             0x08002eb8   Number         4  stm32f0xx_hal_i2c.o(.text.HAL_I2C_Master_Transmit)
    __arm_cp.4_1                             0x08002ebc   Number         4  stm32f0xx_hal_i2c.o(.text.HAL_I2C_Master_Transmit)
    __arm_cp.4_2                             0x08002ec0   Number         4  stm32f0xx_hal_i2c.o(.text.HAL_I2C_Master_Transmit)
    __arm_cp.4_3                             0x08002ec4   Number         4  stm32f0xx_hal_i2c.o(.text.HAL_I2C_Master_Transmit)
    __arm_cp.4_4                             0x08002ec8   Number         4  stm32f0xx_hal_i2c.o(.text.HAL_I2C_Master_Transmit)
    [Anonymous Symbol]                       0x08002ecc   Section        0  stm32f0xx_hal_i2c.o(.text.HAL_I2C_Mem_Read)
    __arm_cp.30_0                            0x080030e0   Number         4  stm32f0xx_hal_i2c.o(.text.HAL_I2C_Mem_Read)
    __arm_cp.30_1                            0x080030e4   Number         4  stm32f0xx_hal_i2c.o(.text.HAL_I2C_Mem_Read)
    __arm_cp.30_2                            0x080030e8   Number         4  stm32f0xx_hal_i2c.o(.text.HAL_I2C_Mem_Read)
    __arm_cp.30_3                            0x080030ec   Number         4  stm32f0xx_hal_i2c.o(.text.HAL_I2C_Mem_Read)
    __arm_cp.30_4                            0x080030f0   Number         4  stm32f0xx_hal_i2c.o(.text.HAL_I2C_Mem_Read)
    __arm_cp.30_5                            0x080030f4   Number         4  stm32f0xx_hal_i2c.o(.text.HAL_I2C_Mem_Read)
    __arm_cp.30_6                            0x080030f8   Number         4  stm32f0xx_hal_i2c.o(.text.HAL_I2C_Mem_Read)
    [Anonymous Symbol]                       0x080030fc   Section        0  stm32f0xx_hal_msp.o(.text.HAL_I2C_MspInit)
    __arm_cp.1_0                             0x08003154   Number         4  stm32f0xx_hal_msp.o(.text.HAL_I2C_MspInit)
    __arm_cp.1_1                             0x08003158   Number         4  stm32f0xx_hal_msp.o(.text.HAL_I2C_MspInit)
    [Anonymous Symbol]                       0x0800315c   Section        0  stm32f0xx_hal.o(.text.HAL_IncTick)
    __arm_cp.5_1                             0x0800316c   Number         4  stm32f0xx_hal.o(.text.HAL_IncTick)
    [Anonymous Symbol]                       0x08003170   Section        0  stm32f0xx_hal.o(.text.HAL_Init)
    [Anonymous Symbol]                       0x0800318c   Section        0  stm32f0xx_hal.o(.text.HAL_InitTick)
    __arm_cp.1_0                             0x080031c8   Number         4  stm32f0xx_hal.o(.text.HAL_InitTick)
    [Anonymous Symbol]                       0x080031cc   Section        0  stm32f0xx_hal_msp.o(.text.HAL_MspInit)
    __arm_cp.0_0                             0x080031f4   Number         4  stm32f0xx_hal_msp.o(.text.HAL_MspInit)
    [Anonymous Symbol]                       0x080031f8   Section        0  stm32f0xx_hal_cortex.o(.text.HAL_NVIC_SetPriority)
    __arm_cp.0_0                             0x08003228   Number         4  stm32f0xx_hal_cortex.o(.text.HAL_NVIC_SetPriority)
    __arm_cp.0_1                             0x0800322c   Number         4  stm32f0xx_hal_cortex.o(.text.HAL_NVIC_SetPriority)
    [Anonymous Symbol]                       0x08003230   Section        0  stm32f0xx_hal_pwr.o(.text.HAL_PWR_EnableBkUpAccess)
    [Anonymous Symbol]                       0x08003240   Section        0  stm32f0xx_hal_rcc_ex.o(.text.HAL_RCCEx_PeriphCLKConfig)
    __arm_cp.0_0                             0x08003334   Number         4  stm32f0xx_hal_rcc_ex.o(.text.HAL_RCCEx_PeriphCLKConfig)
    __arm_cp.0_1                             0x08003338   Number         4  stm32f0xx_hal_rcc_ex.o(.text.HAL_RCCEx_PeriphCLKConfig)
    __arm_cp.0_2                             0x0800333c   Number         4  stm32f0xx_hal_rcc_ex.o(.text.HAL_RCCEx_PeriphCLKConfig)
    [Anonymous Symbol]                       0x08003340   Section        0  stm32f0xx_hal_rcc.o(.text.HAL_RCC_ClockConfig)
    __arm_cp.2_0                             0x08003468   Number         4  stm32f0xx_hal_rcc.o(.text.HAL_RCC_ClockConfig)
    __arm_cp.2_1                             0x0800346c   Number         4  stm32f0xx_hal_rcc.o(.text.HAL_RCC_ClockConfig)
    __arm_cp.2_2                             0x08003470   Number         4  stm32f0xx_hal_rcc.o(.text.HAL_RCC_ClockConfig)
    __arm_cp.2_3                             0x08003474   Number         4  stm32f0xx_hal_rcc.o(.text.HAL_RCC_ClockConfig)
    __arm_cp.2_4                             0x08003478   Number         4  stm32f0xx_hal_rcc.o(.text.HAL_RCC_ClockConfig)
    __arm_cp.2_5                             0x0800347c   Number         4  stm32f0xx_hal_rcc.o(.text.HAL_RCC_ClockConfig)
    __arm_cp.2_6                             0x08003480   Number         4  stm32f0xx_hal_rcc.o(.text.HAL_RCC_ClockConfig)
    __arm_cp.2_7                             0x08003484   Number         4  stm32f0xx_hal_rcc.o(.text.HAL_RCC_ClockConfig)
    [Anonymous Symbol]                       0x08003488   Section        0  stm32f0xx_hal_rcc.o(.text.HAL_RCC_OscConfig)
    __arm_cp.1_0                             0x0800388c   Number         4  stm32f0xx_hal_rcc.o(.text.HAL_RCC_OscConfig)
    __arm_cp.1_1                             0x08003890   Number         4  stm32f0xx_hal_rcc.o(.text.HAL_RCC_OscConfig)
    __arm_cp.1_2                             0x08003894   Number         4  stm32f0xx_hal_rcc.o(.text.HAL_RCC_OscConfig)
    [Anonymous Symbol]                       0x08003898   Section        0  stm32f0xx_hal_rtc.o(.text.HAL_RTC_GetDate)
    [Anonymous Symbol]                       0x080038e8   Section        0  stm32f0xx_hal_rtc.o(.text.HAL_RTC_GetTime)
    __arm_cp.8_0                             0x08003950   Number         4  stm32f0xx_hal_rtc.o(.text.HAL_RTC_GetTime)
    [Anonymous Symbol]                       0x08003954   Section        0  stm32f0xx_hal_rtc.o(.text.HAL_RTC_Init)
    __arm_cp.0_0                             0x08003a48   Number         4  stm32f0xx_hal_rtc.o(.text.HAL_RTC_Init)
    [Anonymous Symbol]                       0x08003a4c   Section        0  stm32f0xx_hal_msp.o(.text.HAL_RTC_MspInit)
    __arm_cp.3_0                             0x08003a64   Number         4  stm32f0xx_hal_msp.o(.text.HAL_RTC_MspInit)
    __arm_cp.3_1                             0x08003a68   Number         4  stm32f0xx_hal_msp.o(.text.HAL_RTC_MspInit)
    [Anonymous Symbol]                       0x08003a6c   Section        0  stm32f0xx_hal_rtc.o(.text.HAL_RTC_SetDate)
    [Anonymous Symbol]                       0x08003bc4   Section        0  stm32f0xx_hal_rtc.o(.text.HAL_RTC_SetTime)
    __arm_cp.6_0                             0x08003d3c   Number         4  stm32f0xx_hal_rtc.o(.text.HAL_RTC_SetTime)
    __arm_cp.6_1                             0x08003d40   Number         4  stm32f0xx_hal_rtc.o(.text.HAL_RTC_SetTime)
    [Anonymous Symbol]                       0x08003d44   Section        0  stm32f0xx_hal_cortex.o(.text.HAL_SYSTICK_Config)
    __arm_cp.4_0                             0x08003d6c   Number         4  stm32f0xx_hal_cortex.o(.text.HAL_SYSTICK_Config)
    __arm_cp.4_1                             0x08003d70   Number         4  stm32f0xx_hal_cortex.o(.text.HAL_SYSTICK_Config)
    __arm_cp.4_2                             0x08003d74   Number         4  stm32f0xx_hal_cortex.o(.text.HAL_SYSTICK_Config)
    [Anonymous Symbol]                       0x08003d78   Section        0  stm32f0xx_it.o(.text.HardFault_Handler)
    I2C_IsErrorOccurred                      0x08003d7d   Thumb Code   380  stm32f0xx_hal_i2c.o(.text.I2C_IsErrorOccurred)
    [Anonymous Symbol]                       0x08003d7c   Section        0  stm32f0xx_hal_i2c.o(.text.I2C_IsErrorOccurred)
    I2C_WaitOnFlagUntilTimeout               0x08003ef9   Thumb Code   250  stm32f0xx_hal_i2c.o(.text.I2C_WaitOnFlagUntilTimeout)
    [Anonymous Symbol]                       0x08003ef8   Section        0  stm32f0xx_hal_i2c.o(.text.I2C_WaitOnFlagUntilTimeout)
    I2C_WaitOnRXNEFlagUntilTimeout           0x08003ff5   Thumb Code   208  stm32f0xx_hal_i2c.o(.text.I2C_WaitOnRXNEFlagUntilTimeout)
    [Anonymous Symbol]                       0x08003ff4   Section        0  stm32f0xx_hal_i2c.o(.text.I2C_WaitOnRXNEFlagUntilTimeout)
    __arm_cp.9_0                             0x080040c4   Number         4  stm32f0xx_hal_i2c.o(.text.I2C_WaitOnRXNEFlagUntilTimeout)
    I2C_WaitOnSTOPFlagUntilTimeout           0x080040c9   Thumb Code   134  stm32f0xx_hal_i2c.o(.text.I2C_WaitOnSTOPFlagUntilTimeout)
    [Anonymous Symbol]                       0x080040c8   Section        0  stm32f0xx_hal_i2c.o(.text.I2C_WaitOnSTOPFlagUntilTimeout)
    I2C_WaitOnTXISFlagUntilTimeout           0x0800414f   Thumb Code   166  stm32f0xx_hal_i2c.o(.text.I2C_WaitOnTXISFlagUntilTimeout)
    [Anonymous Symbol]                       0x0800414e   Section        0  stm32f0xx_hal_i2c.o(.text.I2C_WaitOnTXISFlagUntilTimeout)
    [Anonymous Symbol]                       0x080041f4   Section        0  stm32f0xx_it.o(.text.NMI_Handler)
    [Anonymous Symbol]                       0x080041f8   Section        0  ssd1306.o(.text.OLCD_write_string)
    __arm_cp.7_2                             0x080043a4   Number         4  ssd1306.o(.text.OLCD_write_string)
    [Anonymous Symbol]                       0x080043a8   Section        0  stm32f0xx_it.o(.text.PendSV_Handler)
    [Anonymous Symbol]                       0x080043aa   Section        0  stm32f0xx_it.o(.text.SVC_Handler)
    [Anonymous Symbol]                       0x080043ac   Section        0  stm32f0xx_it.o(.text.SysTick_Handler)
    [Anonymous Symbol]                       0x080043b4   Section        0  main.o(.text.SystemClock_Config)
    __arm_cp.1_0                             0x08004438   Number         4  main.o(.text.SystemClock_Config)
    __arm_cp.1_1                             0x0800443c   Number         4  main.o(.text.SystemClock_Config)
    [Anonymous Symbol]                       0x08004440   Section        0  system_stm32f0xx.o(.text.SystemInit)
    [Anonymous Symbol]                       0x08004444   Section        0  ssd1306.o(.text.clear_display)
    [Anonymous Symbol]                       0x080044d4   Section        0  ssd1306.o(.text.init_OLED)
    __arm_cp.0_0                             0x08004504   Number         4  ssd1306.o(.text.init_OLED)
    __arm_cp.0_1                             0x08004508   Number         4  ssd1306.o(.text.init_OLED)
    __arm_cp.0_2                             0x0800450c   Number         4  ssd1306.o(.text.init_OLED)
    [Anonymous Symbol]                       0x08004510   Section        0  main.o(.text.main)
    __arm_cp.0_0                             0x08004748   Number         4  main.o(.text.main)
    __arm_cp.0_1                             0x0800474c   Number         4  main.o(.text.main)
    __arm_cp.0_2                             0x08004750   Number         4  main.o(.text.main)
    __arm_cp.0_3                             0x08004754   Number         4  main.o(.text.main)
    __arm_cp.0_4                             0x08004758   Number         4  main.o(.text.main)
    __arm_cp.0_5                             0x0800475c   Number         4  main.o(.text.main)
    __arm_cp.0_6                             0x08004760   Number         4  main.o(.text.main)
    __arm_cp.0_7                             0x08004764   Number         4  main.o(.text.main)
    __arm_cp.0_9                             0x08004778   Number         4  main.o(.text.main)
    __arm_cp.0_12                            0x080047a4   Number         4  main.o(.text.main)
    __arm_cp.0_13                            0x080047a8   Number         4  main.o(.text.main)
    __arm_cp.0_15                            0x080047c0   Number         4  main.o(.text.main)
    __arm_cp.0_17                            0x080047d8   Number         4  main.o(.text.main)
    __arm_cp.0_19                            0x080047e8   Number         4  main.o(.text.main)
    .text_divfast                            0x08004800   Section      502  aeabi_sdivfast.o(.text_divfast)
    i.__ARM_common_ll_muluu                  0x080049f6   Section        0  btod.o(i.__ARM_common_ll_muluu)
    i.__ARM_fpclassify                       0x08004a28   Section        0  fpclassify.o(i.__ARM_fpclassify)
    i.__kernel_poly                          0x08004a54   Section        0  poly.o(i.__kernel_poly)
    i.__mathlib_dbl_divzero                  0x08004b00   Section        0  dunder.o(i.__mathlib_dbl_divzero)
    i.__mathlib_dbl_infnan2                  0x08004b14   Section        0  dunder.o(i.__mathlib_dbl_infnan2)
    i.__mathlib_dbl_invalid                  0x08004b1c   Section        0  dunder.o(i.__mathlib_dbl_invalid)
    i.__mathlib_dbl_overflow                 0x08004b2c   Section        0  dunder.o(i.__mathlib_dbl_overflow)
    i.__mathlib_dbl_underflow                0x08004b40   Section        0  dunder.o(i.__mathlib_dbl_underflow)
    i._is_digit                              0x08004b54   Section        0  __printf_wp.o(i._is_digit)
    i.pow                                    0x08004b64   Section        0  pow.o(i.pow)
    i.sqrt                                   0x08005538   Section        0  sqrt.o(i.sqrt)
    locale$$code                             0x08005580   Section       44  lc_numeric_c.o(locale$$code)
    x$fpl$drleqf                             0x080055ac   Section      104  drlef.o(x$fpl$drleqf)
    x$fpl$fadd                               0x08005614   Section      140  faddsub.o(x$fpl$fadd)
    _fadd1                                   0x08005621   Thumb Code     0  faddsub.o(x$fpl$fadd)
    x$fpl$fmul                               0x080056a0   Section      176  fmul.o(x$fpl$fmul)
    x$fpl$fsub                               0x08005750   Section      208  faddsub.o(x$fpl$fsub)
    _fsub1                                   0x0800575d   Thumb Code     0  faddsub.o(x$fpl$fsub)
    x$fpl$printf1                            0x08005820   Section       16  printf1.o(x$fpl$printf1)
    uc_hextab                                0x08005830   Data          20  _printf_hex_int.o(.constdata)
    .constdata                               0x08005830   Section       40  _printf_hex_int.o(.constdata)
    x$fpl$usenofp                            0x08005830   Section        0  usenofp.o(x$fpl$usenofp)
    lc_hextab                                0x08005844   Data          20  _printf_hex_int.o(.constdata)
    maptable                                 0x08005858   Data          17  __printf_flags_wp.o(.constdata)
    .constdata                               0x08005858   Section       17  __printf_flags_wp.o(.constdata)
    ddiv_reciptbl                            0x08005869   Data         128  ddiv.o(.constdata)
    .constdata                               0x08005869   Section      128  ddiv.o(.constdata)
    bp                                       0x080058f0   Data          16  pow.o(.constdata)
    .constdata                               0x080058f0   Section      136  pow.o(.constdata)
    dp_h                                     0x08005900   Data          16  pow.o(.constdata)
    dp_l                                     0x08005910   Data          16  pow.o(.constdata)
    L                                        0x08005920   Data          48  pow.o(.constdata)
    P                                        0x08005950   Data          40  pow.o(.constdata)
    .constdata                               0x08005978   Section        8  qnan.o(.constdata)
    tenpwrs_x                                0x08005980   Data          60  bigflt0.o(.constdata)
    .constdata                               0x08005980   Section      148  bigflt0.o(.constdata)
    tenpwrs_i                                0x080059bc   Data          64  bigflt0.o(.constdata)
    HAL_RCC_GetSysClockFreq.aPLLMULFactorTable 0x08005a24   Data          16  stm32f0xx_hal_rcc.o(.rodata.cst16)
    [Anonymous Symbol]                       0x08005a24   Section        0  stm32f0xx_hal_rcc.o(.rodata.cst16)
    HAL_RCC_GetSysClockFreq.aPredivFactorTable 0x08005a34   Data          16  stm32f0xx_hal_rcc.o(.rodata.cst16)
    [Anonymous Symbol]                       0x08005a44   Section        0  main.o(.rodata.str1.1)
    locale$$data                             0x08005a88   Section       28  lc_numeric_c.o(locale$$data)
    __lcnum_c_name                           0x08005a8c   Data           2  lc_numeric_c.o(locale$$data)
    __lcnum_c_start                          0x08005a94   Data           0  lc_numeric_c.o(locale$$data)
    __lcnum_c_point                          0x08005aa0   Data           0  lc_numeric_c.o(locale$$data)
    __lcnum_c_thousands                      0x08005aa2   Data           0  lc_numeric_c.o(locale$$data)
    __lcnum_c_grouping                       0x08005aa3   Data           0  lc_numeric_c.o(locale$$data)
    __lcnum_c_end                            0x08005aa4   Data           0  lc_numeric_c.o(locale$$data)
    [Anonymous Symbol]                       0x20000000   Section        0  main.o(.data..L_MergedGlobals)
    [Anonymous Symbol]                       0x20000038   Section        0  stm32f0xx_hal.o(.data..L_MergedGlobals)
    .bss                                     0x20000360   Section       96  libspace.o(.bss)
    [Anonymous Symbol]                       0x200003c0   Section        0  bmp280+aht20.o(.bss..L_MergedGlobals)
    [Anonymous Symbol]                       0x200003f8   Section        0  main.o(.bss..L_MergedGlobals.16)
    Heap_Mem                                 0x200004a0   Data         512  startup_stm32f030xc.o(HEAP)
    HEAP                                     0x200004a0   Section      512  startup_stm32f030xc.o(HEAP)
    Stack_Mem                                0x200006a0   Data        1024  startup_stm32f030xc.o(STACK)
    STACK                                    0x200006a0   Section     1024  startup_stm32f030xc.o(STACK)
    __initial_sp                             0x20000aa0   Data           0  startup_stm32f030xc.o(STACK)

    Global Symbols

    Symbol Name                              Value     Ov Type        Size  Object(Section)

    BuildAttributes$$THM_ISAv3M$S$PE$A:L22$X:L11$S22$IEEE1$IW$~IW$USESV6$~STKCKD$USESV7$~SHL$OTIME$ROPI$IEEEX$EBA8$UX$STANDARDLIB$REQ8$PRES8$EABIv2 0x00000000   Number         0  anon$$obj.o ABSOLUTE
    _printf_flags                            0x00000000   Number         0  printf_stubs.o ABSOLUTE
    _printf_return_value                     0x00000000   Number         0  printf_stubs.o ABSOLUTE
    _printf_sizespec                         0x00000000   Number         0  printf_stubs.o ABSOLUTE
    _printf_widthprec                        0x00000000   Number         0  printf_stubs.o ABSOLUTE
    __ARM_exceptions_init                     - Undefined Weak Reference
    __alloca_initialize                       - Undefined Weak Reference
    __arm_preinit_                            - Undefined Weak Reference
    __arm_relocate_pie_                       - Undefined Weak Reference
    __cpp_initialize__aeabi_                  - Undefined Weak Reference
    __cxa_finalize                            - Undefined Weak Reference
    __sigvec_lookup                           - Undefined Weak Reference
    _atexit_init                              - Undefined Weak Reference
    _call_atexit_fns                          - Undefined Weak Reference
    _clock_init                               - Undefined Weak Reference
    _fp_trap_init                             - Undefined Weak Reference
    _fp_trap_shutdown                         - Undefined Weak Reference
    _get_lc_collate                           - Undefined Weak Reference
    _get_lc_ctype                             - Undefined Weak Reference
    _get_lc_monetary                          - Undefined Weak Reference
    _get_lc_time                              - Undefined Weak Reference
    _getenv_init                              - Undefined Weak Reference
    _handle_redirection                       - Undefined Weak Reference
    _init_alloc                               - Undefined Weak Reference
    _init_user_alloc                          - Undefined Weak Reference
    _initio                                   - Undefined Weak Reference
    _printf_mbtowc                            - Undefined Weak Reference
    _printf_truncate_unsigned                 - Undefined Weak Reference
    _rand_init                                - Undefined Weak Reference
    _signal_finish                            - Undefined Weak Reference
    _signal_init                              - Undefined Weak Reference
    _terminate_alloc                          - Undefined Weak Reference
    _terminate_user_alloc                     - Undefined Weak Reference
    _terminateio                              - Undefined Weak Reference
    __Vectors_Size                           0x000000b8   Number         0  startup_stm32f030xc.o ABSOLUTE
    __Vectors                                0x08000000   Data           4  startup_stm32f030xc.o(RESET)
    __Vectors_End                            0x080000b8   Data           0  startup_stm32f030xc.o(RESET)
    __main                                   0x080000b9   Thumb Code     8  __main.o(!!!main)
    __scatterload                            0x080000c1   Thumb Code     0  __scatter.o(!!!scatter)
    __scatterload_rt2                        0x080000c1   Thumb Code    74  __scatter.o(!!!scatter)
    __scatterload_rt2_thumb_only             0x080000c1   Thumb Code     0  __scatter.o(!!!scatter)
    __scatterload_loop                       0x080000cb   Thumb Code     0  __scatter.o(!!!scatter)
    __scatterload_null                       0x08000115   Thumb Code     2  __scatter.o(!!handler_null)
    __scatterload_zeroinit                   0x08000119   Thumb Code    28  __scatter_zi.o(!!handler_zi)
    _printf_percent                          0x08000135   Thumb Code     0  _printf_percent.o(.ARM.Collect$$_printf_percent$$00000000)
    _printf_f                                0x08000137   Thumb Code     0  _printf_f.o(.ARM.Collect$$_printf_percent$$00000003)
    _printf_x                                0x08000141   Thumb Code     0  _printf_x.o(.ARM.Collect$$_printf_percent$$0000000C)
    _printf_c                                0x0800014b   Thumb Code     0  _printf_c.o(.ARM.Collect$$_printf_percent$$00000013)
    _printf_s                                0x08000155   Thumb Code     0  _printf_s.o(.ARM.Collect$$_printf_percent$$00000014)
    _printf_percent_end                      0x0800015f   Thumb Code     0  _printf_percent_end.o(.ARM.Collect$$_printf_percent$$00000017)
    __rt_lib_init                            0x08000163   Thumb Code     0  libinit.o(.ARM.Collect$$libinit$$00000000)
    __rt_lib_init_fp_1                       0x08000165   Thumb Code     0  libinit2.o(.ARM.Collect$$libinit$$00000002)
    __rt_lib_init_heap_1                     0x08000165   Thumb Code     0  libinit2.o(.ARM.Collect$$libinit$$0000000C)
    __rt_lib_init_lc_common                  0x08000165   Thumb Code     0  libinit2.o(.ARM.Collect$$libinit$$00000011)
    __rt_lib_init_preinit_1                  0x08000165   Thumb Code     0  libinit2.o(.ARM.Collect$$libinit$$00000006)
    __rt_lib_init_rand_1                     0x08000165   Thumb Code     0  libinit2.o(.ARM.Collect$$libinit$$00000010)
    __rt_lib_init_relocate_pie_1             0x08000165   Thumb Code     0  libinit2.o(.ARM.Collect$$libinit$$00000004)
    __rt_lib_init_user_alloc_1               0x08000165   Thumb Code     0  libinit2.o(.ARM.Collect$$libinit$$0000000E)
    __rt_lib_init_lc_collate_1               0x0800016b   Thumb Code     0  libinit2.o(.ARM.Collect$$libinit$$00000013)
    __rt_lib_init_lc_ctype_1                 0x0800016b   Thumb Code     0  libinit2.o(.ARM.Collect$$libinit$$00000015)
    __rt_lib_init_lc_monetary_1              0x0800016b   Thumb Code     0  libinit2.o(.ARM.Collect$$libinit$$00000017)
    __rt_lib_init_lc_numeric_2               0x0800016b   Thumb Code     0  libinit2.o(.ARM.Collect$$libinit$$00000018)
    __rt_lib_init_alloca_1                   0x08000175   Thumb Code     0  libinit2.o(.ARM.Collect$$libinit$$00000030)
    __rt_lib_init_argv_1                     0x08000175   Thumb Code     0  libinit2.o(.ARM.Collect$$libinit$$0000002E)
    __rt_lib_init_atexit_1                   0x08000175   Thumb Code     0  libinit2.o(.ARM.Collect$$libinit$$0000001D)
    __rt_lib_init_clock_1                    0x08000175   Thumb Code     0  libinit2.o(.ARM.Collect$$libinit$$00000023)
    __rt_lib_init_cpp_1                      0x08000175   Thumb Code     0  libinit2.o(.ARM.Collect$$libinit$$00000034)
    __rt_lib_init_exceptions_1               0x08000175   Thumb Code     0  libinit2.o(.ARM.Collect$$libinit$$00000032)
    __rt_lib_init_fp_trap_1                  0x08000175   Thumb Code     0  libinit2.o(.ARM.Collect$$libinit$$00000021)
    __rt_lib_init_getenv_1                   0x08000175   Thumb Code     0  libinit2.o(.ARM.Collect$$libinit$$00000025)
    __rt_lib_init_lc_numeric_1               0x08000175   Thumb Code     0  libinit2.o(.ARM.Collect$$libinit$$00000019)
    __rt_lib_init_lc_time_1                  0x08000175   Thumb Code     0  libinit2.o(.ARM.Collect$$libinit$$0000001B)
    __rt_lib_init_return                     0x08000175   Thumb Code     0  libinit2.o(.ARM.Collect$$libinit$$00000035)
    __rt_lib_init_signal_1                   0x08000175   Thumb Code     0  libinit2.o(.ARM.Collect$$libinit$$0000001F)
    __rt_lib_init_stdio_1                    0x08000175   Thumb Code     0  libinit2.o(.ARM.Collect$$libinit$$00000027)
    __rt_lib_shutdown                        0x08000177   Thumb Code     0  libshutdown.o(.ARM.Collect$$libshutdown$$00000000)
    __rt_lib_shutdown_cpp_1                  0x08000179   Thumb Code     0  libshutdown2.o(.ARM.Collect$$libshutdown$$00000002)
    __rt_lib_shutdown_fp_trap_1              0x08000179   Thumb Code     0  libshutdown2.o(.ARM.Collect$$libshutdown$$00000007)
    __rt_lib_shutdown_heap_1                 0x08000179   Thumb Code     0  libshutdown2.o(.ARM.Collect$$libshutdown$$0000000F)
    __rt_lib_shutdown_return                 0x08000179   Thumb Code     0  libshutdown2.o(.ARM.Collect$$libshutdown$$00000010)
    __rt_lib_shutdown_signal_1               0x08000179   Thumb Code     0  libshutdown2.o(.ARM.Collect$$libshutdown$$0000000A)
    __rt_lib_shutdown_stdio_1                0x08000179   Thumb Code     0  libshutdown2.o(.ARM.Collect$$libshutdown$$00000004)
    __rt_lib_shutdown_user_alloc_1           0x08000179   Thumb Code     0  libshutdown2.o(.ARM.Collect$$libshutdown$$0000000C)
    __rt_entry                               0x0800017b   Thumb Code     0  __rtentry.o(.ARM.Collect$$rtentry$$00000000)
    __rt_entry_presh_1                       0x0800017b   Thumb Code     0  __rtentry2.o(.ARM.Collect$$rtentry$$00000002)
    __rt_entry_sh                            0x0800017b   Thumb Code     0  __rtentry4.o(.ARM.Collect$$rtentry$$00000004)
    __rt_entry_li                            0x08000181   Thumb Code     0  __rtentry2.o(.ARM.Collect$$rtentry$$0000000A)
    __rt_entry_postsh_1                      0x08000181   Thumb Code     0  __rtentry2.o(.ARM.Collect$$rtentry$$00000009)
    __rt_entry_main                          0x08000185   Thumb Code     0  __rtentry2.o(.ARM.Collect$$rtentry$$0000000D)
    __rt_entry_postli_1                      0x08000185   Thumb Code     0  __rtentry2.o(.ARM.Collect$$rtentry$$0000000C)
    __rt_exit                                0x0800018d   Thumb Code     0  rtexit.o(.ARM.Collect$$rtexit$$00000000)
    __rt_exit_ls                             0x0800018f   Thumb Code     0  rtexit2.o(.ARM.Collect$$rtexit$$00000003)
    __rt_exit_prels_1                        0x0800018f   Thumb Code     0  rtexit2.o(.ARM.Collect$$rtexit$$00000002)
    __rt_exit_exit                           0x08000193   Thumb Code     0  rtexit2.o(.ARM.Collect$$rtexit$$00000004)
    Reset_Handler                            0x08000199   Thumb Code     8  startup_stm32f030xc.o(.text)
    ADC1_IRQHandler                          0x080001ab   Thumb Code     0  startup_stm32f030xc.o(.text)
    DMA1_Channel1_IRQHandler                 0x080001ab   Thumb Code     0  startup_stm32f030xc.o(.text)
    DMA1_Channel2_3_IRQHandler               0x080001ab   Thumb Code     0  startup_stm32f030xc.o(.text)
    DMA1_Channel4_5_IRQHandler               0x080001ab   Thumb Code     0  startup_stm32f030xc.o(.text)
    EXTI0_1_IRQHandler                       0x080001ab   Thumb Code     0  startup_stm32f030xc.o(.text)
    EXTI2_3_IRQHandler                       0x080001ab   Thumb Code     0  startup_stm32f030xc.o(.text)
    EXTI4_15_IRQHandler                      0x080001ab   Thumb Code     0  startup_stm32f030xc.o(.text)
    FLASH_IRQHandler                         0x080001ab   Thumb Code     0  startup_stm32f030xc.o(.text)
    I2C1_IRQHandler                          0x080001ab   Thumb Code     0  startup_stm32f030xc.o(.text)
    I2C2_IRQHandler                          0x080001ab   Thumb Code     0  startup_stm32f030xc.o(.text)
    RCC_IRQHandler                           0x080001ab   Thumb Code     0  startup_stm32f030xc.o(.text)
    RTC_IRQHandler                           0x080001ab   Thumb Code     0  startup_stm32f030xc.o(.text)
    SPI1_IRQHandler                          0x080001ab   Thumb Code     0  startup_stm32f030xc.o(.text)
    SPI2_IRQHandler                          0x080001ab   Thumb Code     0  startup_stm32f030xc.o(.text)
    TIM14_IRQHandler                         0x080001ab   Thumb Code     0  startup_stm32f030xc.o(.text)
    TIM15_IRQHandler                         0x080001ab   Thumb Code     0  startup_stm32f030xc.o(.text)
    TIM16_IRQHandler                         0x080001ab   Thumb Code     0  startup_stm32f030xc.o(.text)
    TIM17_IRQHandler                         0x080001ab   Thumb Code     0  startup_stm32f030xc.o(.text)
    TIM1_BRK_UP_TRG_COM_IRQHandler           0x080001ab   Thumb Code     0  startup_stm32f030xc.o(.text)
    TIM1_CC_IRQHandler                       0x080001ab   Thumb Code     0  startup_stm32f030xc.o(.text)
    TIM3_IRQHandler                          0x080001ab   Thumb Code     0  startup_stm32f030xc.o(.text)
    TIM6_IRQHandler                          0x080001ab   Thumb Code     0  startup_stm32f030xc.o(.text)
    TIM7_IRQHandler                          0x080001ab   Thumb Code     0  startup_stm32f030xc.o(.text)
    USART1_IRQHandler                        0x080001ab   Thumb Code     0  startup_stm32f030xc.o(.text)
    USART2_IRQHandler                        0x080001ab   Thumb Code     0  startup_stm32f030xc.o(.text)
    USART3_6_IRQHandler                      0x080001ab   Thumb Code     0  startup_stm32f030xc.o(.text)
    WWDG_IRQHandler                          0x080001ab   Thumb Code     0  startup_stm32f030xc.o(.text)
    __user_initial_stackheap                 0x080001ad   Thumb Code     0  startup_stm32f030xc.o(.text)
    __2sprintf                               0x080001d1   Thumb Code    36  noretval__2sprintf.o(.text)
    _printf_pre_padding                      0x080001f9   Thumb Code    44  _printf_pad.o(.text)
    _printf_post_padding                     0x08000225   Thumb Code    34  _printf_pad.o(.text)
    _printf_str                              0x08000247   Thumb Code    82  _printf_str.o(.text)
    _printf_int_hex                          0x08000299   Thumb Code    84  _printf_hex_int.o(.text)
    _printf_longlong_hex                     0x08000299   Thumb Code     0  _printf_hex_int.o(.text)
    __printf                                 0x080002f1   Thumb Code   306  __printf_flags_wp.o(.text)
    __aeabi_uidivmod                         0x08000429   Thumb Code    28  aeabi_sdivfast.o(.text)
    __aeabi_idivmod                          0x08000445   Thumb Code   472  aeabi_sdivfast.o(.text)
    __use_two_region_memory                  0x08000621   Thumb Code     2  heapauxi.o(.text)
    __rt_heap_escrow$2region                 0x08000623   Thumb Code     2  heapauxi.o(.text)
    __rt_heap_expand$2region                 0x08000625   Thumb Code     2  heapauxi.o(.text)
    __aeabi_d2f                              0x08000629   Thumb Code     0  d2f.o(.text)
    _d2f                                     0x08000629   Thumb Code   120  d2f.o(.text)
    __aeabi_dadd                             0x0800099d   Thumb Code     0  daddsub.o(.text)
    _dadd                                    0x0800099d   Thumb Code    26  daddsub.o(.text)
    __aeabi_dsub                             0x080009b7   Thumb Code     0  daddsub.o(.text)
    _dsub                                    0x080009b7   Thumb Code    22  daddsub.o(.text)
    __aeabi_drsub                            0x080009cd   Thumb Code     0  daddsub.o(.text)
    _drsb                                    0x080009cd   Thumb Code    28  daddsub.o(.text)
    __aeabi_ddiv                             0x080009fd   Thumb Code     0  ddiv.o(.text)
    _ddiv                                    0x080009fd   Thumb Code  1072  ddiv.o(.text)
    _drdiv                                   0x08000e2d   Thumb Code    20  ddiv.o(.text)
    __aeabi_d2iz                             0x08000e45   Thumb Code     0  dfixi.o(.text)
    _dfix                                    0x08000e45   Thumb Code    98  dfixi.o(.text)
    __aeabi_i2d_normalise                    0x08000eb1   Thumb Code    66  dflti.o(.text)
    __aeabi_i2d                              0x08000ef3   Thumb Code    16  dflti.o(.text)
    _dflt                                    0x08000ef3   Thumb Code     0  dflti.o(.text)
    __aeabi_ui2d                             0x08000f03   Thumb Code     6  dflti.o(.text)
    _dfltu                                   0x08000f03   Thumb Code     0  dflti.o(.text)
    __aeabi_dmul                             0x08000f09   Thumb Code     0  dmul.o(.text)
    _dmul                                    0x08000f09   Thumb Code   558  dmul.o(.text)
    __aeabi_f2d                              0x08001151   Thumb Code     0  f2d.o(.text)
    _f2d                                     0x08001151   Thumb Code    80  f2d.o(.text)
    __aeabi_i2f_normalise                    0x080011a5   Thumb Code    72  fflti.o(.text)
    __aeabi_i2f                              0x080011ed   Thumb Code    16  fflti.o(.text)
    _fflt                                    0x080011ed   Thumb Code     0  fflti.o(.text)
    __aeabi_ui2f                             0x080011fd   Thumb Code     6  fflti.o(.text)
    _ffltu                                   0x080011fd   Thumb Code     0  fflti.o(.text)
    __read_errno                             0x08001203   Thumb Code    10  _rserrno.o(.text)
    __set_errno                              0x0800120d   Thumb Code    12  _rserrno.o(.text)
    _printf_int_common                       0x08001219   Thumb Code   176  _printf_intcommon.o(.text)
    _printf_fp_dec_real                      0x08001465   Thumb Code   620  _printf_fp_dec.o(.text)
    _printf_char_common                      0x080016e7   Thumb Code    32  _printf_char_common.o(.text)
    _sputc                                   0x0800170d   Thumb Code    10  _sputc.o(.text)
    _printf_cs_common                        0x08001717   Thumb Code    22  _printf_char.o(.text)
    _printf_char                             0x0800172d   Thumb Code    16  _printf_char.o(.text)
    _printf_string                           0x0800173d   Thumb Code     8  _printf_char.o(.text)
    __ARM_scalbn                             0x08001745   Thumb Code    84  dscalbn.o(.text)
    __rt_locale                              0x080017a5   Thumb Code     8  rt_locale_intlibspace.o(.text)
    __aeabi_errno_addr                       0x080017ad   Thumb Code     8  rt_errno_addr_intlibspace.o(.text)
    __errno$intlibspace                      0x080017ad   Thumb Code     0  rt_errno_addr_intlibspace.o(.text)
    __rt_errno_addr$intlibspace              0x080017ad   Thumb Code     0  rt_errno_addr_intlibspace.o(.text)
    _ll_udiv10                               0x080017b5   Thumb Code   122  lludiv10.o(.text)
    _printf_fp_infnan                        0x08001831   Thumb Code   120  _printf_fp_infnan.o(.text)
    _btod_etento                             0x080018b9   Thumb Code   210  bigflt0.o(.text)
    _btod_d2e                                0x08001991   Thumb Code    64  btod.o(.text)
    _btod_emul                               0x08001dc5   Thumb Code    28  btod.o(.text)
    _btod_emuld                              0x08001de1   Thumb Code   144  btod.o(.text)
    _btod_ediv                               0x08001e71   Thumb Code    26  btod.o(.text)
    _btod_edivd                              0x08001e8b   Thumb Code   124  btod.o(.text)
    __rt_udiv10                              0x08001f11   Thumb Code    40  rtudiv10.o(.text)
    __fpl_dcmp_InfNaN                        0x08001f39   Thumb Code   154  dcmpin.o(.text)
    _dsqrt                                   0x08001fd9   Thumb Code   248  dsqrt.o(.text)
    __user_libspace                          0x080020d9   Thumb Code     8  libspace.o(.text)
    __user_perproc_libspace                  0x080020d9   Thumb Code     0  libspace.o(.text)
    __user_perthread_libspace                0x080020d9   Thumb Code     0  libspace.o(.text)
    __user_setup_stackheap                   0x080020e1   Thumb Code    62  sys_stackheap_outer.o(.text)
    exit                                     0x0800211f   Thumb Code    16  exit.o(.text)
    strcmp                                   0x08002131   Thumb Code   176  strcmpv6m.o(.text)
    __fpl_cmpreturn                          0x080021e1   Thumb Code    46  cmpret.o(.text)
    __fpl_dcheck_NaN2                        0x08002211   Thumb Code    14  dnan2.o(.text)
    __fpl_return_NaN                         0x08002225   Thumb Code    94  retnan.o(.text)
    _sys_exit                                0x08002285   Thumb Code     8  sys_exit.o(.text)
    __I$use$semihosting                      0x08002291   Thumb Code     0  use_no_semi.o(.text)
    __use_no_semihosting_swi                 0x08002291   Thumb Code     2  use_no_semi.o(.text)
    __decompress                             0x08002293   Thumb Code     0  __dczerorl2.o(.text)
    __decompress1                            0x08002293   Thumb Code    86  __dczerorl2.o(.text)
    __semihosting_library_function           0x08002293   Thumb Code     0  indicate_semi.o(.text)
    AHT20_Read                               0x080022e9   Thumb Code   132  bmp280+aht20.o(.text.AHT20_Read)
    BMP280_calc_values                       0x08002381   Thumb Code   888  bmp280+aht20.o(.text.BMP280_calc_values)
    BMP280_init                              0x08002749   Thumb Code   252  bmp280+aht20.o(.text.BMP280_init)
    HAL_Delay                                0x0800284d   Thumb Code    32  stm32f0xx_hal.o(.text.HAL_Delay)
    HAL_GPIO_Init                            0x08002871   Thumb Code   424  stm32f0xx_hal_gpio.o(.text.HAL_GPIO_Init)
    HAL_GetTick                              0x08002a31   Thumb Code     8  stm32f0xx_hal.o(.text.HAL_GetTick)
    HAL_I2CEx_ConfigAnalogFilter             0x08002a3d   Thumb Code    66  stm32f0xx_hal_i2c_ex.o(.text.HAL_I2CEx_ConfigAnalogFilter)
    HAL_I2CEx_ConfigDigitalFilter            0x08002a7f   Thumb Code    66  stm32f0xx_hal_i2c_ex.o(.text.HAL_I2CEx_ConfigDigitalFilter)
    HAL_I2C_Init                             0x08002ac1   Thumb Code   172  stm32f0xx_hal_i2c.o(.text.HAL_I2C_Init)
    HAL_I2C_Master_Receive                   0x08002b75   Thumb Code   400  stm32f0xx_hal_i2c.o(.text.HAL_I2C_Master_Receive)
    HAL_I2C_Master_Transmit                  0x08002d0d   Thumb Code   428  stm32f0xx_hal_i2c.o(.text.HAL_I2C_Master_Transmit)
    HAL_I2C_Mem_Read                         0x08002ecd   Thumb Code   532  stm32f0xx_hal_i2c.o(.text.HAL_I2C_Mem_Read)
    HAL_I2C_MspInit                          0x080030fd   Thumb Code    88  stm32f0xx_hal_msp.o(.text.HAL_I2C_MspInit)
    HAL_IncTick                              0x0800315d   Thumb Code    16  stm32f0xx_hal.o(.text.HAL_IncTick)
    HAL_Init                                 0x08003171   Thumb Code    28  stm32f0xx_hal.o(.text.HAL_Init)
    HAL_InitTick                             0x0800318d   Thumb Code    60  stm32f0xx_hal.o(.text.HAL_InitTick)
    HAL_MspInit                              0x080031cd   Thumb Code    40  stm32f0xx_hal_msp.o(.text.HAL_MspInit)
    HAL_NVIC_SetPriority                     0x080031f9   Thumb Code    48  stm32f0xx_hal_cortex.o(.text.HAL_NVIC_SetPriority)
    HAL_PWR_EnableBkUpAccess                 0x08003231   Thumb Code    16  stm32f0xx_hal_pwr.o(.text.HAL_PWR_EnableBkUpAccess)
    HAL_RCCEx_PeriphCLKConfig                0x08003241   Thumb Code   244  stm32f0xx_hal_rcc_ex.o(.text.HAL_RCCEx_PeriphCLKConfig)
    HAL_RCC_ClockConfig                      0x08003341   Thumb Code   296  stm32f0xx_hal_rcc.o(.text.HAL_RCC_ClockConfig)
    HAL_RCC_OscConfig                        0x08003489   Thumb Code  1028  stm32f0xx_hal_rcc.o(.text.HAL_RCC_OscConfig)
    HAL_RTC_GetDate                          0x08003899   Thumb Code    78  stm32f0xx_hal_rtc.o(.text.HAL_RTC_GetDate)
    HAL_RTC_GetTime                          0x080038e9   Thumb Code   104  stm32f0xx_hal_rtc.o(.text.HAL_RTC_GetTime)
    HAL_RTC_Init                             0x08003955   Thumb Code   244  stm32f0xx_hal_rtc.o(.text.HAL_RTC_Init)
    HAL_RTC_MspInit                          0x08003a4d   Thumb Code    24  stm32f0xx_hal_msp.o(.text.HAL_RTC_MspInit)
    HAL_RTC_SetDate                          0x08003a6d   Thumb Code   344  stm32f0xx_hal_rtc.o(.text.HAL_RTC_SetDate)
    HAL_RTC_SetTime                          0x08003bc5   Thumb Code   376  stm32f0xx_hal_rtc.o(.text.HAL_RTC_SetTime)
    HAL_SYSTICK_Config                       0x08003d45   Thumb Code    40  stm32f0xx_hal_cortex.o(.text.HAL_SYSTICK_Config)
    HardFault_Handler                        0x08003d79   Thumb Code     2  stm32f0xx_it.o(.text.HardFault_Handler)
    NMI_Handler                              0x080041f5   Thumb Code     2  stm32f0xx_it.o(.text.NMI_Handler)
    OLCD_write_string                        0x080041f9   Thumb Code   428  ssd1306.o(.text.OLCD_write_string)
    PendSV_Handler                           0x080043a9   Thumb Code     2  stm32f0xx_it.o(.text.PendSV_Handler)
    SVC_Handler                              0x080043ab   Thumb Code     2  stm32f0xx_it.o(.text.SVC_Handler)
    SysTick_Handler                          0x080043ad   Thumb Code     8  stm32f0xx_it.o(.text.SysTick_Handler)
    SystemClock_Config                       0x080043b5   Thumb Code   132  main.o(.text.SystemClock_Config)
    SystemInit                               0x08004441   Thumb Code     2  system_stm32f0xx.o(.text.SystemInit)
    clear_display                            0x08004445   Thumb Code   144  ssd1306.o(.text.clear_display)
    init_OLED                                0x080044d5   Thumb Code    48  ssd1306.o(.text.init_OLED)
    main                                     0x08004511   Thumb Code   568  main.o(.text.main)
    __aeabi_uidiv                            0x08004801   Thumb Code    68  aeabi_sdivfast.o(.text_divfast)
    __aeabi_idiv                             0x08004845   Thumb Code   434  aeabi_sdivfast.o(.text_divfast)
    __ARM_common_ll_muluu                    0x080049f7   Thumb Code    48  btod.o(i.__ARM_common_ll_muluu)
    __ARM_fpclassify                         0x08004a29   Thumb Code    40  fpclassify.o(i.__ARM_fpclassify)
    __kernel_poly                            0x08004a55   Thumb Code   172  poly.o(i.__kernel_poly)
    __mathlib_dbl_divzero                    0x08004b01   Thumb Code    16  dunder.o(i.__mathlib_dbl_divzero)
    __mathlib_dbl_infnan2                    0x08004b15   Thumb Code     8  dunder.o(i.__mathlib_dbl_infnan2)
    __mathlib_dbl_invalid                    0x08004b1d   Thumb Code    16  dunder.o(i.__mathlib_dbl_invalid)
    __mathlib_dbl_overflow                   0x08004b2d   Thumb Code    16  dunder.o(i.__mathlib_dbl_overflow)
    __mathlib_dbl_underflow                  0x08004b41   Thumb Code    14  dunder.o(i.__mathlib_dbl_underflow)
    _is_digit                                0x08004b55   Thumb Code    14  __printf_wp.o(i._is_digit)
    pow                                      0x08004b65   Thumb Code  2506  pow.o(i.pow)
    sqrt                                     0x08005539   Thumb Code    66  sqrt.o(i.sqrt)
    _get_lc_numeric                          0x08005581   Thumb Code    44  lc_numeric_c.o(locale$$code)
    __aeabi_cdrcmple                         0x080055ad   Thumb Code     0  drlef.o(x$fpl$drleqf)
    _drcmple                                 0x080055ad   Thumb Code   100  drlef.o(x$fpl$drleqf)
    __aeabi_fadd                             0x08005615   Thumb Code     0  faddsub.o(x$fpl$fadd)
    _fadd                                    0x08005615   Thumb Code   134  faddsub.o(x$fpl$fadd)
    __aeabi_fmul                             0x080056a1   Thumb Code     0  fmul.o(x$fpl$fmul)
    _fmul                                    0x080056a1   Thumb Code   172  fmul.o(x$fpl$fmul)
    __aeabi_fsub                             0x08005751   Thumb Code     0  faddsub.o(x$fpl$fsub)
    _fsub                                    0x08005751   Thumb Code   204  faddsub.o(x$fpl$fsub)
    _printf_fp_dec                           0x08005821   Thumb Code    16  printf1.o(x$fpl$printf1)
    __I$use$fp                               0x08005830   Number         0  usenofp.o(x$fpl$usenofp)
    __mathlib_zero                           0x08005978   Data           8  qnan.o(.constdata)
    AHBPrescTable                            0x08005a14   Data          16  system_stm32f0xx.o(.rodata.AHBPrescTable)
    Region$$Table$$Base                      0x08005a68   Number         0  anon$$obj.o(Region$$Table)
    Region$$Table$$Limit                     0x08005a88   Number         0  anon$$obj.o(Region$$Table)
    day_zone                                 0x20000000   Data           8  main.o(.data..L_MergedGlobals)
    display_time                             0x20000008   Data          16  main.o(.data..L_MergedGlobals)
    day_name                                 0x20000018   Data          32  main.o(.data..L_MergedGlobals)
    uwTickFreq                               0x20000038   Data           1  stm32f0xx_hal.o(.data..L_MergedGlobals)
    uwTickPrio                               0x2000003c   Data           4  stm32f0xx_hal.o(.data..L_MergedGlobals)
    OLED_init                                0x20000040   Data          30  ssd1306.o(.data.OLED_init)
    SystemCoreClock                          0x20000060   Data           4  system_stm32f0xx.o(.data.SystemCoreClock)
    myFont                                   0x20000064   Data         760  ssd1306.o(.data.myFont)
    __libspace_start                         0x20000360   Data          96  libspace.o(.bss)
    __temporary_stack_top$libspace           0x200003c0   Data           0  libspace.o(.bss)
    chipID                                   0x200003c0   Data           1  bmp280+aht20.o(.bss..L_MergedGlobals)
    dig_T1                                   0x200003c2   Data           2  bmp280+aht20.o(.bss..L_MergedGlobals)
    dig_T2                                   0x200003c4   Data           2  bmp280+aht20.o(.bss..L_MergedGlobals)
    dig_T3                                   0x200003c6   Data           2  bmp280+aht20.o(.bss..L_MergedGlobals)
    dig_P1                                   0x200003c8   Data           2  bmp280+aht20.o(.bss..L_MergedGlobals)
    dig_P2                                   0x200003ca   Data           2  bmp280+aht20.o(.bss..L_MergedGlobals)
    dig_P3                                   0x200003cc   Data           2  bmp280+aht20.o(.bss..L_MergedGlobals)
    dig_P4                                   0x200003ce   Data           2  bmp280+aht20.o(.bss..L_MergedGlobals)
    dig_P5                                   0x200003d0   Data           2  bmp280+aht20.o(.bss..L_MergedGlobals)
    dig_P6                                   0x200003d2   Data           2  bmp280+aht20.o(.bss..L_MergedGlobals)
    dig_P7                                   0x200003d4   Data           2  bmp280+aht20.o(.bss..L_MergedGlobals)
    dig_P8                                   0x200003d6   Data           2  bmp280+aht20.o(.bss..L_MergedGlobals)
    dig_P9                                   0x200003d8   Data           2  bmp280+aht20.o(.bss..L_MergedGlobals)
    temperature_raw                          0x200003dc   Data           4  bmp280+aht20.o(.bss..L_MergedGlobals)
    pressure_raw                             0x200003e0   Data           4  bmp280+aht20.o(.bss..L_MergedGlobals)
    BMP280_Temperature                       0x200003e4   Data           4  bmp280+aht20.o(.bss..L_MergedGlobals)
    BMP280_Pressure                          0x200003e8   Data           4  bmp280+aht20.o(.bss..L_MergedGlobals)
    BMP280_Altitude                          0x200003ec   Data           4  bmp280+aht20.o(.bss..L_MergedGlobals)
    AHT20_Temperature                        0x200003f0   Data           4  bmp280+aht20.o(.bss..L_MergedGlobals)
    AHT20_Humidity                           0x200003f4   Data           4  bmp280+aht20.o(.bss..L_MergedGlobals)
    sDate                                    0x200003f8   Data           4  main.o(.bss..L_MergedGlobals.16)
    display_Sensor_Data                      0x200003fc   Data          16  main.o(.bss..L_MergedGlobals.16)
    sTime                                    0x2000040c   Data          20  main.o(.bss..L_MergedGlobals.16)
    hrtc                                     0x20000420   Data          32  main.o(.bss..L_MergedGlobals.16)
    data_stream                              0x20000440   Data           3  ssd1306.o(.bss.data_stream)
    hi2c1                                    0x20000444   Data          84  main.o(.bss.hi2c1)
    uwTick                                   0x20000498   Data           4  stm32f0xx_hal.o(.bss.uwTick)



==============================================================================

Memory Map of the image

  Image Entry point : 0x080000b9

  Load Region LR_IROM1 (Base: 0x08000000, Size: 0x00005e08, Max: 0x00040000, ABSOLUTE, COMPRESSED[0x00005d00])

    Execution Region ER_IROM1 (Exec base: 0x08000000, Load base: 0x08000000, Size: 0x00005aa4, Max: 0x00040000, ABSOLUTE)

    Exec Addr    Load Addr    Size         Type   Attr      Idx    E Section Name        Object

    0x08000000   0x08000000   0x000000b8   Data   RO            3    RESET               startup_stm32f030xc.o
    0x080000b8   0x080000b8   0x00000008   Code   RO          800  * !!!main             c_p.l(__main.o)
    0x080000c0   0x080000c0   0x00000054   Code   RO         1100    !!!scatter          c_p.l(__scatter.o)
    0x08000114   0x08000114   0x00000002   Code   RO         1101    !!handler_null      c_p.l(__scatter.o)
    0x08000116   0x08000116   0x00000002   PAD
    0x08000118   0x08000118   0x0000001c   Code   RO         1104    !!handler_zi        c_p.l(__scatter_zi.o)
    0x08000134   0x08000134   0x00000002   Code   RO          789    .ARM.Collect$$_printf_percent$$00000000  c_p.l(_printf_percent.o)
    0x08000136   0x08000136   0x0000000a   Code   RO          788    .ARM.Collect$$_printf_percent$$00000003  c_p.l(_printf_f.o)
    0x08000140   0x08000140   0x0000000a   Code   RO          787    .ARM.Collect$$_printf_percent$$0000000C  c_p.l(_printf_x.o)
    0x0800014a   0x0800014a   0x0000000a   Code   RO          785    .ARM.Collect$$_printf_percent$$00000013  c_p.l(_printf_c.o)
    0x08000154   0x08000154   0x0000000a   Code   RO          786    .ARM.Collect$$_printf_percent$$00000014  c_p.l(_printf_s.o)
    0x0800015e   0x0800015e   0x00000004   Code   RO          853    .ARM.Collect$$_printf_percent$$00000017  c_p.l(_printf_percent_end.o)
    0x08000162   0x08000162   0x00000002   Code   RO          956    .ARM.Collect$$libinit$$00000000  c_p.l(libinit.o)
    0x08000164   0x08000164   0x00000000   Code   RO          958    .ARM.Collect$$libinit$$00000002  c_p.l(libinit2.o)
    0x08000164   0x08000164   0x00000000   Code   RO          960    .ARM.Collect$$libinit$$00000004  c_p.l(libinit2.o)
    0x08000164   0x08000164   0x00000000   Code   RO          962    .ARM.Collect$$libinit$$00000006  c_p.l(libinit2.o)
    0x08000164   0x08000164   0x00000000   Code   RO          965    .ARM.Collect$$libinit$$0000000C  c_p.l(libinit2.o)
    0x08000164   0x08000164   0x00000000   Code   RO          967    .ARM.Collect$$libinit$$0000000E  c_p.l(libinit2.o)
    0x08000164   0x08000164   0x00000000   Code   RO          969    .ARM.Collect$$libinit$$00000010  c_p.l(libinit2.o)
    0x08000164   0x08000164   0x00000006   Code   RO          970    .ARM.Collect$$libinit$$00000011  c_p.l(libinit2.o)
    0x0800016a   0x0800016a   0x00000000   Code   RO          972    .ARM.Collect$$libinit$$00000013  c_p.l(libinit2.o)
    0x0800016a   0x0800016a   0x00000000   Code   RO          974    .ARM.Collect$$libinit$$00000015  c_p.l(libinit2.o)
    0x0800016a   0x0800016a   0x00000000   Code   RO          976    .ARM.Collect$$libinit$$00000017  c_p.l(libinit2.o)
    0x0800016a   0x0800016a   0x0000000a   Code   RO          977    .ARM.Collect$$libinit$$00000018  c_p.l(libinit2.o)
    0x08000174   0x08000174   0x00000000   Code   RO          978    .ARM.Collect$$libinit$$00000019  c_p.l(libinit2.o)
    0x08000174   0x08000174   0x00000000   Code   RO          980    .ARM.Collect$$libinit$$0000001B  c_p.l(libinit2.o)
    0x08000174   0x08000174   0x00000000   Code   RO          982    .ARM.Collect$$libinit$$0000001D  c_p.l(libinit2.o)
    0x08000174   0x08000174   0x00000000   Code   RO          984    .ARM.Collect$$libinit$$0000001F  c_p.l(libinit2.o)
    0x08000174   0x08000174   0x00000000   Code   RO          986    .ARM.Collect$$libinit$$00000021  c_p.l(libinit2.o)
    0x08000174   0x08000174   0x00000000   Code   RO          988    .ARM.Collect$$libinit$$00000023  c_p.l(libinit2.o)
    0x08000174   0x08000174   0x00000000   Code   RO          990    .ARM.Collect$$libinit$$00000025  c_p.l(libinit2.o)
    0x08000174   0x08000174   0x00000000   Code   RO          992    .ARM.Collect$$libinit$$00000027  c_p.l(libinit2.o)
    0x08000174   0x08000174   0x00000000   Code   RO          996    .ARM.Collect$$libinit$$0000002E  c_p.l(libinit2.o)
    0x08000174   0x08000174   0x00000000   Code   RO          998    .ARM.Collect$$libinit$$00000030  c_p.l(libinit2.o)
    0x08000174   0x08000174   0x00000000   Code   RO         1000    .ARM.Collect$$libinit$$00000032  c_p.l(libinit2.o)
    0x08000174   0x08000174   0x00000000   Code   RO         1002    .ARM.Collect$$libinit$$00000034  c_p.l(libinit2.o)
    0x08000174   0x08000174   0x00000002   Code   RO         1003    .ARM.Collect$$libinit$$00000035  c_p.l(libinit2.o)
    0x08000176   0x08000176   0x00000002   Code   RO         1063    .ARM.Collect$$libshutdown$$00000000  c_p.l(libshutdown.o)
    0x08000178   0x08000178   0x00000000   Code   RO         1081    .ARM.Collect$$libshutdown$$00000002  c_p.l(libshutdown2.o)
    0x08000178   0x08000178   0x00000000   Code   RO         1083    .ARM.Collect$$libshutdown$$00000004  c_p.l(libshutdown2.o)
    0x08000178   0x08000178   0x00000000   Code   RO         1086    .ARM.Collect$$libshutdown$$00000007  c_p.l(libshutdown2.o)
    0x08000178   0x08000178   0x00000000   Code   RO         1089    .ARM.Collect$$libshutdown$$0000000A  c_p.l(libshutdown2.o)
    0x08000178   0x08000178   0x00000000   Code   RO         1091    .ARM.Collect$$libshutdown$$0000000C  c_p.l(libshutdown2.o)
    0x08000178   0x08000178   0x00000000   Code   RO         1094    .ARM.Collect$$libshutdown$$0000000F  c_p.l(libshutdown2.o)
    0x08000178   0x08000178   0x00000002   Code   RO         1095    .ARM.Collect$$libshutdown$$00000010  c_p.l(libshutdown2.o)
    0x0800017a   0x0800017a   0x00000000   Code   RO          834    .ARM.Collect$$rtentry$$00000000  c_p.l(__rtentry.o)
    0x0800017a   0x0800017a   0x00000000   Code   RO          883    .ARM.Collect$$rtentry$$00000002  c_p.l(__rtentry2.o)
    0x0800017a   0x0800017a   0x00000006   Code   RO          895    .ARM.Collect$$rtentry$$00000004  c_p.l(__rtentry4.o)
    0x08000180   0x08000180   0x00000000   Code   RO          885    .ARM.Collect$$rtentry$$00000009  c_p.l(__rtentry2.o)
    0x08000180   0x08000180   0x00000004   Code   RO          886    .ARM.Collect$$rtentry$$0000000A  c_p.l(__rtentry2.o)
    0x08000184   0x08000184   0x00000000   Code   RO          888    .ARM.Collect$$rtentry$$0000000C  c_p.l(__rtentry2.o)
    0x08000184   0x08000184   0x00000008   Code   RO          889    .ARM.Collect$$rtentry$$0000000D  c_p.l(__rtentry2.o)
    0x0800018c   0x0800018c   0x00000002   Code   RO         1009    .ARM.Collect$$rtexit$$00000000  c_p.l(rtexit.o)
    0x0800018e   0x0800018e   0x00000000   Code   RO         1028    .ARM.Collect$$rtexit$$00000002  c_p.l(rtexit2.o)
    0x0800018e   0x0800018e   0x00000004   Code   RO         1029    .ARM.Collect$$rtexit$$00000003  c_p.l(rtexit2.o)
    0x08000192   0x08000192   0x00000006   Code   RO         1030    .ARM.Collect$$rtexit$$00000004  c_p.l(rtexit2.o)
    0x08000198   0x08000198   0x00000038   Code   RO            4    .text               startup_stm32f030xc.o
    0x080001d0   0x080001d0   0x00000028   Code   RO          736    .text               c_p.l(noretval__2sprintf.o)
    0x080001f8   0x080001f8   0x0000004e   Code   RO          740    .text               c_p.l(_printf_pad.o)
    0x08000246   0x08000246   0x00000052   Code   RO          742    .text               c_p.l(_printf_str.o)
    0x08000298   0x08000298   0x00000058   Code   RO          747    .text               c_p.l(_printf_hex_int.o)
    0x080002f0   0x080002f0   0x00000138   Code   RO          777    .text               c_p.l(__printf_flags_wp.o)
    0x08000428   0x08000428   0x000001f8   Code   RO          790    .text               c_p.l(aeabi_sdivfast.o)
    0x08000620   0x08000620   0x00000006   Code   RO          798    .text               c_p.l(heapauxi.o)
    0x08000626   0x08000626   0x00000002   PAD
    0x08000628   0x08000628   0x0000007c   Code   RO          802    .text               fz_ps.l(d2f.o)
    0x080006a4   0x080006a4   0x00000358   Code   RO          804    .text               fz_ps.l(daddsub.o)
    0x080009fc   0x080009fc   0x00000448   Code   RO          806    .text               fz_ps.l(ddiv.o)
    0x08000e44   0x08000e44   0x0000006c   Code   RO          809    .text               fz_ps.l(dfixi.o)
    0x08000eb0   0x08000eb0   0x00000058   Code   RO          811    .text               fz_ps.l(dflti.o)
    0x08000f08   0x08000f08   0x00000248   Code   RO          813    .text               fz_ps.l(dmul.o)
    0x08001150   0x08001150   0x00000054   Code   RO          815    .text               fz_ps.l(f2d.o)
    0x080011a4   0x080011a4   0x0000005e   Code   RO          823    .text               fz_ps.l(fflti.o)
    0x08001202   0x08001202   0x00000016   Code   RO          839    .text               c_p.l(_rserrno.o)
    0x08001218   0x08001218   0x000000b0   Code   RO          841    .text               c_p.l(_printf_intcommon.o)
    0x080012c8   0x080012c8   0x00000414   Code   RO          843    .text               c_p.l(_printf_fp_dec.o)
    0x080016dc   0x080016dc   0x00000030   Code   RO          847    .text               c_p.l(_printf_char_common.o)
    0x0800170c   0x0800170c   0x0000000a   Code   RO          849    .text               c_p.l(_sputc.o)
    0x08001716   0x08001716   0x0000002e   Code   RO          851    .text               c_p.l(_printf_char.o)
    0x08001744   0x08001744   0x00000060   Code   RO          856    .text               fz_ps.l(dscalbn.o)
    0x080017a4   0x080017a4   0x00000008   Code   RO          902    .text               c_p.l(rt_locale_intlibspace.o)
    0x080017ac   0x080017ac   0x00000008   Code   RO          907    .text               c_p.l(rt_errno_addr_intlibspace.o)
    0x080017b4   0x080017b4   0x0000007a   Code   RO          909    .text               c_p.l(lludiv10.o)
    0x0800182e   0x0800182e   0x00000002   PAD
    0x08001830   0x08001830   0x00000088   Code   RO          911    .text               c_p.l(_printf_fp_infnan.o)
    0x080018b8   0x080018b8   0x000000d8   Code   RO          915    .text               c_p.l(bigflt0.o)
    0x08001990   0x08001990   0x00000580   Code   RO          918    .text               c_p.l(btod.o)
    0x08001f10   0x08001f10   0x00000028   Code   RO          927    .text               c_p.l(rtudiv10.o)
    0x08001f38   0x08001f38   0x000000a0   Code   RO          929    .text               fz_ps.l(dcmpin.o)
    0x08001fd8   0x08001fd8   0x00000100   Code   RO          931    .text               fz_ps.l(dsqrt.o)
    0x080020d8   0x080020d8   0x00000008   Code   RO          935    .text               c_p.l(libspace.o)
    0x080020e0   0x080020e0   0x0000003e   Code   RO          938    .text               c_p.l(sys_stackheap_outer.o)
    0x0800211e   0x0800211e   0x00000010   Code   RO          943    .text               c_p.l(exit.o)
    0x0800212e   0x0800212e   0x00000002   PAD
    0x08002130   0x08002130   0x000000b0   Code   RO          949    .text               c_p.l(strcmpv6m.o)
    0x080021e0   0x080021e0   0x0000002e   Code   RO         1004    .text               fz_ps.l(cmpret.o)
    0x0800220e   0x0800220e   0x00000002   PAD
    0x08002210   0x08002210   0x00000014   Code   RO         1006    .text               fz_ps.l(dnan2.o)
    0x08002224   0x08002224   0x0000005e   Code   RO         1021    .text               fz_ps.l(retnan.o)
    0x08002282   0x08002282   0x00000002   PAD
    0x08002284   0x08002284   0x0000000c   Code   RO         1023    .text               c_p.l(sys_exit.o)
    0x08002290   0x08002290   0x00000002   Code   RO         1050    .text               c_p.l(use_no_semi.o)
    0x08002292   0x08002292   0x00000000   Code   RO         1052    .text               c_p.l(indicate_semi.o)
    0x08002292   0x08002292   0x00000056   Code   RO         1098    .text               c_p.l(__dczerorl2.o)
    0x080022e8   0x080022e8   0x00000098   Code   RO           73    .text.AHT20_Read    bmp280+aht20.o
    0x08002380   0x08002380   0x000003c8   Code   RO           69    .text.BMP280_calc_values  bmp280+aht20.o
    0x08002748   0x08002748   0x00000104   Code   RO           65    .text.BMP280_init   bmp280+aht20.o
    0x0800284c   0x0800284c   0x00000024   Code   RO          350    .text.HAL_Delay     stm32f0xx_hal.o
    0x08002870   0x08002870   0x000001c0   Code   RO          386    .text.HAL_GPIO_Init  stm32f0xx_hal_gpio.o
    0x08002a30   0x08002a30   0x0000000c   Code   RO          342    .text.HAL_GetTick   stm32f0xx_hal.o
    0x08002a3c   0x08002a3c   0x00000042   Code   RO          265    .text.HAL_I2CEx_ConfigAnalogFilter  stm32f0xx_hal_i2c_ex.o
    0x08002a7e   0x08002a7e   0x00000042   Code   RO          267    .text.HAL_I2CEx_ConfigDigitalFilter  stm32f0xx_hal_i2c_ex.o
    0x08002ac0   0x08002ac0   0x000000b4   Code   RO          111    .text.HAL_I2C_Init  stm32f0xx_hal_i2c.o
    0x08002b74   0x08002b74   0x00000198   Code   RO          127    .text.HAL_I2C_Master_Receive  stm32f0xx_hal_i2c.o
    0x08002d0c   0x08002d0c   0x000001c0   Code   RO          119    .text.HAL_I2C_Master_Transmit  stm32f0xx_hal_i2c.o
    0x08002ecc   0x08002ecc   0x00000230   Code   RO          171    .text.HAL_I2C_Mem_Read  stm32f0xx_hal_i2c.o
    0x080030fc   0x080030fc   0x00000060   Code   RO           49    .text.HAL_I2C_MspInit  stm32f0xx_hal_msp.o
    0x0800315c   0x0800315c   0x00000014   Code   RO          340    .text.HAL_IncTick   stm32f0xx_hal.o
    0x08003170   0x08003170   0x0000001c   Code   RO          330    .text.HAL_Init      stm32f0xx_hal.o
    0x0800318c   0x0800318c   0x00000040   Code   RO          332    .text.HAL_InitTick  stm32f0xx_hal.o
    0x080031cc   0x080031cc   0x0000002c   Code   RO           47    .text.HAL_MspInit   stm32f0xx_hal_msp.o
    0x080031f8   0x080031f8   0x00000038   Code   RO          442    .text.HAL_NVIC_SetPriority  stm32f0xx_hal_cortex.o
    0x08003230   0x08003230   0x00000010   Code   RO          476    .text.HAL_PWR_EnableBkUpAccess  stm32f0xx_hal_pwr.o
    0x08003240   0x08003240   0x00000100   Code   RO          316    .text.HAL_RCCEx_PeriphCLKConfig  stm32f0xx_hal_rcc_ex.o
    0x08003340   0x08003340   0x00000148   Code   RO          285    .text.HAL_RCC_ClockConfig  stm32f0xx_hal_rcc.o
    0x08003488   0x08003488   0x00000410   Code   RO          283    .text.HAL_RCC_OscConfig  stm32f0xx_hal_rcc.o
    0x08003898   0x08003898   0x0000004e   Code   RO          610    .text.HAL_RTC_GetDate  stm32f0xx_hal_rtc.o
    0x080038e6   0x080038e6   0x00000002   PAD
    0x080038e8   0x080038e8   0x0000006c   Code   RO          604    .text.HAL_RTC_GetTime  stm32f0xx_hal_rtc.o
    0x08003954   0x08003954   0x000000f8   Code   RO          588    .text.HAL_RTC_Init  stm32f0xx_hal_rtc.o
    0x08003a4c   0x08003a4c   0x00000020   Code   RO           53    .text.HAL_RTC_MspInit  stm32f0xx_hal_msp.o
    0x08003a6c   0x08003a6c   0x00000158   Code   RO          608    .text.HAL_RTC_SetDate  stm32f0xx_hal_rtc.o
    0x08003bc4   0x08003bc4   0x00000180   Code   RO          600    .text.HAL_RTC_SetTime  stm32f0xx_hal_rtc.o
    0x08003d44   0x08003d44   0x00000034   Code   RO          450    .text.HAL_SYSTICK_Config  stm32f0xx_hal_cortex.o
    0x08003d78   0x08003d78   0x00000002   Code   RO           32    .text.HardFault_Handler  stm32f0xx_it.o
    0x08003d7a   0x08003d7a   0x00000002   PAD
    0x08003d7c   0x08003d7c   0x0000017c   Code   RO          255    .text.I2C_IsErrorOccurred  stm32f0xx_hal_i2c.o
    0x08003ef8   0x08003ef8   0x000000fa   Code   RO          121    .text.I2C_WaitOnFlagUntilTimeout  stm32f0xx_hal_i2c.o
    0x08003ff2   0x08003ff2   0x00000002   PAD
    0x08003ff4   0x08003ff4   0x000000d4   Code   RO          129    .text.I2C_WaitOnRXNEFlagUntilTimeout  stm32f0xx_hal_i2c.o
    0x080040c8   0x080040c8   0x00000086   Code   RO          125    .text.I2C_WaitOnSTOPFlagUntilTimeout  stm32f0xx_hal_i2c.o
    0x0800414e   0x0800414e   0x000000a6   Code   RO          123    .text.I2C_WaitOnTXISFlagUntilTimeout  stm32f0xx_hal_i2c.o
    0x080041f4   0x080041f4   0x00000002   Code   RO           30    .text.NMI_Handler   stm32f0xx_it.o
    0x080041f6   0x080041f6   0x00000002   PAD
    0x080041f8   0x080041f8   0x000001b0   Code   RO           98    .text.OLCD_write_string  ssd1306.o
    0x080043a8   0x080043a8   0x00000002   Code   RO           36    .text.PendSV_Handler  stm32f0xx_it.o
    0x080043aa   0x080043aa   0x00000002   Code   RO           34    .text.SVC_Handler   stm32f0xx_it.o
    0x080043ac   0x080043ac   0x00000008   Code   RO           38    .text.SysTick_Handler  stm32f0xx_it.o
    0x080043b4   0x080043b4   0x0000008c   Code   RO           13    .text.SystemClock_Config  main.o
    0x08004440   0x08004440   0x00000002   Code   RO          716    .text.SystemInit    system_stm32f0xx.o
    0x08004442   0x08004442   0x00000002   PAD
    0x08004444   0x08004444   0x00000090   Code   RO           96    .text.clear_display  ssd1306.o
    0x080044d4   0x080044d4   0x0000003c   Code   RO           84    .text.init_OLED     ssd1306.o
    0x08004510   0x08004510   0x000002f0   Code   RO           11    .text.main          main.o
    0x08004800   0x08004800   0x000001f6   Code   RO          791    .text_divfast       c_p.l(aeabi_sdivfast.o)
    0x080049f6   0x080049f6   0x00000030   Code   RO          920    i.__ARM_common_ll_muluu  c_p.l(btod.o)
    0x08004a26   0x08004a26   0x00000002   PAD
    0x08004a28   0x08004a28   0x0000002c   Code   RO          873    i.__ARM_fpclassify  m_ps.l(fpclassify.o)
    0x08004a54   0x08004a54   0x000000ac   Code   RO          875    i.__kernel_poly     m_ps.l(poly.o)
    0x08004b00   0x08004b00   0x00000014   Code   RO          859    i.__mathlib_dbl_divzero  m_ps.l(dunder.o)
    0x08004b14   0x08004b14   0x00000008   Code   RO          861    i.__mathlib_dbl_infnan2  m_ps.l(dunder.o)
    0x08004b1c   0x08004b1c   0x00000010   Code   RO          862    i.__mathlib_dbl_invalid  m_ps.l(dunder.o)
    0x08004b2c   0x08004b2c   0x00000014   Code   RO          863    i.__mathlib_dbl_overflow  m_ps.l(dunder.o)
    0x08004b40   0x08004b40   0x00000014   Code   RO          865    i.__mathlib_dbl_underflow  m_ps.l(dunder.o)
    0x08004b54   0x08004b54   0x0000000e   Code   RO          775    i._is_digit         c_p.l(__printf_wp.o)
    0x08004b62   0x08004b62   0x00000002   PAD
    0x08004b64   0x08004b64   0x000009d4   Code   RO          830    i.pow               m_ps.l(pow.o)
    0x08005538   0x08005538   0x00000048   Code   RO          879    i.sqrt              m_ps.l(sqrt.o)
    0x08005580   0x08005580   0x0000002c   Code   RO          925    locale$$code        c_p.l(lc_numeric_c.o)
    0x080055ac   0x080055ac   0x00000068   Code   RO          854    x$fpl$drleqf        fz_ps.l(drlef.o)
    0x08005614   0x08005614   0x0000008c   Code   RO          817    x$fpl$fadd          fz_ps.l(faddsub.o)
    0x080056a0   0x080056a0   0x000000b0   Code   RO          825    x$fpl$fmul          fz_ps.l(fmul.o)
    0x08005750   0x08005750   0x000000d0   Code   RO          819    x$fpl$fsub          fz_ps.l(faddsub.o)
    0x08005820   0x08005820   0x00000010   Code   RO          827    x$fpl$printf1       fz_ps.l(printf1.o)
    0x08005830   0x08005830   0x00000000   Code   RO          858    x$fpl$usenofp       fz_ps.l(usenofp.o)
    0x08005830   0x08005830   0x00000028   Data   RO          748    .constdata          c_p.l(_printf_hex_int.o)
    0x08005858   0x08005858   0x00000011   Data   RO          778    .constdata          c_p.l(__printf_flags_wp.o)
    0x08005869   0x08005869   0x00000080   Data   RO          807    .constdata          fz_ps.l(ddiv.o)
    0x080058e9   0x080058e9   0x00000007   PAD
    0x080058f0   0x080058f0   0x00000088   Data   RO          831    .constdata          m_ps.l(pow.o)
    0x08005978   0x08005978   0x00000008   Data   RO          877    .constdata          m_ps.l(qnan.o)
    0x08005980   0x08005980   0x00000094   Data   RO          916    .constdata          c_p.l(bigflt0.o)
    0x08005a14   0x08005a14   0x00000010   Data   RO          721    .rodata.AHBPrescTable  system_stm32f0xx.o
    0x08005a24   0x08005a24   0x00000020   Data   RO          307    .rodata.cst16       stm32f0xx_hal_rcc.o
    0x08005a44   0x08005a44   0x00000022   Data   RO           17    .rodata.str1.1      main.o
    0x08005a66   0x08005a66   0x00000002   PAD
    0x08005a68   0x08005a68   0x00000020   Data   RO         1097    Region$$Table       anon$$obj.o
    0x08005a88   0x08005a88   0x0000001c   Data   RO          924    locale$$data        c_p.l(lc_numeric_c.o)


    Execution Region RW_IRAM1 (Exec base: 0x20000000, Load base: 0x08005aa8, Size: 0x00000aa0, Max: 0x00008000, ABSOLUTE, COMPRESSED[0x00000258])

    Exec Addr    Load Addr    Size         Type   Attr      Idx    E Section Name        Object

    0x20000000   COMPRESSED   0x00000038   Data   RW           20    .data..L_MergedGlobals  main.o
    0x20000038   COMPRESSED   0x00000008   Data   RW          377    .data..L_MergedGlobals  stm32f0xx_hal.o
    0x20000040   COMPRESSED   0x0000001e   Data   RW          101    .data.OLED_init     ssd1306.o
    0x2000005e   COMPRESSED   0x00000002   PAD
    0x20000060   COMPRESSED   0x00000004   Data   RW          720    .data.SystemCoreClock  system_stm32f0xx.o
    0x20000064   COMPRESSED   0x000002f8   Data   RW          100    .data.myFont        ssd1306.o
    0x2000035c   COMPRESSED   0x00000004   PAD
    0x20000360        -       0x00000060   Zero   RW          936    .bss                c_p.l(libspace.o)
    0x200003c0        -       0x00000038   Zero   RW           75    .bss..L_MergedGlobals  bmp280+aht20.o
    0x200003f8        -       0x00000048   Zero   RW           21    .bss..L_MergedGlobals.16  main.o
    0x20000440        -       0x00000003   Zero   RW          102    .bss.data_stream    ssd1306.o
    0x20000443   COMPRESSED   0x00000001   PAD
    0x20000444        -       0x00000054   Zero   RW           18    .bss.hi2c1          main.o
    0x20000498        -       0x00000004   Zero   RW          376    .bss.uwTick         stm32f0xx_hal.o
    0x2000049c   COMPRESSED   0x00000004   PAD
    0x200004a0        -       0x00000200   Zero   RW            2    HEAP                startup_stm32f030xc.o
    0x200006a0        -       0x00000400   Zero   RW            1    STACK               startup_stm32f030xc.o


==============================================================================

Image component sizes


      Code (inc. data)   RO Data    RW Data    ZI Data      Debug   Object Name

      1380        108          0          0         56       4562   bmp280+aht20.o
       892        192         34         56        156       8423   main.o
       636         16          0        790          3       5141   ssd1306.o
        56         26        184          0       1536        636   startup_stm32f030xc.o
       160         16          0          8          4       5302   stm32f0xx_hal.o
       108         20          0          0          0       5449   stm32f0xx_hal_cortex.o
       448         24          0          0          0       4981   stm32f0xx_hal_gpio.o
      2738         68          0          0          0      66918   stm32f0xx_hal_i2c.o
       132          0          0          0          0       4902   stm32f0xx_hal_i2c_ex.o
       172         20          0          0          0       6088   stm32f0xx_hal_msp.o
        16          0          0          0          0       3035   stm32f0xx_hal_pwr.o
      1368         44         32          0          0       7599   stm32f0xx_hal_rcc.o
       256         12          0          0          0       3256   stm32f0xx_hal_rcc_ex.o
      1162         16          0          0          0      16361   stm32f0xx_hal_rtc.o
        16          0          0          0          0        719   stm32f0xx_it.o
         2          0         16          4          0       1707   system_stm32f0xx.o

    ----------------------------------------------------------------------
      9552        562        300        860       1764     145079   Object Totals
         0          0         32          0          0          0   (incl. Generated)
        10          0          2          2          9          0   (incl. Padding)

    ----------------------------------------------------------------------

      Code (inc. data)   RO Data    RW Data    ZI Data      Debug   Library Member Name

        86          0          0          0          0          0   __dczerorl2.o
         8          0          0          0          0         68   __main.o
       312          6         17          0          0         76   __printf_flags_wp.o
        14          0          0          0          0         60   __printf_wp.o
         0          0          0          0          0          0   __rtentry.o
        12          0          0          0          0          0   __rtentry2.o
         6          0          0          0          0          0   __rtentry4.o
        86         10          0          0          0          0   __scatter.o
        28          0          0          0          0          0   __scatter_zi.o
        10          0          0          0          0          0   _printf_c.o
        46          0          0          0          0        100   _printf_char.o
        48          6          0          0          0         88   _printf_char_common.o
        10          0          0          0          0          0   _printf_f.o
      1044         12          0          0          0        116   _printf_fp_dec.o
       136         16          0          0          0         76   _printf_fp_infnan.o
        88          4         40          0          0         72   _printf_hex_int.o
       176          0          0          0          0         84   _printf_intcommon.o
        78          0          0          0          0        100   _printf_pad.o
         2          0          0          0          0          0   _printf_percent.o
         4          0          0          0          0          0   _printf_percent_end.o
        10          0          0          0          0          0   _printf_s.o
        82          0          0          0          0         72   _printf_str.o
        10          0          0          0          0          0   _printf_x.o
        22          0          0          0          0         92   _rserrno.o
        10          0          0          0          0         60   _sputc.o
      1006          4          0          0          0        184   aeabi_sdivfast.o
       216          6        148          0          0         80   bigflt0.o
      1456         30          0          0          0        336   btod.o
        16          0          0          0          0         68   exit.o
         6          0          0          0          0        136   heapauxi.o
         0          0          0          0          0          0   indicate_semi.o
        44         10         28          0          0         76   lc_numeric_c.o
         2          0          0          0          0          0   libinit.o
        18          0          0          0          0          0   libinit2.o
         2          0          0          0          0          0   libshutdown.o
         2          0          0          0          0          0   libshutdown2.o
         8          4          0          0         96         68   libspace.o
       122          0          0          0          0         72   lludiv10.o
        40          4          0          0          0         84   noretval__2sprintf.o
         8          4          0          0          0         68   rt_errno_addr_intlibspace.o
         8          4          0          0          0         68   rt_locale_intlibspace.o
         2          0          0          0          0          0   rtexit.o
        10          0          0          0          0          0   rtexit2.o
        40          0          0          0          0         60   rtudiv10.o
       176          4          0          0          0         80   strcmpv6m.o
        12          4          0          0          0         60   sys_exit.o
        62          0          0          0          0         80   sys_stackheap_outer.o
         2          0          0          0          0         68   use_no_semi.o
        46          0          0          0          0         60   cmpret.o
       124          4          0          0          0         72   d2f.o
       856         20          0          0          0        208   daddsub.o
       160          6          0          0          0         76   dcmpin.o
      1096         26        128          0          0        112   ddiv.o
       108         10          0          0          0         72   dfixi.o
        88          0          0          0          0         92   dflti.o
       584         26          0          0          0         84   dmul.o
        20          6          0          0          0         68   dnan2.o
       104          4          0          0          0        104   drlef.o
        96         12          0          0          0         72   dscalbn.o
       256          8          0          0          0         76   dsqrt.o
        84          4          0          0          0         60   f2d.o
       348          8          0          0          0        160   faddsub.o
        94          0          0          0          0         92   fflti.o
       176          4          0          0          0         80   fmul.o
        16          4          0          0          0         76   printf1.o
        94          0          0          0          0         68   retnan.o
         0          0          0          0          0          0   usenofp.o
        84         14          0          0          0        340   dunder.o
        44          4          0          0          0         60   fpclassify.o
       172          0          0          0          0         76   poly.o
      2516        206        136          0          0        236   pow.o
         0          0          8          0          0          0   qnan.o
        72          6          0          0          0         76   sqrt.o

    ----------------------------------------------------------------------
     12840        500        512          0         96       5072   Library Totals
        16          0          7          0          0          0   (incl. Padding)

    ----------------------------------------------------------------------

      Code (inc. data)   RO Data    RW Data    ZI Data      Debug   Library Name

      5586        128        233          0         96       2652   c_p.l
      4350        142        128          0          0       1632   fz_ps.l
      2888        230        144          0          0        788   m_ps.l

    ----------------------------------------------------------------------
     12840        500        512          0         96       5072   Library Totals

    ----------------------------------------------------------------------

==============================================================================


      Code (inc. data)   RO Data    RW Data    ZI Data      Debug   

     22392       1062        812        860       1860     147475   Grand Totals
     22392       1062        812        600       1860     147475   ELF Image Totals (compressed)
     22392       1062        812        600          0          0   ROM Totals

==============================================================================

    Total RO  Size (Code + RO Data)                23204 (  22.66kB)
    Total RW  Size (RW Data + ZI Data)              2720 (   2.66kB)
    Total ROM Size (Code + RO Data + RW Data)      23804 (  23.25kB)

==============================================================================

